:020000040800F2
:10800000E0DE0020A1810008A981000821AA000863
:10801000AD810008AF810008B181000800000000B8
:10802000000000000000000000000000B381000814
:10803000B581000800000000B7810008B981000880
:10804000BB810008BB810008BB810008BB81000820
:10805000BB810008BB810008BB810008BB81000810
:10806000BB810008BB810008BB810008BB81000800
:10807000BB810008BB810008379900083F990008C0
:10808000BB81000847990008BB810008BB8100083C
:10809000BB810008BB810008BB810008BB810008D0
:1080A000BB810008BB810008BB810008BB810008C0
:1080B00091940208BB810008BB810008BB810008C5
:1080C000BB810008BB810008BB810008BB810008A0
:1080D000BB8100089FA00208A7A00208AFA0020869
:1080E0009D9D0008BB810008BB810008BB81000882
:1080F000BB810008BB810008BB8100084F990008C4
:10810000BB810008BB810008BB810008BB8100085F
:108110008FA0020897A00208BB810008BB8100085D
:10812000BB810008BB810008BB810008BB8100083F
:10813000BB810008BB810008BB810008BB8100082F
:10814000BB810008BB810008BB810008BB8100081F
:10815000BB810008579900085F990008B7A0020882
:10816000BB810008BB810008BB810008BB810008FF
:10817000BB810008BB810008BB810008BB810008EF
:10818000BB810008BB810008DFF810D000F058FC6C
:1081900000480047F9BE0208AFF30080E0DE00208F
:1081A0000648804706480047FEE7FEE7FEE7FEE791
:1081B000FEE7FEE7FEE7FEE7FEE7FEE7299402089A
:1081C000898100082DE9F0410024061B254671F144
:1081D000000605DA01240027D0EB070067EB010158
:1081E000161E73F1000605DA0027D2EB07020125FF
:1081F00067EB030300F0C1FA86460E4617469C461D
:10820000AC4204D00025D0EB050E65EB010624B18D
:108210000020D2EB000760EB030C704631463A4673
:108220006346BDE8F081202A06DBCB17203A41FAED
:1082300002F043EAE07306E041FA02F3D040C2F1F3
:108240002002914008431946704740EA01039B070A
:1082500003D009E008C9121F08C0042AFAD203E0BB
:1082600011F8013B00F8013B521EF9D27047421E43
:1082700012F8013F002BFBD111F8013B02F8013B42
:10828000002BF9D17047421C10F8011B0029FBD1CB
:10829000801A704730B505460020034600E05B1C9D
:1082A000934205D2EC5CC85C201A01D1002CF6D1B7
:1082B00030BD2DE9FE4F804681EA0300C00F0C4619
:1082C000009021F0004123F00045B8EB0200A941E5
:1082D00005D24046214690461C460B46024623F0F6
:1082E0000040104347D0270DC7F30A00C3F30A51DB
:1082F0000290401A019040286BDAC3F3130040F457
:10830000801B0098924620B10023D2EB030A63EB56
:108310000B0B01985946C0F14002504600F05EFA3E
:1083200006460D4650465946019AFFF77CFF10EB72
:1083300008006141002487EA115284EAE7731A4376
:1083400040D0009A62B3019A012A4FEA075215DC25
:10835000001B61EB02014FF0004202EA0752CDE937
:108360000042001C41F5801132462B4600F0EAFA2B
:1083700003B0BDE8F08F40462146F9E7001B61EBF2
:108380000201001C41F5801300185B412018A2F582
:10839000001747EB030140EAD570B6196D4111E0B3
:1083A0006D084FEA360645EAC0754FEA0752001BD2
:1083B00061EB0201001C41F5801149084FEA3000D1
:1083C0000019514132462B4603B0BDE8F04F00F092
:1083D000AABA0098012240000023D0EB020263EB0E
:1083E000E073009821464FEAE074B8EB000061EBBF
:1083F0000401E9E783F000435BE781F0004158E7BF
:108400002DE9FE4F81EA030404F0004421F000410D
:1084100000944FF0000B23F0004350EA01045ED0BB
:1084200052EA03045BD0C3F30A54C1F30A552C4447
:10843000A4F2F3340194A0FB0254C1F3130141F4FC
:108440008011C3F3130343F4801301FB024400FBC8
:10845000034E840A970A44EA815447EA8357A4FBEF
:10846000076802958D0A05FB07854FEA932C04FBEC
:108470000C542705029D4FEA065847EA1637B5EB1C
:1084800008056EEB070C870E920E47EA811742EA49
:108490008312A7FB0201B6EB0B0164EB00042B0D6A
:1084A00043EA0C335E1844EB1C50DA465146E7FBB6
:1084B0000201C5F313044FEA0B3343EA14534FEAA6
:1084C0000432019C43EA0603A4F10C040294009CCC
:1084D000CDE900B400F036FA03B0BDE8F08F00201B
:1084E0000146F9E72DE9F04D81EA030404F0004B61
:1084F00021F0004514464FF0000A23F0004150EAF5
:10850000050220D054EA01021DD0C5F30A570246E5
:10851000C5F31303C1F31300C1F30A5640F48015E9
:1085200043F48013A7EB0608101BD64608F2FD386B
:1085300073EB050002D308F1010801E092185B41DA
:10854000B8F1000F03DA00200146BDE8F08D0020ED
:108550004FF48011064684460EE0171B73EB0507A7
:1085600005D3121B63EB050306434CEA010C4908D3
:108570004FEA300092185B4150EA0107EDD152EA10
:10858000030012D082EA040083EA0501084305D003
:10859000101BAB4106D20122002306E000224FF05F
:1085A000004302E06FF0010253101AEB06004CEB9F
:1085B000085110EB0A0041EB0B01BDE8F04D00F053
:1085C000B2B9F0B4CA17CB0F50405140C61841F1B0
:1085D00000054FEAC372314628004FF0960303D0DE
:1085E000B623F0BC00F071B930460021F9E70EB5B2
:1085F000C10F80EAE0700844CA07002140F233430B
:108600008DE80E000A460B4600F09CF903B000BD51
:108610000EB540F2334102910021CDE900110A4626
:108620000B4600F08FF903B000BD3EB5CA17CB0F63
:10863000002450405140C0186141DA0740F23343F2
:108640000094CDE901232246234600F07BF903B0D4
:1086500030BD10B500F0004420F00040C20DC0F362
:10866000160040F400007F2A02DA0020014610BD07
:108670000021962A03DCC2F19602D04002E0963A2D
:1086800000F0ACF8002CF2D00023D0EB030063EB39
:10869000010110BD70B5C1F30A5201F0004500247C
:1086A000C1F3130140F2FF3341F480119A4201DA21
:1086B000002070BD40F233439A42A2F2334203DC01
:1086C000524200F09AF800E090402C43F1D0404232
:1086D00070BD70B5C1F30A5201F000450024C1F32A
:1086E000130140F2FF3341F480119A4202DA002074
:1086F000014670BD40F233439A42A2F2334203DC9A
:10870000524200F07AF801E000F068F82C43F0D013
:108710000023D0EB030063EB010170BD00F00042C9
:1087200030F000400AD0C10D01F56071C0F31600B1
:1087300042EA0151C2084007114370470020014638
:10874000704701F0004330B421F0004150EA0102CB
:1087500006D00A0DA2F56072C1F31301002A02DCF3
:1087600030BC00207047440F44EAC104C100E01847
:1087700030BC00EBC25000F09FB82DE9F05F054619
:10878000002092469B4688460646814640241BE0D0
:10879000284641464746224600F02FF853465A469F
:1087A000C01A914110D311461846224600F016F81F
:1087B0002D1A67EB01084F4622460120002100F0E8
:1087C0000DF817EB00094E41201EA4F10104DFDC77
:1087D000484631462A464346BDE8F09F202A04DB3E
:1087E000203A00FA02F1002070479140C2F12003C4
:1087F00020FA03F3194390407047202A04DB203A03
:1088000021FA02F00021704721FA02F3D040C2F1B0
:108810002002914008431946704700000FB400231E
:1088200000B589B00CA900910B996FF00042CB60A4
:108830001E4B06931E4B07930423CDE901321D4ABC
:10884000089202466B46002000F0A6F909B05DF8D8
:1088500014FB70B586B006464FF0FF300091CDE9AD
:108860000101002015460C4604903246694604A8D2
:10887000FFF7D4FF02460498211825B108B1084635
:1088800000E020462860049800280DD0002A02DD70
:108890000098884208D0081B0094CDE901043246B4
:1088A000694604A8FFF7BAFF06B070BDD18D000875
:1088B000EF8D0008658A00080029A8BF7047401C9A
:1088C000490008BF20F00100704710B4B0FA80FCE6
:1088D00000FA0CF050EA010404BF10BC704749B123
:1088E000CCF1200421FA04F411FA0CF118BF012193
:1088F00021430843A3EB0C01CB1D4FEA00614FEA73
:10890000102042BF002010BC704700EBC350104441
:108910000029A4BF10BC7047401C490008BF20F0CC
:10892000010010BC704710B5141E73F1000408DA82
:10893000401C41F1000192185B411A4301D120F023
:10894000010010BD2DE9F04D92469B4611B1B1FAE0
:1089500081F202E0B0FA80F220329046FFF73EFF4B
:1089600004460F4640EA0A0041EA0B0153465A46C4
:10897000084313D0114653EA010019D0C8F1400250
:108980005046FFF73AFF05460E46504659464246C6
:10899000FFF724FF084305D0012004E020463946B4
:1089A000BDE8F08D0020054346EAE0762C433743CE
:1089B0000A986305E40AA0EB08000022FD0A44EAD5
:1089C00047540A3002D500200146E9E70105101995
:1089D0006941DDE9084500196941BDE8F04DA2E7AC
:1089E00070B521F0004303430CD0C1F30A550024B5
:1089F000D5EB040564EB0403D617AD1AB34102DBD3
:108A00000020014670BD201841EB025170BD0000EE
:108A100030B5041E71F1000404DB4FF00044404205
:108A200064EB0101141E73F1000405DB1C464FF0DA
:108A30000043524263EB0403994208BF904230BDA9
:108A4000064C074D06E0E06840F0010394E807009B
:108A500098471034AC42F6D3FFF79AFBC84403089A
:108A6000E8440308C0B24FF4F05100F03BBA0000F4
:108A70002DE9FF4F087883B09946FF2805D0491C9F
:108A80002D2804D00024002008E000200BE0012461
:108A9000F9E700EB800003EB4000491C0B78FF2B4B
:108AA000F7D104B1404200230293147819461D46C1
:108AB0002D2C01D02B2C04D1521C2D2C13D0002492
:108AC0000294AA461478FF2C0FD00A25A3FB057840
:108AD00001FB05814FF0000C03FB0C11521CE31944
:108AE0004AEB0101EEE70124EAE7814453EA010081
:108AF00002D019F5C87F06DA03980021C0E90011F9
:108B000007B0BDE8F08F0025AE4E2F46DFF8B882E3
:108B1000184600F0FBF9CDE90001B9F1000002DAD6
:108B2000C9F1000400E004460023A74A1AEB030B36
:108B300042EB045A12E0E00707D02A463346384693
:108B40004146FFF75DFC074688462A4633461046F5
:108B50001946FFF755FC05460E466410002CEAD175
:108B6000DDE90001B9F1000F5A46534606DAFFF776
:108B7000B9FC3A464346FFF7B5FC05E0FFF740FC79
:108B80003A464346FFF73CFC029A0AB181F00041A5
:108B9000039AC2E90001B3E72DE9FF4F1F468DB0EC
:108BA000D7E901464FF0FF382E2045464FF0000927
:108BB0000B90B9696D1C0E988847396A82468847C0
:108BC0000028F6D1BAF1FF3F0AD024F4D064002E79
:108BD00011DDBAF12B0F08D0BAF12D0F0BD102E045
:108BE000404611B08DE744F48064B9696D1C0E985D
:108BF00088478246761E6946600501D52D2000E033
:108C00002B208DF8000001F1010B0DF1200809E087
:108C1000B9696D1C0E98884782460F9844F4007419
:108C2000761E0560002E02DDBAF1300FF0D00B99F0
:108C30008A453ED144F0800406E00F99681CA9F1F2
:108C4000010944F400740860B9696D1C761E0E9821
:108C5000884782463028F0D02BE00B998A4505D111
:108C6000200603D444F08004761E18E0504622F01B
:108C70005DFD08B30DF11301761E44F400748B45BD
:108C800008D2AAF130000BF8010B200607D5A9F194
:108C9000010003E0200602D409F101008146A0058D
:108CA00002D50F99681C0860B9696D1C0E98884739
:108CB0008246002ED1DC53E0002E51DDBAF1650F63
:108CC00002D0BAF1450F4BD1A00549D5B9696D1C49
:108CD00024F44074761E0E9888478246002E0CDDE0
:108CE0002B2804D0BAF12D0F07D144F48074B96950
:108CF0006D1C0E9888478246761EE00501D52D2111
:108D000000E02B2108F8011BCDF82C8021E00DF1AB
:108D10002901761E44F4007488450CD2AAF1300073
:108D200010F0FF0088F8000002D10B99884509D99E
:108D300008F1010806E0E00501D5244801E042F20F
:108D40000F708146B9696D1C0E98884782460F984E
:108D50000560002E04DD504622F0E8FC0028D6D144
:108D6000F9690E988847FF208BF8000088F800000A
:108D70000020069007904B466A4608A906A8FFF710
:108D800077FEA00502D46FF001002AE714F0240F4B
:108D90000AD0E00714D1DDE906123868031D3B60F4
:108DA0000068C0E900120BE0DDE90601FFF7C9FC2D
:108DB0000146E00704D13868021D3A60006801608E
:108DC00028460EE7000014400000F03FF1D8FFFFF6
:108DD000426842B1016811F8013B23B1521EC0E95B
:108DE0000012184670470121C160881E7047426812
:108DF0005AB1C368016843B983688B4205D0491EE4
:108E0000521CC0E90012002070474FF0FF3070473D
:108E10002DE9F04D00231A461B1A8A4103DB00207E
:108E20000146BDE8F08DC1F30A52C1F3130141F4CC
:108E300080154FF0000BD10702D100186D41521E72
:108E40000027044640F2FF11384601EB620A3E4615
:108E50008046024600204FF48011FFF7CEFCC21975
:108E60007141BB1846EB0100B4EB030C75EB000C31
:108E700004D3E41A65EB000517460E46241908F1E1
:108E800001006D4180463428E3DDF91946EB060008
:108E9000091BA84103D24FF0FF32134601E0002224
:108EA00013461BEB070046EB0A51BDE8F04DFFF7F8
:108EB0003ABD000030B5041E71F1000404DB4FF030
:108EC0000044404264EB0101141E73F1000405DB11
:108ED0001C464FF00043524263EB04038B4208BF31
:108EE000824230BD7F2801D9002208E0064A02EB09
:108EF0005002C007127800D1120902F00F020120BF
:108F00009040084070470000884403080EB540F2C6
:108F1000334202920022CDE900221346FFF712FDF0
:108F200003B000BD70B58C1810F8015B15F0070395
:108F300001D110F8013B2A1106D110F8012B03E0F2
:108F400010F8016B01F8016B5B1EF9D12B0705D4FA
:108F50000023521E0DD401F8013BFAE710F8013B43
:108F6000CB1A921C03E013F8015B01F8015B521E5F
:108F7000F9D5A142D8D3002070BD10B502461078B3
:108F800003E012F8014B2318D8B20B1EA1F1010423
:108F9000A1B2F6D110BD000070B5ADF5287D044634
:108FA0000D460020A790A690002604EB44004549FA
:108FB00001EBC000408AA84203DC00200DF5287DAB
:108FC00070BD0020A69077E004EB44003D4B03EB1E
:108FD000C000028A04EB440003EBC00080892844EF
:108FE00081B2394800F010F90020A79011E004EB9D
:108FF0004400344901EBC0004068BDF89C12405C5D
:1090000001A9BDF89C228854BDF89C02401C80B286
:10901000A79004EB44002B4901EBC000008ABDF887
:109020009C128842E3DC04EB4400264A02EBC000B9
:10903000008A401E81B201A8FFF79FFF23490870F4
:1090400004EB44001F4901EBC000008A401E01A947
:10905000085C1E490978884226D10020A79016E0B6
:1090600004EB4400174901EBC0004068BDF89C12B6
:10907000405C04EB4401134A02EBC1018968BDF86E
:109080009C228854BDF89C02401C80B2A79004EB3F
:1090900044000C4901EBC000008A401EBDF89C1240
:1090A0008842DDDC012089E7642022F07DFDBDF8E7
:1090B0009802401C80B2A690BDF89802062883DB77
:1090C00000207BE7F41C03084C980020310A0020A4
:1090D0002DE9F043ADF5257D04460E460025002719
:1090E000A846A94604EB4400324901EBC000408A7F
:1090F000B04204DC00200DF5257DBDE8F08300259D
:1091000018E004EB44002B4901EBC0008068405D8F
:1091100004EB4401274A02EBC1014968485504EBBE
:109120004400114601EBC0004068405D0DF80500A9
:10913000681C85B204EB44001E4901EBC000008AA4
:10914000401EA842DDDC04EB44000A4602EBC000EE
:10915000008A401E81B26846FFF70FFF04EB44010E
:10916000144A02EBC101098A491E0DF801000027CB
:109170001BE004EB44000F4B03EBC000028A04EB3E
:10918000440003EBC0008089304481B2684600F09F
:109190004FF931462046FFF7FFFE012800D1AAE72C
:1091A000642022F001FD781C87B2062FE1DB00204D
:1091B000A1E70000F41C030808B5002000901DF092
:1091C000FFFB0F49087000F09BF80D480078242839
:1091D00004D0272807D028280FD109E0002109480A
:1091E00080F8191E09E00121064880F8191E04E0E4
:1091F0000221044880F8191E00BF00BF08BD00000E
:109200002C0A0020BC2200202DE9F04106460D4624
:1092100017460024012022F07FFA00202849088008
:109220000DE01DF0AFFB00F0800000B10BE001206D
:1092300022F0BAFC22480088401C214908802048BE
:109240000088C828EDDB00BF1D480088C82832DA36
:1092500010211C4801F0D8FB08211A4801F0D6FB68
:10926000E82000F031F8C5F3871000F02DF8A906CA
:10927000080E00F029F8002000F026F8002404E091
:10928000002000F021F8601C84B2042CF8DB0024DC
:1092900005E0FF2000F018F83055601C84B2BC4295
:1092A000F7DB1021074801F0B1FB002022F034FA6F
:1092B0000120BDE8F081002022F02EFA0020F8E71E
:1092C0002E0A00200000024010B5044600BF022113
:1092D0000A481DF085FC0028F9D0214607481DF0FA
:1092E0008BFC00BF012105481DF07AFC0028F9D055
:1092F00002481DF07EFCC0B210BD000000300140ED
:1093000010B5012022F008FA00201E4908800DE067
:109310001DF038FB00F0800000B10BE0012022F0CE
:1093200043FC18480088401C1649088015480088EE
:10933000C828EDDB00BF13480088C8281CDA1021BC
:10934000114801F061FB08210F4801F05FFB3D204F
:10935000FFF7BAFF2A20FFF7B7FF8020FFF7B4FF1F
:10936000A720FFF7B1FF1021074801F04FFB0020B5
:1093700022F0D2F9012010BD002022F0CDF900200A
:10938000F9E700002E0A00200000024070B50546F3
:109390000E460024012022F0BFF900202249088057
:1093A0000DE01DF0EFFA00F0800000B10BE00120AD
:1093B00022F0FAFB1C480088401C1B4908801A4810
:1093C0000088C828EDDB00BF17480088C82825DAC8
:1093D0001021164801F018FB0821144801F016FB73
:1093E0008420FFF771FF0020FFF76EFF0020FFF7DA
:1093F0006BFF0020FFF768FF002404E0285DFFF703
:1094000063FF601C84B2B442F8DB1021074801F00E
:10941000FDFA002022F080F9012070BD002022F02A
:109420007BF90020F9E700002E0A0020000002402E
:1094300070B506460C461546012022F06DF9294606
:109440003046FFF7A3FF08B9002070BD00201F4978
:1094500008800DE01DF096FA00F0800000B10BE0EE
:10946000012022F0A1FB19480088401C1749088000
:1094700016480088C828EDDB00BF14480088C828BB
:109480001EDA1021124801F0BFFA0821104801F03D
:10949000BDFA8320FFF718FFC4F38710FFF714FF0E
:1094A000A106080EFFF710FF0020FFF70DFF1021A7
:1094B000074801F0ABFA002022F02EF90120C4E7A2
:1094C000002022F029F90020BFE700002E0A00202A
:1094D0000000024030B502460020002304E012F8EC
:1094E000014B60405C1CE3B28B42F8DB30BD0000F6
:1094F00010B50446392022F099FDE0B222F0B6FD05
:10950000C4F3072022F0B2FDC4F3074022F0AEFD01
:10951000200E22F0ABFD4FF48051034801F076FAA3
:1095200020F00CFF10BD0000000402402DE9F041C6
:1095300007460E4614463A2022F078FDF0B222F09B
:1095400095FD301222F092FD4FF480510F4801F04A
:109550005DFA19E020F0F2FE05461D2D11D13846C6
:1095600000F0ACF805463B2022F060FD4FF480513E
:10957000064801F04BFA2F4434B12088284420805B
:1095800002E02846BDE8F081E4E700000004024064
:109590002DE9F04107460E4614463C2022F046FDD8
:1095A000F0B222F063FD301222F060FD4FF48051E2
:1095B000104801F02BFA0CB10020208019E020F0B7
:1095C000BDFE05461E2D11D1384600F02BF905468B
:1095D0003D2022F02BFD4FF48051064801F016FA91
:1095E0002F4434B120882844208002E02846BDE87A
:1095F000F081E4E70004024010B51DF0BBF808B1AB
:1096000000F02EF8302000F0A9F810BD10B5044687
:109610002146362000F08EF810BD10B5044614B176
:10962000204600F0ABF8342000F098F810BD10B5DB
:109630000446204600F0A2F820785C2802D020786A
:109640002F2803D10021642000F008F9322000F017
:1096500085F810BD10B5682000F04CF810BD000072
:1096600010B5222022F0E2FC22F0D5FC04464FF493
:109670008051024801F0CAF9204610BD00040240A2
:109680002DE9F04122F0C7FC044622F0C4FC054657
:1096900022F0C1FC064622F0BEFC07464FF4805182
:1096A000054801F0B3F944EA052040EA064040EAE3
:1096B0000760BDE8F08100000004024070B5044678
:1096C000272022F0B3FC22F0A6FC0646054646B150
:1096D00000BF22F0A0FC2070641C701EC0B2061EE9
:1096E000F7D14FF48051024801F090F9284670BD3F
:1096F0000004024010B504460C2022F097FC2046DE
:1097000022F0B4FCFFF7BCFF10BD000070B50446AA
:109710000A2022F08BFC204622F0A8FC22F07BFCE1
:1097200005464FF48051024801F070F9284670BD9B
:109730000004024070B505460C46284622F076FC2F
:10974000204622F093FC4FF48051034801F05EF96B
:1097500020F0F4FD70BD00000004024010B5044686
:10976000204622F063FC4FF48051034801F04EF98B
:1097700020F0E4FD10BD0000000402402DE9F0419E
:109780000646012022F052FC22F045FC43282BDA49
:109790002B20FFF7BBFF102826DA2F2022F046FCF3
:1097A000002022F063FC3220FFF7D8FF0446142C7F
:1097B0001AD1CF20FFF7AAFF0446ACB14C20FFF727
:1097C00099FF00EB042739464C2000F047F8502061
:1097D000FFF790FF00EB04273946502000F03EF8D9
:1097E0000021702000F03AF82F2022F01FFC35787D
:1097F000284622F03BFC09E0761C35785C2D01D030
:109800002F2D00D10025284622F030FC002DF3D169
:109810004FF48051024801F0F9F8BDE8F0810000F2
:109820000004024070B504462D2022F0FFFB22F018
:10983000F2FB0646054646B100BF207822F016FC32
:10984000641C701EC0B2061EF7D14FF4805102484E
:1098500001F0DCF8284670BD0004024070B50546F2
:109860000C460D2022F0E2FB284622F0FFFBE0B27E
:1098700022F0FCFBC4F3072022F0F8FBC4F30740FE
:1098800022F0F4FB200E22F0F1FB4FF4805102484D
:1098900001F0BCF870BD00000004024070B5024643
:1098A0000C46FF25FF2309E012F8010B80EA0501B1
:1098B0000648405C80EA03050548435C201EA4F18D
:1098C0000106B4B2F0D145EA032070BD581A03086E
:1098D000581B03082DE9F04103460C4600200146C1
:1098E000024606E013F8010B411842F10002601E27
:1098F00084B2002CF6DC080C40EA024C100C8DB24D
:109900001CEB050140F10002080C40EA024041183E
:109910006FEA010080B2BDE8F08130B50246002058
:10992000002305E012F8015B2C18E0B25C1CE3B2E6
:109930008B42F7DB30BD10B513F00EFE10BD10B535
:1099400013F0A8FD10BD10B513F074FD10BD10B5D7
:1099500013F0D0FD10BD10B515F042FD10BD10B5CF
:109960001CF0F6FA10BD00000246094B9A4201D2E3
:10997000084801E00648103801F000531BB1064BBF
:109980000B40C36002E0044B0B4083607047000053
:1099900010640240006002407D0F7D0F21B102681B
:1099A00042F00102026003E0026822F0010202605C
:1099B00070470000016821F0010101600021016091
:1099C00041608160C1600161212141614A49884251
:1099D00004D13D21484A103A91608CE04649183143
:1099E000884205D14FF47461434A103A916082E095
:1099F00041493031884205D14FF474113E4A103A42
:109A0000916078E03C494831884205D14FF074615B
:109A1000394A103A91606EE037496031884204D18A
:109A20003649354A103AD16065E033497831884289
:109A300004D13349304A103AD1605CE02E4990316C
:109A4000884204D12F492C4A103AD16053E02A4968
:109A5000A831884205D14FF03D51274A103AD160D4
:109A600049E02949884204D13D21274A083A11603A
:109A700041E025491831884205D14FF47461224AEA
:109A8000083A116037E020493031884205D14FF45F
:109A900074111D4A083A11602DE01B494831884273
:109AA00005D14FF07461184A083A116023E0164955
:109AB0006031884204D11149134A121F11601AE023
:109AC00011497831884204D10D490F4A121F1160A3
:109AD00011E00D499031884204D10A490A4A121F07
:109AE000116008E00849A831884204D14FF03D5187
:109AF000054A121F11607047106002403D000020AF
:109B0000400F002000003D201064024010B501F01D
:109B100080034BB122B1436943F08003436103E00A
:109B2000436923F08003436180290BD02AB1036885
:109B300001F01E042343036004E0036801F01E04E7
:109B4000A343036010BD000010B500220268134B50
:109B50001A40CC680B6823434C6923438C69234328
:109B6000CC6923430C6A23434C6A23438C6A234306
:109B70004C6B23438C6B23431A430260426922F0EF
:109B80000702D1E90B3423431A4342610B69436056
:109B90004B6883608B68C36010BD00003F801CF081
:109BA0001CB50024012120201CF0F0FD3020009085
:109BB00001208DF8040000208DF8060003208DF8A8
:109BC000050000208DF807006946164800F0A8FE41
:109BD0003021144800F01AFF0021134880F8441780
:109BE00000201249887001204870C8704FF4FA7044
:109BF000886000F01DF80C48007F592810DD2420F3
:109C000009491C314871082008713020C87014209F
:109C100088702020487000210348017700F04AF83E
:109C20001CBD000000140240BC320020003A00209D
:109C30001CB522F0C1F8D02022F08AF822F0F0F80A
:109C4000002022F085F822F0EBF822F0B5F8D120C0
:109C500022F07EF822F0E4F800240EE0062C05DA6B
:109C6000012022F045F80DF8040004E0002022F065
:109C70003FF80DF80400601CC4B2072CEEDB22F0A4
:109C8000B5F89DF806000A4948719DF8050008716D
:109C90009DF80400C8709DF8020088709DF80100CE
:109CA00048709DF8001002481C3801771CBD000068
:109CB000D83200201CB500241D48007F8DF800001C
:109CC0001B481C3040788DF8010019481C30807802
:109CD0008DF8020001208DF8030015481C30C07873
:109CE0008DF8040012481C3000798DF805001048EA
:109CF0001C3040798DF8060022F05EF8D02022F06A
:109D000027F822F08DF8002022F022F822F088F8BF
:109D100000BF07E01DF8040022F01AF822F080F8D6
:109D2000601CC4B2072CF5DB22F060F81CBD0000FB
:109D3000BC32002070B502460C460025002309E025
:109D400012F8010B80EA05010648405C80EA030531
:109D50000548435C201EA4F10106B4B2F0D145EAE7
:109D6000032070BD581A0308581B030810B5044699
:109D70000B460021072A00DD072244EA04200146A1
:109D80002BB901FA02F081B20912084610BD012B6D
:109D900002D11141C8B2F9E700BFF7E7704710B52B
:109DA00004460B460021072A00DD072244EA04206E
:109DB000014613B91141C8B210BD012B05D101FAFA
:109DC00002F081B209120846F6E700BFF4E700008E
:109DD000F0B5ADF21C5D04460D460020CDF8180527
:109DE000CDF81405002604EB4400584901EBC000EF
:109DF000408AA84203DC00200DF21C5DF0BD00206B
:109E0000CDF814059AE051480122C168504800F08D
:109E1000A3FA4E48406800788DF800009DF80000D5
:109E200038287DD104EB4400484B03EBC000C068E8
:109E300004EB4403454F07EBC3031B8A03FB0501F7
:109E400004EB44003B4603EBC000028A404800F0AC
:109E500083FA0020CDF8180512E004EB44003B49DA
:109E600001EBC0004068BDF81815405CBDF818252E
:109E70000DF80200BDF81805401C80B2CDF8180599
:109E800004EB4400314901EBC000008ABDF818150D
:109E90008842E2DC04EB44002C4A02EBC000008A5A
:109EA000401E81B2684600F01DFB064604EB4400EC
:109EB000264901EBC000008A401E1DF80000B04298
:109EC00033D10020CDF8180520E004EB44001F49F1
:109ED00001EBC0004068BDF81815415C04EB44007C
:109EE0001A4A02EBC0008068BDF81825024404EB52
:109EF0004400164B03EBC000008A401E6843115417
:109F0000BDF81805401C80B2CDF8180504EB4400DC
:109F10000E4901EBC000008A401EBDF8181500E094
:109F200003E08842D1DC012066E7642021F03CFE9A
:109F3000BDF81405401C80B2CDF81405BDF8140519
:109F40000628FFF660AF002056E7000044CB020869
:109F5000906A00202DE9F041ADF5A36D04460E4650
:109F600000250027A8460020009004EB4400474944
:109F700001EBC000408AB04204DC00200DF5A36D67
:109F8000BDE8F08100210846FFF722FF01287AD1C1
:109F9000002520E004EB44003C4901EBC000806850
:109FA000411904EB4400394A02EBC000008A401E0C
:109FB0007043085C04EB440102EBC1014968485559
:109FC00004EB4400114601EBC0004068405D01A96C
:109FD0004855681C85B204EB44002C4901EBC000D5
:109FE000008AA842D6DC00274BE004EB4400274B54
:109FF00003EBC000C06804EB4403DFF890C00CEB37
:10A00000C3031B8A03FB060104EB4400634603EB16
:10A01000C000008A401E82B21D4800F01FFA04EB07
:10A0200044001A4A02EBC000008A401E81B201A817
:10A0300000F058FA009004EB4400144A02EBC00010
:10A04000C06804EB4402114B03EBC202128A1044B5
:10A0500004EB440203EBC202128A02FB0600411E1B
:10A060000122684600F0FAF931462046FFF7B0FEBB
:10A07000012801D182E706E0642021F095FD781CDB
:10A0800087B2062FB1DB002078E7000044CB02083E
:10A09000906A0020F0B5ADF21C5D00250024002080
:10A0A0000190002600210120FFF792FE4B4890F816
:10A0B0000C6E00204A49088080E000256FE00024F3
:10A0C00014E04748008800EB4000464951F8300052
:10A0D000005D4349098801EB4101424A02EBC1019D
:10A0E0004968085502A90855601C84B23C4800889C
:10A0F00000EB40003B4901EBC000008A401EA0423B
:10A10000DFDC3748008800EB40000A4602EBC00065
:10A11000008A401E81B202A800F0E4F901903048A4
:10A12000008800EB40002F4B03EBC000C0682C4BB5
:10A130001B8803EB43032B4F07EBC3031B8A03FB73
:10A1400005012748008800EB40003B4603EBC000B8
:10A15000008A401E82B2244800F080F9204800881E
:10A1600000EB40003A4602EBC000C0681C4A12886F
:10A1700002EB42023B4603EBC202128A1044184A29
:10A18000128802EB420203EBC202128A02FB0500B4
:10A19000411E012201A800F061F9681C85B2104837
:10A1A000008800EB40000F4901EBC000408AA84244
:10A1B00085DC0B480088401C094908800848008855
:10A1C0000D28FFF67AAF054880F80C6E00210120BB
:10A1D000FFF7C0FE0DF21C5DF0BD0000BC220020A8
:10A1E0001000002044CB0208906A00201CB5012119
:10A1F00008461CF0CBFA01208DF8040002208DF8EF
:10A20000050000208DF8060001208DF807001820B9
:10A2100000906946144800F083FB0522114612485D
:10A2200000F0C6FB052206210F4800F0C1FB052205
:10A2300007210D4800F0BCFBA020009002208DF803
:10A24000040003208DF8050000208DF806008DF82D
:10A2500007006946044800F063FB4020009069460F
:10A26000014800F05DFB1CBD000002402DE9F843F1
:10A27000002400250027002000908046FFF7B6FF4D
:10A2800000F0BCF80A2021F08FFC6E4608212D4812
:10A2900000F0BAFB10212B4800F0B8FB062000F0BC
:10A2A00091F80821274800F0B1FB0821254800F06B
:10A2B000ABFB1021234800F0A9FB012000F082F83D
:10A2C000002000F07FF808211E4800F09FFB1E4888
:10A2D000D0F82C11B0F83021B0F8320102FB001098
:10A2E000B0F5003F02D900BE00BFFEE71748006886
:10A2F00008B9FFF7CFFE00201549088017E00024B9
:10A3000006E0134908782146FFF762FD601C84B21D
:10A310000F48008800EB40000B4901EBC000408A69
:10A32000A042EEDC0A480088401C09490880084821
:10A3300000880D28E3DB0748D0F81802054988712A
:10A34000BDE8F8830000024044CB02081C024342EF
:10A3500010000020BC1200202DE9F04105460C46FB
:10A3600016460027012021F0D4F90821144800F0F6
:10A370004BFB1021124800F049FB032000F022F8AB
:10A38000C4F3074000F01EF8C4F3072000F01AF8E9
:10A39000E0B200F017F800BF06E0002000F012F86D
:10A3A00028706D1C781C87B2B742F6DB0821044880
:10A3B00000F02CFB002021F0ACF9BDE8F08100009A
:10A3C0000000024010B5044600BF02210A481CF0FC
:10A3D00007FC0028F9D0214607481CF00DFC00BFFF
:10A3E000012105481CF0FCFB0028F9D002481CF0B4
:10A3F00000FCC0B210BD00000030014000B585B0C7
:10A40000012108031CF012FA13481CF0BDFB0020C8
:10A41000ADF80000ADF80400ADF80600ADF8080096
:10A420004FF40070ADF80A000820ADF80C000020D1
:10A43000ADF80E000720ADF810004FF48270ADF8B3
:10A440000200694604481CF0D9FB012102481CF0B7
:10A450008FFB05B000BD0000003001402DE9F04148
:10A4600005460C4616460027012021F052F9082126
:10A470001B4800F0C9FA1021194800F0C7FA06205D
:10A48000FFF7A0FF0821164800F0C0FA0821144881
:10A4900000F0BAFA1021124800F0B8FA0220FFF7D3
:10A4A00091FFC4F30740FFF78DFFC4F30720FFF7C8
:10A4B00089FFE0B2FFF786FF00BF05E02878FFF7CD
:10A4C00081FF6D1C781C87B2B742F7DB0821044876
:10A4D00000F09CFA002021F01CF9BDE8F08100009A
:10A4E0000000024010B50246107803E012F8014B5C
:10A4F0002318D8B20B1EA1F10104A1B2F6D110BDF0
:10A500002C48807D012854D100212A4881752A4891
:10A510000078C0B901202849087028480068C000A8
:10A520002749D1F8301240EA81002549D1F82C1290
:10A5300040EA41002249D1F8281208430F21814303
:10A540002048017017E000201B4908701B48006874
:10A55000C0001B49D1F8301240EA81001849D1F8F7
:10A560002C1240EA41001649D1F8281208430F2165
:10A5700081431548017013480078134909788842CF
:10A5800017D1104800781149087008460078104922
:10A59000097888420DD00D480078064908740B48A8
:10A5A00000780B4908700948007810B10120014972
:10A5B000C8737047BC120020DE0A002034024242F9
:10A5C00000004242DF0A0020E00A0020E10A0020E9
:10A5D000DD0A002010B5ADF57C7D00247CA000686C
:10A5E000FB9000200090FFF707F814287CD17948F1
:10A5F000FFF71DF87849087008460078142874D1D0
:10A60000FFF728F80021754A03C2BDF80000FEF7E5
:10A610006FFF6A464FF4FA7101A8FEF787FF70A139
:10A6200001A821F09FFC704908800846008810B3FB
:10A6300000BF04E000216D480155601C84B2282C45
:10A64000F8DB01A9684A1288881869A121F08AFC00
:10A6500068490880002409E063480088C01C204441
:10A6600001A9095C61480155601C84B261480088F9
:10A67000001FA042F0DC60A101A821F073FC5A4940
:10A6800008800846008820B3002405E000215748D0
:10A6900028300155601C84B2282CF7DB01A9524AEE
:10A6A0001288881852A121F05DFC524908800024CC
:10A6B0000AE04D4800880830204401A9095C4B4855
:10A6C00028300155601C84B24A4800880938A042ED
:10A6D000EFDC4CA101A821F045FC43490880084665
:10A6E000008830B3002407E06BE05BE000213F48C6
:10A6F00050300155601C84B2142CF7DB01A93A4A92
:10A70000128888183AA121F02DFC3A4908800024CB
:10A710000AE0354800880C30204401A9095C334820
:10A7200050300155601C84B2324800880D38A04278
:10A73000EFDC38A101A821F015FC2B490880084660
:10A74000008820B3002405E0002028494639085538
:10A75000601C84B2322CF7DB01A9234A12888818C6
:10A7600023A121F0FFFB2349088000240AE01E48B2
:10A770000088801D204401A9085C1C494639085501
:10A78000601C84B21B480088C01FA042EFDC00217F
:10A790000320FFF7DFFB0120FEF738FF01200DF556
:10A7A0007C7D10BD0C480078422803D10948FEF793
:10A7B00034FF0BE00120FEF729FF00200649087056
:10A7C00004E000211548C17621F060FB00BFE6E7F8
:10A7D0000D0A0000480A0020380A0020400A002024
:10A7E00041504E3D000000005E0A0020E03A00208B
:10A7F0003B0000005C0A0020574946494E414D4548
:10A800003D0000005749464950415353574F524469
:10A810003D0000005345525645523D00BC320020D9
:10A8200010B504463548844208D1012108461BF082
:10A83000BDFF002101201BF0B9FF5EE030488442DB
:10A8400008D1012102201BF0B1FF002102201BF0E2
:10A85000ADFF52E02B48844208D1012104201BF0B7
:10A86000A5FF002104201BF0A1FF46E026488442FA
:10A8700008D1012108201BF099FF002108201BF0BE
:10A8800095FF3AE02148844208D1012110201BF0B5
:10A890008DFF002110201BF089FF2EE01C48844210
:10A8A00008D1012120201BF081FF002120201BF076
:10A8B0007DFF22E01748844208D1012140201BF08F
:10A8C00075FF002140201BF071FF16E01248844202
:10A8D00008D1012180201BF069FF002180201BF09E
:10A8E00065FF0AE00D48844207D1012180151BF065
:10A8F0005DFF0021A0151BF059FF10BD00000240B4
:10A900000004024000080240000C02400010024017
:10A910000014024000180240001C024000200240C7
:10A92000F0B50A4600210023002400BF3DE00125C8
:10A9300005FA01F3156805EA03049C4234D1056861
:10A940004F000326BE40B543056015794E00B54063
:10A950000668354305601579012D02D01579022D61
:10A9600016D185684F000326BE40B54385605579F2
:10A970004E00B540866835438560456801268E40A7
:10A98000B5434560456896798E40B6B2354345601B
:10A99000C5684F000326BE40B543C560D5794E005B
:10A9A000B540C6683543C560491C1029BFD3F0BD0A
:10A9B000F0B5002300244D07ED0E02FA05F3CE108A
:10A9C00000F1200555F826504E07F70E0F26BE4021
:10A9D000B543CF1000F1200646F82750CE1000F105
:10A9E000200555F8265045EA0304CE1000F1200555
:10A9F00045F82640F0BD0246002013690B400BB11C
:10AA0000012000E0002070474183704701837047B8
:10AA10000249087C0021014A11747047BC120020D1
:10AA20000E48006800F0010000B100BE012080F374
:10AA3000138800BF00BFBFF34F8F0848E438006899
:10AA400000F4E06006490843001D0449E439086049
:10AA5000BFF34F8F00BF00BFFEE70000F0ED00E046
:10AA60000000FA054AF6AA20014908607047000074
:10AA70000030004030B502460024002305E012F803
:10AA8000015B2819C4B2581CC3B28B42F7DB604289
:10AA9000C0B230BD10B5002421F0F8F9642021F0D7
:10AAA00083F810BD2DE9F043ADF2DC7D80460E4603
:10AAB000144699460025002783A00068CDF8D807E2
:10AAC00000200190042C7CDC80480079302101EBCF
:10AAD000101004EBC40101EB04117D4A114408710C
:10AAE0007A48007900F00F00303004EBC40101EB2C
:10AAF0000411114448717548C078302101EB1010E1
:10AB000004EBC40101EB0411114488716F48C07853
:10AB100000F00F00303004EBC40101EB04111144CC
:10AB2000C871FEF769FD14287ED16A4800781428A0
:10AB300009D004EBC40101EB0411654A8818FEF743
:10AB400076FD644908706348007814286DD1B6F525
:10AB50007A7F01DD4FF47A76FEF77CFD00215E4AB4
:10AB600003C25D480068FEF7C3FC5848C078302136
:10AB700001EB10108DF808005448C07800F00F0069
:10AB800030308DF809005148807801EB10108DF8B5
:10AB90000A004E48807800F00F0030308DF80B002E
:10ABA0004A48407801EB10108DF80C004748407877
:10ABB00000F00F0030308DF80D0044481C38007F45
:10ABC00000E07CE001EB10108DF80E003F481C38CF
:10ABD000007F00F00F0030308DF80F00B9F1000F4A
:10ABE00003D154208DF8100005E0B9F1010F02D116
:10ABF00052208DF810003A208DF8110000252CE02D
:10AC0000284605EBD071491018F801100F110A20E1
:10AC100097FBF0F0C0EBC00107F130000844C1B26F
:10AC200002AA05F10A0001E043E02EE01154284693
:10AC300005EBD071491018F8011001F00F070A2038
:10AC400097FBF0F0C0EBC00107F130000844C1B23F
:10AC500005F10B001154A81C85B2B5EB460FCFDBF4
:10AC60000A2000EB460081B201AA02A8FEF790FC80
:10AC700001AA02210DF5FB60FEF78AFC0120FEF718
:10AC8000C5FC00201349087019E0124800784228DA
:10AC900008D104EBC40101EB04110D4A8818FEF73A
:10ACA000BCFC0CE00120FEF7B1FC00200949087053
:10ACB00005E0002105481C38C17621F0E7F80DF2C7
:10ACC000DC7DBDE8F08300000D0A0000D8320020D2
:10ACD000600A0020380A0020400A002070B5B8B091
:10ACE00000213791369135913491339132913191E0
:10ACF000309100222E922F922C922D922B912A91FC
:10AD0000299128912791269125912491239115919C
:10AD1000149113911291119110910F919FEDFE0AD0
:10AD20008DED0E0AFDA006C8CDE90C12FDA006C8E7
:10AD3000CDE90A12BAE0FD48807858B30020FB49FB
:10AD40008870FB48B0F88007FA490968C1F57A7144
:10AD500088421FD1F7480068C0F57A7081B2F44884
:10AD6000A0F878170021F348001FFEF717FEF249FC
:10AD7000F048001FFEF7F8FD0120F04908704FF47D
:10AD80007A70EC498C39C1F88C000121E948001F28
:10AD9000FEF704FEE548807B50B30021E348817351
:10ADA000E7484088E3498C39496CC1F57A7188429B
:10ADB0001ED1E0488C38406CC0F57A70E049083903
:10ADC00048800021DB484C38FEF7E8FDDD49D948D2
:10ADD0004C38FEF7C9FD0120DB4908704FF47A7149
:10ADE000D4488C3841640121D2484C38FEF7D6FD56
:10ADF000CE48807E50B30021CC488176D0488088F0
:10AE0000CC498C394969C1F57A7188421ED1C9484B
:10AE10008C384069C0F57A70C949083988800021AA
:10AE2000C4487C38FEF7BAFDC849C2487C38FEF7F2
:10AE30009BFD0120C64908704FF47A70BD498C39DA
:10AE400048610121BB487C38FEF7A8FDB74890F85F
:10AE5000260058B30021B54880F82610B848C088AD
:10AE6000B4498C39C96AC1F57A7188421ED1B1489A
:10AE70008C38C06AC0F57A70B1490839C8800021A1
:10AE8000AC486438FEF78AFDB249AA486438FEF738
:10AE90006BFD0120B04908704FF47A70A5498C39D8
:10AEA000C8620121A3486438FEF778FD9F48817885
:10AEB000807B01449D48807E01449C4890F8260098
:10AEC000084400287FF437AF0BF088BC9B4800781B
:10AED00020B10021994801702B9119E09A4800781F
:10AEE00028B100209849087001212B9110E0984862
:10AEF000007828B100209649087002202B9007E0C6
:10AF00009548007820B100209349087003212B91C7
:10AF10009DF8AC1001EB4100C0EBC1108F4911F856
:10AF20003000C12836D19DF8AC1001EB4100C0EBD8
:10AF3000C1108A4901EBC000807808282AD101217C
:10AF40007B4880F8D0179DF8AC0030B101280AD0BA
:10AF500002280ED0032818D111E04FF48041804818
:10AF6000FFF752FD11E04FF400517D48FFF74CFD13
:10AF70000BE04FF480517A48FFF746FD05E04FF4AF
:10AF800000617748FFF740FD00BF00BF0020754912
:10AF9000086099E765480C389DF8AC1010F811006E
:10AFA0000121B1EBD01F4BF074826F48C07EB8B165
:10AFB000634908399DF8AC0031F8101009919DF8EB
:10AFC000AC0000EB4001C1EBC010644901EBC001D3
:10AFD000012308919DF8AC20DDE90801FFF762FD2F
:10AFE0009DF8AC0000EB400101EB00105F4901EB64
:10AFF000001081792A919DF8A80009288BF014820D
:10B00000DFE810F028510900B314DD238E30B93287
:10B01000CA362542304D9DF8AC0000EB4001C1EB33
:10B02000C0104E4901EBC00041780846099100214B
:10B0300012F01CF9C1B22691002134911CE09DF858
:10B04000AC0000EB400101EB0010484901EB00119E
:10B050003031BDF8D00001EB001041789DF8980028
:10B06000814204D1BDF8D000C1B2269112E0BDF8F2
:10B07000D000401C81B234919DF8AC1001EB41002E
:10B0800000EB0110394901EB0010C179BDF8D00087
:10B090008142D4DC00BF9DF8AC1001EB4100C0EB55
:10B0A000C1102E4901EBC000807800F0F000A0280C
:10B0B0000DD19DF8AC0000EB4001C1EBC010274959
:10B0C00001EBC000807800F00F0127910AE09DF8A5
:10B0D000AC0000EB4001C1EBC010204901EBC00007
:10B0E00081782791BDF89C0008B9102127919DF81F
:10B0F000AC1001EB4100C0EBC110184901EBC001DD
:10B10000BDF89C00401C095C2491BDF89C00401CCB
:10B1100081B209912CE0000000000000016932308A
:10B12000313030000169323045303000E83E0020D7
:10B13000BC6200208C6002400088002012000020C9
:10B140003C6A0020008020101300002020800010A6
:10B15000140000200088001015000020A8780020AE
:10B160000018024088024242BC32002014410020F4
:10B170009DF8AC0000EB4001C1EBC010FE4901EBB3
:10B18000C0010891DDE9080112F002FD35909DF83B
:10B19000AC0000EB4001C1EBC010F74901EBC0016E
:10B1A000BDF89C00801C095CBDF8D400814242F0CF
:10B1B000DA839DF8AC0000EB4001C1EBC010EE4912
:10B1C00001EBC0004078002842F3CD839DF8AC002D
:10B1D00000EB4001C1EBC010E74901EBC001BDF835
:10B1E0009C00C01C0A5C9DF8AC0040F2231110FBCF
:10B1F00001F0E24901EBC00118319DF8980000EB25
:10B20000C00001EB001080F83C200021DC4A9DF8D2
:10B21000AC0002EB00129DF898001154D94890F848
:10B220002000012840D19DF8AC0000EB400101EB6B
:10B230000010D54901EB001030309DF8981000EB5C
:10B240000110801C0990007820F08000803009995E
:10B250000870BDF89000B62814D0C52819D0D5289C
:10B2600002D0D9281CD106E0BDF89C00032801DAE1
:10B270000020249017E0BDF89C00032801DA00208C
:10B28000249010E0BDF89C00032801DA00202490EF
:10B2900009E0BDF89C00032801DA0020249002E0B8
:10B2A0000020249000BF00BFBDF89000C52801F029
:10B2B000558418DCB5287CD00DDC112802F0ED8116
:10B2C000122802F02C82132802F0B582B22842F034
:10B2D000498301F00FBCB62801F0DB82B92869D0A0
:10B2E000C328F4D1FEE3D92865D007DCCA287CD076
:10B2F000CE2802F0E680D528E9D109E0E12802F065
:10B30000F380E52802F00381E728E0D102F0AEB92E
:10B310009DF8AC1001EB4100C0EBC110964901EB68
:10B32000C000C178994880F8121E9DF8AC1040F218
:10B33000231011FB00F0914901EBC00118319DF879
:10B34000980000EBC00001EB001001789DF8AC0004
:10B3500040F2231210FB02F0884A02EBC000407951
:10B3600081427DDA9DF8AC1001EB410000EB011049
:10B37000854901EB001030309DF8981000EB01106A
:10B38000801C0990814890F8121E0120A0EBD1107A
:10B390000999097860F30001099801707B4890F8D9
:10B3A000120EC0F34010E0BB9DF8AC1001EB410061
:10B3B00002E0FDE3FDE3FDE300EB0110724901EB68
:10B3C000001030309DF8981000EB01108078C0F329
:10B3D000401030B39DF8AC0000EB400101EB0010D1
:10B3E000694901EB0010303000E0FCE39DF8981053
:10B3F00000EB0110801C0990007820F00200801CF6
:10B40000099908709DF8AC0040F2231110FB01F07F
:10B41000114601EBC00018309DF8981001EBC101F6
:10B4200000E00EE000EB011018300990007820F0E9
:10B430000200801C099908709DF8AC100220FEF7EC
:10B4400089FD00219DF8AC0040F2231210FB02F0B0
:10B450004A4A02EBC000017102229DF8AC0000E0F4
:10B4600021E040F2231110FB01F0444901EBC0013F
:10B4700018319DF8980000EBC00001EB001002703D
:10B48000B6229DF8AC0040F2231110FB01F03B49BD
:10B4900001EBC00018309DF8981001EBC10100EBE2
:10B4A00001104271FEE3394890F8120EC0F3C0005B
:10B4B00090B9E5229DF8AC0040F2231110FB01F099
:10B4C0002E4901EBC00018309DF8981001EBC10126
:10B4D00000EB01104271E5E39DF8AC1001EB410077
:10B4E00000EB0110284901EB001030309DF8981056
:10B4F00000EB0110801C0990244890F8120E0121E5
:10B50000A1EBD01009990A7860F300020A709DF847
:10B51000AC1001EB410000EB01101B4901EB0010E6
:10B5200030309DF8981000EB0110801C09901748EE
:10B5300090F8120E42090998007862F341000999C7
:10B5400008709DF8AC0000EB400101EB00100E49C3
:10B5500001EB001030309DF8981000EB011080785E
:10B56000C0F340029DF8AC0040F2231110FB01F043
:10B57000024901EBC0000BE0A8780020D445002070
:10B58000483F0020BC12002014410020BC220020B3
:10B5900018309DF8981001EBC10100EB0110007EFE
:10B5A000C0F34000824277D09DF8AC0040F22311F6
:10B5B00010FB01F0FE4901EBC00018309DF8981017
:10B5C00001EBC10100EB0110183009909DF8AC109F
:10B5D00001EB410000EB0110F64901EB00103030A7
:10B5E0009DF8981000EB01108078420809980078C7
:10B5F00062F34100099908709DF8AC1001EB41001D
:10B6000000EB0110EB4901EB001030309DF8981071
:10B6100000EB01108078C0F34000E0B3D9229DF820
:10B62000AC0040F2231110FB01F0E14901EBC00036
:10B6300018309DF8981001EBC10100EB0110427128
:10B64000DD4890F8A00800287BD19DF8AC0040F2BE
:10B65000231110FB01F0D64901EBC00018309DF812
:10B66000981001EBC10100EB011090F87E0000285A
:10B6700067D011239DF8AC0040F2231110FB01F0BC
:10B68000CB4901EBC00118319DF8980000EBC000D8
:10B6900001EB001001E055E043E190F87F0040F23B
:10B6A000231110FB01F0C24901EBC00118319DF8D4
:10B6B000AC0040F2231210FB02F0BD4A02EBC002C4
:10B6C00018329DF8980000EBC00002EB001090F8D3
:10B6D000800000EBC00001EB001080F87730F3230E
:10B6E0009DF8AC0040F2231110FB01F0B04901EBD2
:10B6F000C00118319DF8980000EBC00001EB00106C
:10B7000090F87F0040F2231110FB01F0A84901EBF3
:10B71000C00118319DF8AC0040F2231210FB02F07A
:10B72000A34A02EBC00018309DF8982002EBC20239
:10B7300000EB021090F8800000EBC00001EB00105D
:10B740004371E9E001229DF8AC0040F2231110FBA7
:10B7500001F0974901EBC00118319DF8980000EB0A
:10B76000C00001EB00104273D9229DF8AC0040F2FA
:10B77000231110FB01F08E4901EBC00118319DF837
:10B78000980000EBC00001EB0010427101229DF80F
:10B79000AC0040F2231110FB01F0854901EBC00021
:10B7A00018309DF8981001EBC10100EB011080F8F2
:10B7B0003E20814890F8A008E8BB9DF8AC0040F21C
:10B7C000231110FB01F07A4901EBC00018309DF8FD
:10B7D000981001EBC10100EB011090F87E0050B30E
:10B7E0009DF8AC1040F2231011FB00F0704901EB02
:10B7F000C00118319DF8980000EBC00001EB00106B
:10B8000090F87F1001EB410000EB0110694901EB5A
:10B81000001130319DF8AC0040F2231210FB02F011
:10B82000634A02EBC00218329DF8980000EBC0009A
:10B8300002EB001000E06FE090F8800001EB0010D8
:10B84000801C0990007820F00402099802700023FF
:10B850009DF8AC0040F2231110FB01F0544901EBBC
:10B86000C00018309DF8981001EBC10100EB0110E9
:10B8700090F87F0040F2231110FB01F04C4901EBDE
:10B88000C00018309DF8AC1040F2231211FB02F1F9
:10B89000474A02EBC10218329DF8981001EBC10132
:10B8A00002EB011191F8801001EBC10100EB0110D6
:10B8B00080F87730F3239DF8AC0040F2231110FBA1
:10B8C00001F03B4901EBC00018309DF8981001EBE6
:10B8D000C10100EB011090F87F0040F2231110FB32
:10B8E00001F0334901EBC00018309DF8AC1040F274
:10B8F000231211FB02F12E4A02EBC10118319DF80F
:10B90000982002EBC20201EB021191F8801001EBCA
:10B91000C10100EB011043719DF8AC100220FEF74D
:10B9200019FB9DF8AC0000EB400101EB0010214930
:10B9300001EB001130319DF8980001EB0010807888
:10B9400000F001029DF8AC0040F2231110FB01F061
:10B95000174901EBC00018309DF8981001EBC101A8
:10B9600000EB0110007E00F0010082427DD09DF8C6
:10B97000AC0040F2231110FB01F00D4901EBC000B7
:10B9800018309DF8981001EBC10100EB0110183040
:10B9900009909DF8AC0000EB400101EB0010054957
:10B9A00001EB001030309DF8981000EB011005E01D
:10B9B000D445002014410020BC3200208078099931
:10B9C0000A7860F300020A709DF8AC0000EB4001B9
:10B9D00001EB0010FE4901EB001030309DF898108B
:10B9E00000EB0110807800F00100E8BB9DF8AC008E
:10B9F00000EB400101EB0010F54901EB0010303085
:10BA00009DF8981000EB01108078C0F3401068B3E7
:10BA10009DF8AC0040F2231110FB01F0ED4901EB61
:10BA2000C00018309DF8981001EBC10100EB011027
:10BA300090F83E00D0B99DF8AC0040F2231110FB05
:10BA400001F0E44901EBC00018309DF8981001EBBB
:10BA5000C10100EB0110407B40B99DF8AC0000EB48
:10BA6000400101EB001002E05BE034E23BE0D8492A
:10BA700001EB001030309DF8981000EB0110807839
:10BA8000C0F3400078BB01229DF8AC0040F22311C6
:10BA900010FB01F0CF4901EBC00118319DF898006F
:10BAA00000EBC00001EB00104273D9229DF8AC00FE
:10BAB00040F2231110FB01F0C64901EBC00118311F
:10BAC0009DF8980000EBC00001EB001042710122CC
:10BAD0009DF8AC0040F2231110FB01F0BD4901EBD1
:10BAE000C00001E0FDE308E018309DF8981001EB7C
:10BAF000C10100EB011080F83E2000229DF8AC004F
:10BB000040F2231110FB01F0B24901EBC0001830E4
:10BB10009DF8981001EBC10100EB011080F83D2069
:10BB2000D4E19DF8AC1040F2231011FB00F0A949BC
:10BB300001EBC00018309DF8981001EBC10100EB3B
:10BB4000011090F83E0098B901229DF8AC0040F237
:10BB5000231110FB01F09F4901EBC00018309DF844
:10BB6000981001EBC10100EB011080F83D202BE0A3
:10BB700000229DF8AC0040F2231110FB01F0954922
:10BB800001EBC00118319DF8980000EBC00001EBFB
:10BB9000001080F83D209DF8AC1001EB410000EB57
:10BBA00001108B4901EB001130319DF8980002E043
:10BBB000FEE3FEE31FE301EB0010801C0990007818
:10BBC00020F0010209980270834890F8A00890B113
:10BBD0009DF8AC1001EB410000EB01107C4901EB3A
:10BBE0000010303000E0F6E39DF8981000EB0110F3
:10BBF000807A022894D1794890F8210001288FD1C9
:10BC00007648D0F818027549498C884288D29DF848
:10BC1000AC1040F2231011FB00F06E4901EBC000A4
:10BC200018309DF8981001EBC10100EB011090F85D
:10BC30003D00012850D19DF8AC1040F2231011FBBB
:10BC400000F0644901EBC00018309DF8981001EB3A
:10BC5000C10100EB011090F87E00E8BB9DF8AC003C
:10BC600000EB400101EB0010594901EB00113031AC
:10BC70009DF8980001EB001001789DF8AC0040F2AF
:10BC8000231210FB02F0534A02EBC0004170C322A2
:10BC90009DF8AC0040F2231110FB01F04D4901EB7F
:10BCA000C00100E084E118319DF8980000EBC0006D
:10BCB00001EB0010427100229DF8AC0000EB400146
:10BCC00001EB0010424901EB001130319DF8980062
:10BCD00001EB0010426000E047E09DF8AC1002204C
:10BCE000FEF738F90021379119E000229DF8AC00E9
:10BCF00040F2231110FB01F0364901EBC00118316D
:10BD00009DF8980000EBC00001EB00113F31BDF839
:10BD1000DC000A54BDF8DC00401C81B23791BDF84C
:10BD2000DC000A28E1DB0020379019E000229DF8B2
:10BD3000AC0040F2231110FB01F0264901EBC001D9
:10BD400018319DF8980000EBC00001EB00115B3149
:10BD5000BDF8DC000A54BDF8DC00401C81B237910C
:10BD6000BDF8DC000F28E1DBB0E09DF8AC1040F23C
:10BD7000231011FB00F0174901EBC00018309DF8AB
:10BD8000981001EBC10100EB011090F83D00012873
:10BD90007ED19DF8AC1040F2231011FB00F00D494C
:10BDA00001EBC00118319DF8980000EBC00001EBD9
:10BDB000001090F87F1040F2231011FB00F00549AD
:10BDC00001EBC00118319DF8AC0040F2231207E0EE
:10BDD00014410020D4450020BC320020BC120020B9
:10BDE00010FB02F0FE4A02EBC00018309DF89820CC
:10BDF00002EBC20200EB021090F8800000EBC000E2
:10BE000001EB001090F8770003285FD100239DF824
:10BE1000AC0040F2231110FB01F0F14901EBC0012D
:10BE200018319DF8980000EBC00001EB001090F86D
:10BE30007F0040F2231110FB01F0E94901EBC00142
:10BE400018319DF8AC0040F2231210FB02F0E44AD6
:10BE500002EBC00218329DF8980000EBC00002EB24
:10BE6000001090F8800000EBC00001EB001080F89B
:10BE700077309DF8AC0000EB400101EB0010D94990
:10BE800001EB001130319DF8980001EB001000E04B
:10BE90001CE001789DF8AC0040F2231210FB02F088
:10BEA000CF4A02EBC0004170C3229DF8AC0040F2C3
:10BEB000231110FB01F0CA4901EBC00018309DF8B6
:10BEC000981001EBC10100EB011042719DF8AC101C
:10BED0000220FEF73FF89DF8AC0000EB400101EBBB
:10BEE0000010C04901EB001030309DF8981000EBB5
:10BEF00001108078C0F3400088B1D9229DF8AC00D1
:10BF000040F2231110FB01F0B54901EBC0001830DD
:10BF10009DF8981001EBC10100EB011042719DF8F2
:10BF2000AC0040F2231110FB01F0AD4901EBC00061
:10BF300018309DF8981001EBC10100EB01108078DA
:10BF4000B22835D19DF8AC0000EB400101EB0010A8
:10BF5000A44901EB001030309DF8981000EB01105F
:10BF60008078C0F3400018BB9DF8AC0000EB4001A6
:10BF700001EB00109B4901EB001030309DF8981048
:10BF800000EB01108078C0F3401088B9E5229DF8DD
:10BF9000AC0040F2231110FB01F0914901EBC0000D
:10BFA00018309DF8981001EBC10100EB01104271AF
:10BFB0009DF8AC0000EB400101EB0010894901EB5A
:10BFC000001030309DF8981000EB011080780121AE
:10BFD000B1EBD01F75D19DF8AC0000EB400101EB37
:10BFE0000010804901EB001030309DF8981000EBF4
:10BFF0000110807800F00100002862D19DF8AC00AB
:10C0000040F2231110FB01F0754901EBC00018301C
:10C010009DF8981001EBC10100EB011090F83E0073
:10C0200000284ED19DF8AC0000EB400101EB001060
:10C030006C4901EB001030309DF8981000EB0110B6
:10C040008078C0F3C000E0BB9DF8AC0000EB40017D
:10C0500001EB0010634901EB001030309DF898109F
:10C0600000EB0110407A00F0010050B39DF8AC00E5
:10C0700040F2231110FB01F0594901EBC0001830C8
:10C080009DF8981001EBC10100EB011090F88E00B3
:10C0900000F00100A8B99DF8AC0040F2231110FB9C
:10C0A00001F04F4901EBC00018309DF8981001EBEA
:10C0B000C10100EB011090F8810010B10020379011
:10C0C0002AE096E09DF8AC0040F2231110FB01F04D
:10C0D000434901EBC00118319DF8980000EBC00006
:10C0E00001EB001000F18201BDF8DC000A5C9DF854
:10C0F000AC0000EB400101EB00103A4901EB0010ED
:10C100000E30BDF8DC10405C824200D008E0BDF883
:10C11000DC00401C81B23791BDF8DC000628D1DB81
:10C1200000BFBDF8DC00062863D1379029E09DF8F8
:10C13000AC0040F2231110FB01F0294901EBC001D2
:10C1400018319DF8980000EBC00001EB001000F1E1
:10C150008201BDF8DC000A5C9DF8AC0000EB4001F8
:10C1600001EB00101F4901EB00100E30BDF8DC1090
:10C17000405C824200D008E0BDF8DC00401C81B287
:10C180003791BDF8DC000A28D1DB00BFBDF8DC0028
:10C190000A282ED09DF8AC0040F2231110FB01F0CC
:10C1A0000F4901EBC00018309DF8981001EBC10158
:10C1B00000EB01108E300990007820F00100401C47
:10C1C0000999087012229DF8AC0040F2231110FB6F
:10C1D00001F0034901EBC00018309DF8981003E00E
:10C1E000D44500201441002001EBC10100EB0110F7
:10C1F000427101F0B7BB9DF8AC1001EB410000EBC0
:10C200000110FE4901EB0010007BD0BBBDF89C0083
:10C21000082800D0EDE70020379028E09DF8AC100A
:10C2200001EB4100C0EBC110F54901EBC001BDF8C5
:10C23000DC00C01C085C00F00F00092800DD1AE0DB
:10C240009DF8AC1001EB4100C0EBC110EC4901EBD3
:10C25000C001BDF8DC00C01C085C00F0F0009028B4
:10C2600000DD08E0BDF8DC00401C81B23791BDF86C
:10C27000DC000628D2DB00BFBDF8DC00062801DAAE
:10C28000B7E76AE09DF8AC1001EB4100C0EBC110CC
:10C29000DB4901EBC000C07801049DF8AC0000EB65
:10C2A0004002C2EBC010D64A02EBC000007941EA5E
:10C2B00000219DF8AC0000EB4002C2EBC010D04A58
:10C2C00002EBC000407901439DF8AC0040F223121C
:10C2D00010FB02F0CB4A02EBC00218329DF8980026
:10C2E00000E0B6E100EBC00002EB0010C0F81A104D
:10C2F0009DF8AC1001EB4100C0EBC110C04901EB4F
:10C30000C000807901049DF8AC0000EB4002C2EB54
:10C31000C010BB4A02EBC000C07941EA00219DF881
:10C32000AC0000EB4002C2EBC010B54A02EBC0000B
:10C33000007A01439DF8AC0040F2231210FB02F09A
:10C34000B04A02EBC00018309DF8982002EBC20200
:10C3500000EB0210C0F81E10BEE0BDF89C000A28D9
:10C3600000D046E7002037902BE09DF8AC1001EBA1
:10C370004100C0EBC110A24901EBC001BDF8DC00D7
:10C38000C01C085C00F00F00092800DD1DE09DF8CE
:10C39000AC1001EB4100C0EBC110994901EBC001A9
:10C3A000BDF8DC00C01C085C00F0F000902801E043
:10C3B00097E102E200DD08E0BDF8DC00401C81B23C
:10C3C0003791BDF8DC000828CFDB00BFBDF8DC00EA
:10C3D000082801DA0DE771E19DF8AC1001EB41008E
:10C3E000C0EBC111864800EBC100C07801069DF882
:10C3F000AC0000EB4002C2EBC010814A02EBC0006F
:10C40000007941EA00419DF8AC0000EB4002C2EB2C
:10C41000C0107B4A02EBC000407941EA00219DF840
:10C42000AC0000EB4002C2EBC010754A02EBC0004A
:10C43000807901439DF8AC0040F2231210FB02F01A
:10C44000704A02EBC00218329DF8980000EBC00061
:10C4500002EB0010C0F81A109DF8AC1001EB41007F
:10C46000C0EBC110664901EBC000C07901069DF820
:10C47000AC0000EB4002C2EBC010614A02EBC0000E
:10C48000007A41EA00419DF8AC0000EB4002C2EBAB
:10C49000C0105B4A02EBC000407A41EA00219DF8DF
:10C4A000AC0000EB4002C2EBC010554A02EBC000EA
:10C4B000807A01439DF8AC0040F2231210FB02F099
:10C4C000504A02EBC00018309DF8982002EBC202DF
:10C4D00000EB0210C0F81E109DF8AC0040F22311D2
:10C4E00010FB01F0474901EBC00118319DF898009D
:10C4F00000EBC00001EB001001789DF8AC0040F2A9
:10C50000231210FB02F03F4A02EBC0004079814247
:10C510002FDA00219DF8AC0040F2231210FB02F04C
:10C52000384A02EBC000017104229DF8AC0040F2D1
:10C53000231110FB01F0334901EBC00118319DF8C4
:10C54000980000EBC00001EB00100270C5229DF8BE
:10C55000AC0040F2231110FB01F02A4901EBC000AE
:10C5600018309DF8981001EBC10100EB01104271E9
:10C570006EE09DF8AC0000EB400101EB00101F499C
:10C5800001EB001030309DF8981000EB011080781E
:10C59000C0F3400090B1D5229DF8AC0040F22311C9
:10C5A00010FB01F0174901EBC00018309DF89810FE
:10C5B00001EBC10100EB0110427149E09DF8AC00B4
:10C5C00040F2231110FB01F00E4901EBC0001830BE
:10C5D0009DF8981001EBC10100EB0110807B012850
:10C5E00036D100229DF8AC0040F2231110FB01F07F
:10C5F000044901EBC001183106E00000144100209D
:10C60000A8780020D44500209DF8980000EBC000D9
:10C6100001EB00108273B6229DF8AC0040F22311AA
:10C6200010FB01F0FE4901EBC00118319DF89800A4
:10C6300000EBC00001EB0010427100219DF8AC003E
:10C6400040F2231210FB02F0F54A02EBC000017128
:10C65000CFE5D5229DF8AC0040F2231110FB01F08C
:10C66000EF4901EBC00118319DF8980000EBC000C4
:10C6700001EB0010427101219DF8AC0040F2231241
:10C6800010FB02F0E64A02EBC00001719DF8AC001D
:10C6900000EB400101EB0010A2F5986101EB0011E5
:10C6A00030319DF8980001EB0010801C0990007853
:10C6B00020F020002030099908709AE5D5229DF8D5
:10C6C000AC0040F2231110FB01F0D54901EBC00092
:10C6D00018309DF8981001EBC10100EB0110427178
:10C6E00087E59DF8AC0040F2231110FB01F0CC4926
:10C6F00001EBC0001830BDF8D01001EBC10100EB18
:10C700000110807901283AD100229DF8AC0040F256
:10C71000231110FB01F0C24901EBC0011831BDF833
:10C72000D00000EBC00001EB00108271D5229DF813
:10C73000AC0040F2231110FB01F0B94901EBC0013C
:10C7400018319DF8980000EBC00001EB0010427119
:10C750009DF8AC0000EB400101EB0010B14901EB8A
:10C76000001130319DF8980001EB0010801C0990F9
:10C77000007820F00400001D099908701CE0C32215
:10C780009DF8AC0040F2231110FB01F0A44901EB2D
:10C79000C00118319DF8980000EBC00001EB0010BB
:10C7A000427100219DF8AC0040F2231210FB02F010
:10C7B0009B4A02EBC00001711BE59DF8AC0040F202
:10C7C000231110FB01F0964901EBC0001830BDF8B1
:10C7D000D01001EBC10100EB0110807901283AD1A2
:10C7E00000229DF8AC0040F2231110FB01F08C49AF
:10C7F00001EBC0011831BDF8D00000EBC00001EB27
:10C8000000108271D5229DF8AC0040F2231110FB7C
:10C8100001F0834901EBC00118319DF8980000EB4D
:10C82000C00001EB001042719DF8AC1001EB41001B
:10C8300000EB01107B4901EB001130319DF89800AD
:10C8400001EB0010801C0990007820F00400001D0E
:10C85000099908701CE0C3229DF8AC0040F2231136
:10C8600010FB01F06E4901EBC00118319DF89800F2
:10C8700000EBC00001EB0010427100219DF8AC00FC
:10C8800040F2231210FB02F0654A02EBC000017176
:10C89000AFE49DF8AC1001EB410000EB01106149E1
:10C8A00001EB0010007B38BB9DF8AC1001EB4100A0
:10C8B000C0EBC1105C4901EBC00001799DF8AC00F0
:10C8C00000EB4002C2EBC010574A02EBC000C07838
:10C8D00041EA00229DF8AC0040F2231110FB01F068
:10C8E0004F4901EBC00018309DF8981001EBC101D1
:10C8F00000EB0110426332E09DF8AC1001EB410007
:10C90000C0EBC110484901EBC000C07801049DF89C
:10C91000AC0000EB4002C2EBC010434A02EBC00087
:10C92000007941EA00219DF8AC0000EB4002C2EB27
:10C93000C0103D4A02EBC000407901439DF8AC00B5
:10C9400040F2231210FB02F0354A02EBC00018300F
:10C950009DF8982002EBC20200EB021041639DF8A3
:10C96000AC1040F2231011FB00F02D4901EBC00187
:10C9700018319DF8980000EBC00001EB0010017821
:10C980009DF8AC0040F2231210FB02F0244A02EBA7
:10C99000C000407981422FDA00219DF8AC0040F2BE
:10C9A000231210FB02F01E4A02EBC00001710322A9
:10C9B0009DF8AC0040F2231110FB01F0184901EB87
:10C9C000C00118319DF8980000EBC00001EB001089
:10C9D0000270D9229DF8AC0040F2231110FB01F047
:10C9E0000F4901EBC00018309DF8981001EBC10110
:10C9F00000EB011042717CE09DF8AC1040F2231076
:10CA000011FB00F0064901EBC0001830BDF8D01052
:10CA100001EBC10100EB0110807901284CD105E048
:10CA2000D445002014410020A878002000229DF861
:10CA3000AC0040F2231110FB01F0FE4901EBC001F4
:10CA40001831BDF8D00000EBC00001EB001082717E
:10CA5000D9229DF8AC0040F2231110FB01F0F549FA
:10CA600001EBC00118319DF8980000EBC00001EB0C
:10CA7000001042719DF8AC1001EB410000EB011079
:10CA8000ED4901EB001130319DF8980001EB0010E9
:10CA9000801C0990007820F00400001D099908709E
:10CAA00001209DF8AC1040F2231211FB02F1E14A83
:10CAB00002EBC10108711CE0C5229DF8AC0040F2F8
:10CAC000231110FB01F0DB4901EBC00118319DF887
:10CAD000980000EBC00001EB0010427100219DF8AE
:10CAE000AC0040F2231210FB02F0D24A02EBC0006D
:10CAF000017136E400219DF8AC0040F2231210FBD6
:10CB000002F0CC4A02EBC00001719DF8AC1001EBC1
:10CB1000410000EB0110C84901EB001130319DF8D4
:10CB2000980001EB0010801C0990007820F00400B0
:10CB3000001D09990870D5229DF8AC0040F2231120
:10CB400010FB01F0BB4901EBC00018309DF89810B4
:10CB500001EBC10100EB011042713BE49DF8AC0018
:10CB600000EB400101EB0010B34901EB0010007B2A
:10CB7000D0BBBDF89C000C2800D02BE400203790DF
:10CB800028E09DF8AC0000EB4001C1EBC010AB49C0
:10CB900001EBC001BDF8DC00C01C085C00F00F0018
:10CBA000092800DD1AE09DF8AC0000EB4001C1EB64
:10CBB000C010A24901EBC001BDF8DC00C01C085C3C
:10CBC00000F0F000902800DD08E0BDF8DC00401C1B
:10CBD00081B23791BDF8DC000A28D2DB00BFBDF876
:10CBE000DC000A2801DA33E57CE000202C902D904F
:10CBF000002137911EE0DDE92C10000240EA1162AD
:10CC00000902CDE92C129DF8AC0000EB4001C1EB0C
:10CC1000C0108A4901EBC001BDF8DC00C01C085CF3
:10CC2000DDE92C241043CDE92C04BDF8DC00401CC8
:10CC300080B23790BDF8DC000528DCDB9DF8AC0045
:10CC4000DDE92C1240F2231310FB03F0794B03EBC8
:10CC5000C00318339DF8980000EBC00003EB0010F0
:10CC600040F8221F426000222C922D920021379121
:10CC70001EE0DDE92C10000240EA11620902CDE954
:10CC80002C129DF8AC0000EB4001C1EBC0106B49C9
:10CC900001EBC001BDF8DC000830085CDDE92C3494
:10CCA0001843CDE92C04BDF8DC00401C80B237905D
:10CCB000BDF8DC000528DCDB9DF8AC00DDE92C21AB
:10CCC00040F2231310FB03F05A4B03EBC000183063
:10CCD0009DF8983003EBC30300EB03102230826011
:10CCE000C160BEE0BDF89C000E2800D0B0E400207A
:10CCF000379028E09DF8AC0000EB4001C1EBC0107C
:10CD00004E4901EBC001BDF8DC00C01C085C00F01E
:10CD10000F00092800DD1AE09DF8AC0000EB40018F
:10CD2000C1EBC010454901EBC001BDF8DC00C01CDF
:10CD3000085C00F0F000902800DD08E0BDF8DC00A1
:10CD4000401C81B23791BDF8DC000C28D2DB00BF5B
:10CD5000BDF8DC000C2800DA7AE400202C902D903D
:10CD6000002137911EE0DDE92C10000240EA11623B
:10CD70000902CDE92C129DF8AC0000EB4001C1EB9B
:10CD8000C0102E4901EBC001BDF8DC00C01C085CDE
:10CD9000DDE92C341843CDE92C04BDF8DC00401C3F
:10CDA00080B23790BDF8DC000628DCDB9DF8AC00D3
:10CDB000DDE92C2340F2231110FB01F01D4901EBAA
:10CDC000C00118319DF8980000EBC00001EB001085
:10CDD00040F8222F436000222C922D92002137919F
:10CDE0001EE0DDE92C10000240EA11620902CDE9E3
:10CDF0002C129DF8AC1001EB4100C0EBC1100F49A3
:10CE000001EBC001BDF8DC000930085CDDE92C2431
:10CE10001043CDE92C04BDF8DC00401C80B23790F3
:10CE2000BDF8DC000628DCDB9DF8AC00DDE92C1247
:10CE300006E00000D445002014410020A87800201E
:10CE400040F2231310FB03F0FE4B03EBC00018303D
:10CE50009DF8983003EBC30300EB03102230816090
:10CE6000C2609DF8AC1040F2231011FB00F0F549B0
:10CE700001EBC00118319DF8980000EBC00001EBF8
:10CE8000001001789DF8AC0040F2231210FB02F074
:10CE9000EC4A02EBC000407981427CD1EA4890F82C
:10CEA000A00888B19DF8AC1001EB410000EB011027
:10CEB000A2F5986101EB001030309DF8981000EB5E
:10CEC0000110807A022867D1E048D0F818020521C5
:10CED000B0FBF1F201FB120101EBC10000EB01110B
:10CEE000DA48243000EB81000021C0F81D10D7483B
:10CEF000D0F818020521B0FBF1F201FB120101EBA1
:10CF0000C10000EB0111D148243000EB81000D304D
:10CF100009909DF8AC1040F2231011FB00F0C949B4
:10CF200001EBC00118319DF8980000EBC00001EB47
:10CF3000001022301022014608900998FBF785F96D
:10CF4000C248D0F818020521B0FBF1F201FB120132
:10CF500001EBC10000EB0111BC48243000EB810261
:10CF60009DF8AC0040F2231110FB01F0B54901EB34
:10CF7000C00118319DF8980000EBC00001EB0010D3
:10CF800050F81A1F42F8011F40685060AF48D0F8AF
:10CF90001802052101E02FE201E1B0FBF1F201FBF3
:10CFA000120101EBC10000EB0113A84924319DF8E7
:10CFB000AC0000EB400202EB0010A54A02EB0012AD
:10CFC00030329DF8980002EB0010007801F8230041
:10CFD0009E48D0F818020521B0FBF1F201FB1200C7
:10CFE00000EBC00101EB00119848243000EB8101F7
:10CFF0009548C26941F8212F008C88809348D0F869
:10D0000018020521B0FBF1F201FB120000EBC00198
:10D0100001EB00118D48243000EB81029DF8AC003B
:10D0200040F2231110FB01F0864901EBC0011831D9
:10D030009DF8980000EBC00001EB0010406BC2F8B7
:10D0400009008248D0F818020521B0FBF1F201FB7B
:10D05000120000EBC00101EB00117C48243000EB12
:10D0600081029DF8AC0000EB400101EB0010784913
:10D0700001EB001130319DF8980001EB0010406881
:10D08000C2F82700002137914CE07048D0F8180210
:10D090000521B0FBF1F201FB120000EBC00101EB36
:10D0A00000116A48243000EB81012B31BDF8DC40CF
:10D0B0009DF8AC0040F2231210FB02F0614A02EB33
:10D0C000C00218329DF8980000EBC00002EB00107F
:10D0D00090F87F0040F2231210FB02F0594A02EB55
:10D0E000C00218329DF8AC0040F2231310FB03F08D
:10D0F000544B03EBC00318339DF8980000EBC000BD
:10D1000003EB001090F8800000EBC00002EB00126F
:10D110003F32BDF8DC00105C0855BDF8DC00401C57
:10D1200081B23791BDF8DC000A28AEDB4748D0F861
:10D1300018020521B0FBF1F080B2014609900220EF
:10D14000FBF7C6FF00210620FCF704FF3F48D0F89C
:10D1500018023E49498C884206D23C48D0F8180251
:10D16000401C3A49C1F8180200210520FCF7F2FEE4
:10D170009DF8AC0000EB400101EB0010344901EBDD
:10D18000001030309DF8981000EB0110801C0990C1
:10D19000007820F00400001D0999087015E09DF842
:10D1A000AC0000EB400101EB0010294901EB00103D
:10D1B00030309DF8981000EB0110801C0990007829
:10D1C00020F008000830099908709DF8AC0000EBC9
:10D1D000400101EB00101E4901EB001030309DF8BA
:10D1E000981000EB0110801C0990007820F02002BC
:10D1F000099802709DF8AC100220FCF7ABFE9DF878
:10D20000AC009DF8981001EB0010C217CDE92C027C
:10D2100000222C9800EBC00101EB00110D4800EB3F
:10D220008100C0F81D209DF8AC0040F2231110FBD6
:10D2300001F0044901EBC00018309DF8981001EB93
:10D24000C10109E0D4450020BC320020BC120020FE
:10D2500014410020E414002000EB0110223009905A
:10D260002C9800EBC00101EB0011FC4800EB8101A0
:10D270000D3110220891DDE90801FAF7E6FF9DF86B
:10D28000AC0040F2231110FB01F0F54901EBC001A5
:10D2900018319DF8980000EBC00001EB00112C98AC
:10D2A00000EBC00202EB0012EC4800EB820051F8E8
:10D2B0001A2F40F8012F496841609DF8AC0000EB3F
:10D2C000400101EB0010E74901EB001130319DF8FE
:10D2D000980001EB001001782C9800EBC00202EBE3
:10D2E0000012DE4800F822102C9800EBC00101EB80
:10D2F0000011DA4800EB8101DB48C26941F8212FB7
:10D30000008C88809DF8AC0040F2231110FB01F0E6
:10D31000D34901EBC00118319DF8980000EBC00023
:10D3200001EB0010416B2C9800EBC00202EB0012E5
:10D33000CA4800EB8200C0F809109DF8AC0000EB71
:10D34000400101EB0010C74901EB001130319DF89D
:10D35000980001EB001041682C9800EBC00202EB32
:10D360000012BE4800EB8200C0F827100021379160
:10D3700024E09DF8AC0040F2231110FB01F0B84905
:10D3800001EBC00118319DF8980000EBC00001EBE3
:10D3900000113F31BDF8DC000A5C2C9800EBC001A5
:10D3A00001EB0011AD4800EB81012B31BDF8DC0031
:10D3B0000A54BDF8DC00401C81B23791BDF8DC0096
:10D3C0000A28D6DB2C9881B208200991FCF7C2FD0F
:10D3D00000229DF8AC0040F2231110FB01F0A0499F
:10D3E00001EBC00018309DF8981001EBC10100EB73
:10D3F000011080F83E2051E09DF8AC0000EB4001A8
:10D4000001EB0010974901EB001030309DF89810A7
:10D4100000EB0110801C0990007820F00401091D28
:10D42000099801709DF8AC0000EB400101EB001081
:10D430008C4901EB001130319DF8980001EB001090
:10D44000801C0990007820F08001803109980170DB
:10D4500001219DF8AC0040F2231210FB02F0804A3B
:10D4600002EBC00001719DF8AC0040F2231110FBEB
:10D4700001F0114601EBC00042799DF8AC0040F28A
:10D48000231110FB01F0764901EBC00018309DF824
:10D49000981001EBC10100EB01100270D5229DF83C
:10D4A000AC0040F2231110FB01F06D4901EBC0000C
:10D4B00018309DF8981001EBC10100EB011042718A
:10D4C00050E2D5229DF8AC0040F2231110FB01F090
:10D4D000634901EBC00018309DF8981001EBC101C1
:10D4E00000EB011042713DE2D5229DF8AC0040F204
:10D4F000231110FB01F05A4901EBC00018309DF8D0
:10D50000981001EBC10100EB011042712AE20121E8
:10D51000554880F8C4179DF8AC0040F2231110FB69
:10D5200001F04F4901EBC00118319DF8980000EB64
:10D53000C00001EB001001789DF8AC0040F223120E
:10D5400010FB02F0464A02EBC000407981422FDA1C
:10D5500000219DF8AC0040F2231210FB02F0404A7B
:10D5600002EBC000017101229DF8AC0040F22311D2
:10D5700010FB01F03A4901EBC00118319DF8980009
:10D5800000EBC00001EB0010027011229DF8AC000E
:10D5900040F2231110FB01F0314901EBC0001830BB
:10D5A0009DF8981001EBC10100EB0110427154E0AD
:10D5B0009DF8AC0040F2231110FB01F0284901EB6B
:10D5C000C00018309DF8981001EBC10100EB01106C
:10D5D0008078B2282FD100219DF8AC0040F22312B0
:10D5E00010FB02F01E4A02EBC0000171B2229DF84E
:10D5F000AC0040F2231110FB01F0194901EBC0010E
:10D6000018319DF8980000EBC00001EB001042714A
:10D6100000229DF8AC0040F2231110FB01F01049EC
:10D6200001EBC00018309DF8981001EBC10100EB30
:10D630000110827011E0D5229DF8AC0040F2231158
:10D6400010FB01F0064901EBC00018309DF898105E
:10D6500001EBC10100EB0110427183E1E4140020F1
:10D66000D445002014410020BC3200200021FE4897
:10D6700080F8C417D5229DF8AC0040F2231110FBAE
:10D6800001F0FA4901EBC00018309DF8981001EB49
:10D69000C10100EB0110427164E101229DF8AC0070
:10D6A00040F2231110FB01F0F04901EBC0011831E9
:10D6B0009DF8980000EBC00001EB001080F881207D
:10D6C0000021379126E09DF8AC0000EB4001C1EB52
:10D6D000C010E74901EBC001BDF8DC00C01C0A5CCA
:10D6E0009DF8AC0040F2231110FB01F0DF4901EB83
:10D6F000C00118319DF8980000EBC00001EB00104C
:10D7000000F18201BDF8DC000A54BDF8DC00401CC9
:10D7100081B23791BDF8DC000A28D4DB22E19DF804
:10D72000AC1001EB4100C0EBC110D14901EBC000CE
:10D73000C07801049DF8AC0000EB4002C2EBC010C1
:10D74000CB4A02EBC000007941EA00209DF8AC1002
:10D7500001EB4102C2EBC111C54A02EBC10149799B
:10D760000843B0F5E13F65D19DF8AC1001EB4100F5
:10D7700000EB0110BF4901EB001030309DF898100C
:10D7800000EB0110801C0990007820F00402099839
:10D79000027000229DF8AC0040F2231110FB01F052
:10D7A000B24901EBC00018309DF8981001EBC1019F
:10D7B00000EB0110A0F88C2013229DF8AC0040F281
:10D7C000231110FB01F0A94901EBC00018309DF8AE
:10D7D000981001EBC10100EB011042719DF8AC10F3
:10D7E00001EB410000EB0110A24901EB0010407970
:10D7F00003464FF480524FF4E13109909DF8AC009C
:10D8000010F0D8F99DF8AC1040F2231011FB00F095
:10D81000964901EBC00118319DF8980000EBC0005B
:10D8200001EB00108E300990007820F008000830DD
:10D830000999087096E09DF8AC1001EB4100C0EB2F
:10D84000C1108B4901EBC00001799DF8AC0000EBE1
:10D850004002C2EBC010864A02EBC000C07841EA29
:10D8600000229DF8AC0040F2231110FB01F07F492B
:10D8700001EBC00118319DF8980000EBC00001EBEE
:10D880000010A0F88C209DF8AC1040F2231011FB82
:10D8900000F0764901EBC00118319DF8980000EBCB
:10D8A000C00001EB0010B0F88C109DF8AC0000EB4C
:10D8B000400202EB00106F4A02EB0010408B8142E5
:10D8C0004FDBE5229DF8AC0040F2231110FB01F084
:10D8D000664901EBC00118319DF8980000EBC000CB
:10D8E00001EB0010427100229DF8AC0040F22311C0
:10D8F00010FB01F05D4901EBC00118319DF8980063
:10D9000000EBC00001EB001002709DF8AC1001EBC1
:10D91000410000EB0110574901EB001130319DF837
:10D92000980001EB0010801C0990007820F0800224
:10D93000099802709DF8AC1040F2231011FB00F022
:10D940004A4901EBC00018309DF8981001EBC10165
:10D9500000EB01108E300990007820F00102099848
:10D96000027000BF00BF08F05FBD9DF8AC1001EB76
:10D970004100C0EBC1103E4911F83000042801D12C
:10D9800024900BE09DF8AC1001EB4100C0EBC110FE
:10D99000374911F83000152800D124909DF8AC10BB
:10D9A00001EB4100C0EBC110314901EBC0004178EF
:10D9B0009DF8AC0000EB4002C2EBC0102C4A12F8FC
:10D9C000300041EA002041F23001884202D1A62015
:10D9D00024903DE09DF8AC1001EB4100C0EBC1107C
:10D9E000234901EBC00041789DF8AC0000EB4002F8
:10D9F000C2EBC0101E4A12F8300041EA002041F28A
:10DA00003101884202D1A720249021E09DF8AC107A
:10DA100001EB4100C0EBC110154911F8300002289C
:10DA200016D19DF8AC1001EB4100C0EBC1101049BC
:10DA300001EBC00001799DF8AC0000EB4002C2EBA5
:10DA4000C0100B4A02EBC000C07841EA00212491CB
:10DA50009DF8AC1040F2231011FB00F0034901EBDC
:10DA6000C0008178269107E0BC320020D445002018
:10DA7000A8780020144100200021FE4A9DF8AC0047
:10DA800002EB00129DF898001154FB4890F820001A
:10DA9000012815D19DF8AC1001EB410000EB0110FD
:10DAA000F64901EB001030309DF8981000EB0110A2
:10DAB000801C0990007820F080008030099908705F
:10DAC000BDF8901043F23002881A91427ED009DCF2
:10DAD00004297CD015297BD0A6290ED0A72941F096
:10DAE0006B8635E1B0F5C06F73D0A0F201600028FD
:10DAF00070D00428F3D101F078BB00219DF8AC0070
:10DB000040F2231210FB02F0DD4A02EBC00001716B
:10DB10009DF8AC1040F2231011FB00F0114601EB10
:10DB2000C00018309DF8981001EBC10100EB011006
:10DB30000078032824DC04229DF8AC0040F2231175
:10DB400010FB01F0CE4901EBC00118319DF898009F
:10DB500000EBC00001EB00100270A8229DF8AC00A1
:10DB600040F2231110FB01F0C54901EBC000183051
:10DB70009DF8981001EBC10100EB01104271E5E046
:10DB80009DF8AC1040F2231011FB00F0BC4901EBF2
:10DB9000C00018309DF8981001EBC10100EB011096
:10DBA000007808282ADC09229DF8AC0040F22311F5
:10DBB00010FB01F0B24901EBC00118319DF898004B
:10DBC00000EBC00001EB0010027004E07EE1F3E125
:10DBD000FDE3FDE3FDE3A9229DF8AC0040F2231133
:10DBE00010FB01F0A64901EBC00018309DF8981019
:10DBF00001EBC10100EB01104271A7E09DF8AC10F0
:10DC000040F2231011FB00F09D4901EBC0001830D9
:10DC10009DF8981001EBC10100EB011000780D2870
:10DC200024DC0E229DF8AC0040F2231110FB01F021
:10DC3000934901EBC00118319DF8980000EBC0003A
:10DC400001EB00100270A2229DF8AC0040F22311FB
:10DC500010FB01F08A4901EBC00018309DF89810C4
:10DC600001EBC10100EB011042716FE09DF8AC10B7
:10DC700040F2231011FB00F0814901EBC000183085
:10DC80009DF8981001EBC10100EB01104079A52827
:10DC900015D19DF8AC1001EB410000EB0110774964
:10DCA00001EB001030309DF8981000EB0110801C43
:10DCB0000990007820F00400001D099908709DF873
:10DCC000AC1040F2231011FB00F06D4901EBC000D5
:10DCD00018309DF8981001EBC10100EB011080781D
:10DCE000A12833D09DF8AC0040F2231110FB01F0C5
:10DCF000634901EBC00118319DF8980000EBC000AA
:10DD000001EB001082789DF8AC0040F2231110FB6B
:10DD100001F05B4901EBC00118319DF8980000EB60
:10DD2000C00001EB00104271A1229DF8AC0040F24E
:10DD3000231110FB01F0524901EBC00018309DF88F
:10DD4000981001EBC10100EB0110827001F034BDAD
:10DD500000219DF8AC0040F2231210FB02F0484A6B
:10DD600002EBC00001719DF8AC0040F2231110FBE2
:10DD700001F0114601EBC00018309DF8981001EB3E
:10DD8000C10100EB0110007805281DDC00219DF881
:10DD9000AC0040F2231210FB02F0394A02EBC00043
:10DDA000017106229DF8AC0040F2231110FB01F036
:10DDB000334901EBC00018309DF8981001EBC10108
:10DDC00000EB0110027024E09DF8AC0040F223113A
:10DDD00010FB01F02A4901EBC00018309DF89810A3
:10DDE00001EBC10100EB01100078092811DC0A22C7
:10DDF0009DF8AC0040F2231110FB01F0204901EB2B
:10DE0000C00018309DF8981001EBC10100EB011023
:10DE100002709DF8AC0040F2231110FB01F018498C
:10DE200001EBC00018309DF8981001EBC10100EB28
:10DE300001104079A42836D19DF8AC0000EB4001D8
:10DE400001EB00100D4901EB001030309DF89810E7
:10DE500000EB0110801C0990007820F02000203099
:10DE60000999087000229DF8AC0040F2231110FBC4
:10DE700001F007E0483F0020BC12002014410020C0
:10DE8000D4450020FE4901EBC00018309DF89810E1
:10DE900001EBC10100EB011080F83D209DF8AC10B2
:10DEA0000220FCF757F8A1229DF8AC0040F22311A4
:10DEB00010FB01F0F24901EBC00018309DF89810FA
:10DEC00001EBC10100EB011042713FE700203790E8
:10DED00015E09DF8AC0000EB4001C1EBC010E94932
:10DEE00001EBC001BDF8DC00C01C095C16AABDF83E
:10DEF000DC001154BDF8DC00401C81B23791BDF844
:10DF0000DC000628E5DB062116A81DF091FE0021A5
:10DF1000CDE92E01DDE92E21100A40EA01602E9C98
:10DF2000001941EB21214FF480724FF00003CDE93D
:10DF30000801FAF747F99DF8AC0040F2231110FBF5
:10DF400001F0CF4901EBC00018309DF8981001EBAB
:10DF5000C10100EB0110027100229DF8AC0040F2FB
:10DF6000231110FB01F0C64901EBC0000271012230
:10DF70009DF8AC0040F2231110FB01F0C04901EB09
:10DF8000C00018309DF8981001EBC10100EB0110A2
:10DF90000270A7229DF8AC0040F2231110FB01F0A3
:10DFA000B74901EBC00018309DF8981001EBC10192
:10DFB00000EB01104271C9E69DF8AC0040F223115C
:10DFC00010FB01F0AE4901EBC00018309DF898102D
:10DFD00001EBC10100EB0110007806282EDC0021C6
:10DFE0009DF8AC0040F2231210FB02F0A44A02EBB1
:10DFF000C000017107229DF8AC0040F2231110FB14
:10E0000001F09F4901EBC00118319DF8980000EB29
:10E01000C00001EB00100270A7229DF8AC0040F296
:10E02000231110FB01F0964901EBC00018309DF858
:10E03000981001EBC10100EB011042719DF8AC009A
:10E0400040F2231110FB01F08D4901EBC0001830A4
:10E050009DF8981001EBC10100EB01100078012838
:10E060002FDC00219DF8AC0040F2231210FB02F0DF
:10E07000834A02EBC000017102229DF8AC0040F21D
:10E08000231110FB01F07E4901EBC00118319DF80E
:10E09000980000EBC00001EB00100270A3229DF875
:10E0A000AC0040F2231110FB01F0754901EBC000F8
:10E0B00018309DF8981001EBC10100EB011042717E
:10E0C0001CE29DF8AC0040F2231110FB01F06C49FA
:10E0D00001EBC00018309DF8981001EBC10100EB76
:10E0E0000110007807282FDC00219DF8AC0040F2D9
:10E0F000231210FB02F0624A02EBC00001710822F9
:10E100009DF8AC0040F2231110FB01F05C4901EBDB
:10E11000C00118319DF8980000EBC00001EB001021
:10E120000270A3229DF8AC0040F2231110FB01F015
:10E13000534901EBC00018309DF8981001EBC10164
:10E1400000EB01104271D9E19DF8AC0040F22311BF
:10E1500010FB01F04A4901EBC00018309DF89810FF
:10E1600001EBC10100EB011000780B282FDC00212E
:10E170009DF8AC0040F2231210FB02F0404A02EB83
:10E18000C00001710C229DF8AC0040F2231110FB7D
:10E1900001F03B4901EBC00118319DF8980000EBFC
:10E1A000C00001EB00100270A1229DF8AC0040F20B
:10E1B000231110FB01F0324901EBC00018309DF82B
:10E1C000981001EBC10100EB0110427196E19DF83E
:10E1D000AC0040F2231110FB01F0294901EBC00013
:10E1E00018309DF8981001EBC10100EB0110007888
:10E1F0000C282FDC00219DF8AC0040F2231210FB0C
:10E2000002F01F4A02EBC00001710D229DF8AC0024
:10E2100040F2231110FB01F0194901EBC001183144
:10E220009DF8980000EBC00001EB00100270A322E3
:10E230009DF8AC0040F2231110FB01F0104901EBF6
:10E24000C00018309DF8981001EBC10100EB0110DF
:10E25000427153E19DF8AC0040F2231110FB01F034
:10E26000074901EBC00018309DF8981001EBC1017F
:10E2700000EB011000780E287DDC0F2204E0000086
:10E28000D4450020A87800209DF8AC0040F223116E
:10E2900010FB01F0FE4901EBC00118319DF8980018
:10E2A00000EBC00001EB00100270A1229DF8AC0051
:10E2B00040F2231110FB01F0F54901EBC0011831C8
:10E2C0009DF8980000EBC00001EB001042719DF832
:10E2D000AC0040F2231110FB01F0ED4901EBC0014D
:10E2E00018319DF8980000EBC00001EB001082701F
:10E2F0009DF8AC0000EB400101EB0010E54901EB9B
:10E30000001130319DF8980001EB0010801C09903D
:10E31000007820F080008030099908709DF8AC00EA
:10E3200000EB400101EB0010DA4901EB0010303046
:10E330009DF8981000EB0110801C0990007820F0E7
:10E340000400001D099908709DF8AC0000EB400125
:10E3500001EB0010CF4901EB001030309DF8981010
:10E3600000EB01108078C0F3401098B39DF8AC002A
:10E3700000EB400100E043E001EB0010C54901EB78
:10E38000001030309DF8981000EB0110801C0990AF
:10E39000007820F02002099802709DF8AC0000EB94
:10E3A000400101EB0010BB4901EB001030309DF83B
:10E3B000981000EB01108078C0F34000D0B99DF8B0
:10E3C000AC0000EB400101EB0010B24903E096E025
:10E3D000C4E006E174E001EB001030309DF89810C5
:10E3E00000EB0110801C0990007820F00800083034
:10E3F000099908709DF8AC100220FBF7ABFD7DE099
:10E400009DF8AC1040F2231011FB00F0A04901EB85
:10E41000C00118319DF8980000EBC00001EB00101E
:10E4200001789DF8AC0040F2231210FB02F0984AEC
:10E4300002EBC0004079814260D19DF8AC1040F2FF
:10E44000231011FB00F0114601EBC00018309DF8BD
:10E45000981001EBC10100EB01108078A12830D0A9
:10E46000A3229DF8AC0040F2231110FB01F0884973
:10E4700001EBC00118319DF8980000EBC00001EBE2
:10E48000001042719DF8AC1040F2231011FB00F017
:10E490007F4901EBC00018309DF8981001EBC101D5
:10E4A00000EB01108078A22828D000209DF8AC1045
:10E4B00040F2231211FB02F1754A02EBC10108710F
:10E4C0001CE0A1229DF8AC0040F2231110FB01F0EA
:10E4D0006F4901EBC00118319DF8980000EBC000B6
:10E4E00001EB0010427101219DF8AC0040F22312B3
:10E4F00010FB02F0664A02EBC000017126E4A12283
:10E500009DF8AC0040F2231110FB01F0604901EBD3
:10E51000C00118319DF8980000EBC00001EB00101D
:10E5200082709DF8AC0040F2231110FB01F05849B5
:10E5300001EBC00118319DF8980000EBC00001EB21
:10E540000010427100219DF8AC0040F2231210FB34
:10E5500002F04F4A02EBC0000171B6E49DF8AC1026
:10E5600040F2231011FB00F0494901EBC0001830C4
:10E570009DF8981001EBC10100EB0110007806280E
:10E580002EDC00219DF8AC0040F2231210FB02F0BB
:10E590003F4A02EBC000017107229DF8AC0040F237
:10E5A000231110FB01F03A4901EBC00118319DF82D
:10E5B000980000EBC00001EB00100270A7229DF84C
:10E5C000AC0040F2231110FB01F0314901EBC00017
:10E5D00018309DF8981001EBC10100EB0110427159
:10E5E00073E400219DF8AC0040F2231210FB02F00E
:10E5F000274A02EBC0000171A7229DF8AC0040F24F
:10E60000231110FB01F0224901EBC00118319DF8E4
:10E61000980000EBC00001EB001042719DF8AC10B7
:10E6200001EB4100C0EBC1101B4901EBC000407978
:10E6300030287DD19DF8AC1040F2231011FB00F082
:10E64000134901EBC00118319DF8980000EBC000A0
:10E6500001EB001001789DF8AC0040F2231210FB92
:10E6600002F00B4A02EBC0004079814260D19DF874
:10E67000AC1001EB410000EB0110064901EB00106A
:10E6800030309DF8981000EB0110801C099005E0D7
:10E69000D445002014410020A8780020007820F004
:10E6A0000102099802709DF8AC1001EB410000EBEB
:10E6B0000110FE4901EB001030309DF8981000EB7E
:10E6C0000110801C0990007820F002020998027065
:10E6D0009DF8AC1040F2231011FB00F0F44901EB5F
:10E6E000C00018309DF8981001EBC10100EB01103B
:10E6F000C07831282ED19DF8AC1001EB410000EB21
:10E700000110EA4901EB001030309DF8981000EB41
:10E710000110801C0990007820F0200209980270F6
:10E7200000229DF8AC0040F2231110FB01F000E044
:10E7300037E0DF4901EBC00018309DF8981001EB7D
:10E74000C10100EB011080F83D209DF8AC100220C3
:10E75000FBF700FC9DF8AC1040F2231011FB00F019
:10E76000D34901EBC00018309DF8981001EBC101AE
:10E7700000EB011090F83E00012811D1A9229DF86C
:10E78000AC0040F2231110FB01F0C94901EBC000BD
:10E7900018309DF8981001EBC10100EB0110827058
:10E7A00079E29DF8AC1001EB4100C0EBC110C1490A
:10E7B00001EBC000407931287ED19DF8AC1040F2C9
:10E7C000231011FB00F0BA4901EBC00118319DF88C
:10E7D000980000EBC00001EB001001789DF8AC0040
:10E7E00040F2231210FB02F0B14A02EBC000407964
:10E7F000814261D19DF8AC1040F2231011FB00F072
:10E80000114601EBC00018309DF8981001EBC101D2
:10E8100000EB011090F83E0040BB01229DF8AC00D7
:10E8200040F2231110FB01F0A14901EBC0011831A6
:10E830009DF8980000EBC00001EB001080F83D202F
:10E840009DF8AC1001EB410000EB0110974901EB82
:10E85000001130319DF8980001EB0010801C0990E8
:10E86000007820F00100401C099908709DF8AC1058
:10E8700001EB410000EB01108C4901EB001030303E
:10E880009DF8981000EB0110801C0990007820F092
:10E89000020209980270884890F8A008002872D1F6
:10E8A000864890F8210001286DD18448D0F81802DC
:10E8B0008249498C884200E0A9E064D29DF8AC10FE
:10E8C00040F2231011FB00F0794901EBC000183031
:10E8D0009DF8981001EBC10100EB011090F83D008C
:10E8E000012850D19DF8AC1040F2231011FB00F02C
:10E8F0006F4901EBC00018309DF8981001EBC10181
:10E9000000EB011090F87E00E8BB4FF010429DF83C
:10E91000AC0040F2231110FB01F0654901EBC0018E
:10E9200018319DF8980000EBC00001EB00108260E8
:10E930009DF8AC1001EB410000EB01105B4901EBCD
:10E94000001130319DF8980001EB001001789DF81E
:10E95000AC0040F2231210FB02F0554A02EBC0005B
:10E9600041709DF8AC1040F2231011FB00F01146ED
:10E9700001EBC00118319DF8980000EBC00001EBDD
:10E980000010017800E041E09DF8AC0040F2231255
:10E9900010FB02F0464A02EBC0004079814235D1BB
:10E9A00000229DF8AC0040F2231110FB01F0404919
:10E9B00001EBC00118319DF8980000EBC00001EB9D
:10E9C0000010C271A4229DF8AC0040F2231110FB8C
:10E9D00001F0374901EBC00118319DF8980000EBB8
:10E9E000C00001EB00108270A3229DF8AC0040F241
:10E9F000231110FB01F02E4901EBC00018309DF8E7
:10EA0000981001EBC10100EB0110427143E19DF848
:10EA1000AC0000EB4001C1EBC010264901EBC00087
:10EA2000407933287ED19DF8AC0000EB400101EB2A
:10EA300000101E4901EB001030309DF8981000EBDB
:10EA40000110801C0990007820F00100401C0999F9
:10EA500008709DF8AC0000EB400101EB0010134979
:10EA600001EB001030309DF8981000EB0110801C75
:10EA70000990007820F02002099802709DF8AC10EF
:10EA800001EB410000EB0110084901EB00103030B0
:10EA90009DF8981000EB0110801C0990007820F080
:10EAA0000200801C099908700AE00000144100204F
:10EAB000D4450020A8780020BC320020BC120020E1
:10EAC0009DF8AC0040F2231110FB01F0FE4901EB70
:10EAD000C00042799DF8AC0040F2231110FB01F018
:10EAE000F94901EBC00018309DF8981001EBC10105
:10EAF00000EB011002709DF8AC0000EB400101EB4F
:10EB00000010F24901EB001030309DF8981000EB36
:10EB10000110801C0990007820F080008030099955
:10EB2000087000E029E09DF8AC0000EB400101EB2B
:10EB30000010E64901EB001030309DF8981000EB12
:10EB400001108078C0F3400020B99DF8AC1002207D
:10EB5000FBF700FAA2229DF8AC0040F2231110FB53
:10EB600001F0D94901EBC00018309DF8981001EB75
:10EB7000C10100EB011082708DE09DF8AC0000EB4C
:10EB80004001C1EBC010D24901EBC00040793428EC
:10EB90007ED19DF8AC0000EB400101EB0010CB49A9
:10EBA00001EB001030309DF8981000EB0110801C34
:10EBB0000990007820F02002099802709DF8AC00BE
:10EBC00000EB400101EB0010C04901EB00103030B8
:10EBD0009DF8981000EB0110801C0990007820F03F
:10EBE00002020998027001229DF8AC0040F2231144
:10EBF00010FB01F0B44901EBC00018309DF89810EB
:10EC000001EBC10100EB011080F83E20A9229DF824
:10EC1000AC0040F2231110FB01F0AB4901EBC00046
:10EC200018309DF8981001EBC10100EB01108270C3
:10EC30009DF8AC0040F2231110FB01F0A24901EB5A
:10EC4000C00042799DF8AC0040F2231110FB01F0A6
:10EC50009D4901EBC00018309DF8981001EBC101EF
:10EC600000EB011002709DF8AC0000EB400101EBDD
:10EC70000010964901EB001030309DF8981000EB21
:10EC80000110801C0990007820F08000803000E0A6
:10EC900001E00999087000202C902D9000213791F7
:10ECA00021E0DDE92C10000140EA11720901CDE9F3
:10ECB0002C129DF8AC0000EB4001C1EBC010844960
:10ECC00001EBC001BDF8DC00801D085C3038C117C5
:10ECD000DDE92C2402432143CDE92C21BDF8DC00E1
:10ECE000401C81B23791BDF8DC000628D9DB9DF8C5
:10ECF000AC002C9940F2231210FB02F0724A02EB96
:10ED0000C00218329DF8980000EBC00002EB001022
:10ED1000C0F81A1000222C922D920021379122E087
:10ED2000DDE92C10000140EA11720901CDE92C1235
:10ED30009DF8AC1001EB4100C0EBC110644901EB40
:10ED4000C001BDF8DC000D30085C3038C117DDE9CA
:10ED50002C34184341EA0402CDE92C02BDF8DC0052
:10ED6000401C80B23790BDF8DC000428D8DB9DF849
:10ED7000AC002C9940F2231210FB02F0524A02EB35
:10ED8000C00218329DF8980000EBC00002EB0010A2
:10ED9000416300212C912D91379122E0DDE92C1067
:10EDA000000140EA11720901CDE92C129DF8AC1066
:10EDB00001EB4100C0EBC110454901EBC001BDF8BA
:10EDC000DC001130085C3038C117DDE92C34184301
:10EDD00041EA0402CDE92C02BDF8DC00401C80B2FF
:10EDE0003790BDF8DC000628D8DB9DF8AC002C99E4
:10EDF00040F2231210FB02F0334A02EBC002183239
:10EE00009DF8980000EBC00002EB0010C0F81E1047
:10EE10009DF8AC1001EB4100C0EBC1102C4901EB97
:10EE2000C00042799DF8AC0040F2231110FB01F0C4
:10EE3000254901EBC00118319DF8980000EBC00096
:10EE400001EB0010C2709DF8AC1001EB410000EB2B
:10EE500001101E4901EB001130319DF8980001EBC3
:10EE6000001082789DF8AC0040F2231110FB01F0F5
:10EE7000154901EBC00118319DF8980000EBC00066
:10EE800001EB001002769DF8AC1040F2231011FB4C
:10EE900000F00D4901EBC00118319DF8980000EB1E
:10EEA000C00001EB001001789DF8AC0040F2231285
:10EEB00010FB02F0044A02EBC000407981427CDA88
:10EEC00000219DF8AC0005E0D4450020144100204D
:10EED000A878002040F2231210FB02F0FE4A02EB59
:10EEE000C0000171A7229DF8AC0040F2231110FB75
:10EEF00001F0F94901EBC00118319DF8980000EBD1
:10EF0000C00001EB0010427101219DF8AC0040F2FD
:10EF1000231210FB02F0F04A02EBC00001719DF8D1
:10EF2000AC1040F2231011FB00F0114601EBC000C1
:10EF300042799DF8AC0040F2231110FB01F0E64944
:10EF400001EBC00118319DF8980000EBC00001EB07
:10EF500000100270A1229DF8AC0040F2231110FBBA
:10EF600001F0DD4901EBC00118319DF8980000EB7C
:10EF7000C00001EB001042719DF8AC1001EB4100A4
:10EF800000EB0110D54901EB001130319DF89800DC
:10EF900001EB0010801C0990007820F08000803088
:10EFA000099908709DF8AC1001EB410000EB0110CD
:10EFB000CA4901EB0010303000E05BE09DF898108A
:10EFC00000EB0110801C0990007820F00400001D67
:10EFD000099908709DF8AC1001EB410000EB01109D
:10EFE000BE4901EB001030309DF8981000EB011085
:10EFF0008078C0F34010E8B39DF8AC1001EB4100FD
:10F0000000EB0110B54901EB001030309DF898106D
:10F0100000EB0110801C0990007820F02002099874
:10F0200002709DF8AC1001EB410000EB0110AB4900
:10F0300001EB001030309DF8981000EB0110807843
:10F04000C0F34000F0BB9DF8AC1001EB410000EBB9
:10F050000110A24901EB001030309DF8981000EB30
:10F060000110801C0990007820F0080008300999F0
:10F07000087000E0B8E09DF8AC009DF8981001EB36
:10F080000010C217CDE92C0200222C9800EBC00121
:10F0900001EB0011924800EB8100C0F81D209DF8A3
:10F0A000AC0040F2231110FB01F08B4901EBC000D2
:10F0B00018309DF8981001EBC10100EB01102230CF
:10F0C000099000E08BE02C9800EBC00101EB0011EF
:10F0D000834800EB81010D3110220891DDE9080120
:10F0E000F9F7B3F89DF8AC0040F2231110FB01F0E2
:10F0F000794901EBC00118319DF8980000EBC00080
:10F1000001EB00112C9800EBC00202EB00127448D6
:10F1100000EB820051F81A2F40F8012F4968416036
:10F120009DF8AC0000EB400101EB00106B4901EBD6
:10F13000001130319DF8980001EB001001782C98F7
:10F1400000EBC00202EB0012654800F822102C9878
:10F1500000EBC00101EB0011614800EB8101614847
:10F16000C26941F8212F008C88809DF8AC0040F2E4
:10F17000231110FB01F0584901EBC00118319DF833
:10F18000980000EBC00001EB0010416B2C9800EBE5
:10F19000C00202EB0012524800EB8200C0F80910D6
:10F1A0009DF8AC0000EB400101EB00104B4901EB76
:10F1B000001130319DF8980001EB001041682C9847
:10F1C00000EBC00202EB0012454800EB8200C0F8E1
:10F1D00027102C9881B208200991FAF7BBFE9DF800
:10F1E000AC100220FAF7B6FEE6E200219DF8AC0072
:10F1F00040F2231210FB02F0374A02EBC00001710B
:10F200009DF8AC0040F2231110FB01F0114601EB18
:10F21000C00018309DF8981001EBC10100EB0110FF
:10F2200000780A2812DC0B229DF8AC0040F2231172
:10F2300010FB01F0284901EBC00018309DF8981030
:10F2400001EBC10100EB01100270FFE19DF8AC0081
:10F2500040F2231110FB01F01F4901EBC0011831EE
:10F260009DF8980000EBC00001EB001001789DF8BC
:10F27000AC0040F2231210FB02F0174A02EBC00070
:10F28000407981427ED1174890F8A00870BB16489B
:10F29000D0F818020521B0FBF1F201FB120000EBDF
:10F2A000C00101EB00111048243000EB8100002167
:10F2B000C0F81D100C48D0F818020521B0FBF1F27F
:10F2C00001FB120000EBC00101EB001106482430E5
:10F2D00000EB81000D300AE0D445002014410020ED
:10F2E000E4140020BC320020BC120020CEE00990C3
:10F2F0009DF8AC0040F2231110FB01F0FE4901EB38
:10F30000C00118319DF8980000EBC00001EB00101F
:10F3100022301022014608900998F8F796FFF74826
:10F32000D0F818020521B0FBF1F201FB120000EB4E
:10F33000C00101EB0011F148243000EB81029DF87F
:10F34000AC0040F2231110FB01F0EB4901EBC001CE
:10F3500018319DF8980000EBC00001EB001050F848
:10F360001A1F42F8011F40685060E448D0F81802A4
:10F370000521B0FBF1F201FB120000EBC00101EB33
:10F38000001300E062E1DD4924319DF8AC0000EBA0
:10F39000400202EB0010DA4A02EB001230329DF814
:10F3A000980002EB0010007801F82300D348D0F851
:10F3B00018020521B0FBF1F201FB120000EBC001C5
:10F3C00001EB0011CD48243000EB81029DF8AC0028
:10F3D00040F2231110FB01F0C74901EBC0011831C5
:10F3E0009DF8980000EBC00001EB0010406BC2F8E4
:10F3F0000900C248D0F818020521B0FBF1F201FB68
:10F40000120000EBC00101EB0011BC48243000EBFE
:10F410008101BC48C26941F8212F008C8880B7481F
:10F42000D0F818020521B0FBF1F081B20220099159
:10F43000F9F74EFE00210620FAF78CFDAF48D0F810
:10F440001802AE49498C884206D2AC48D0F818025E
:10F45000401CAA49C1F8180200210520FAF77AFDDC
:10F460009DF8AC0000EB400101EB0010A44901EB5A
:10F47000001030309DF8981000EB0110801C0990AE
:10F48000007820F008020998027015E09DF8AC00A1
:10F4900000EB400101EB0010994901EB0010303006
:10F4A0009DF8981000EB0110801C0990007820F066
:10F4B000080008300999087000229DF8AC0040F25D
:10F4C000231110FB01F08C4901EBC00118319DF8AC
:10F4D000980000EBC00001EB001080F83E209DF882
:10F4E000AC100220FAF736FD9DF8AC109DF898009C
:10F4F00000EB0110C217CDE92C0200222C9800EB82
:10F50000C00101EB0011804800EB8100C0F81D2014
:10F510009DF8AC0040F2231110FB01F0764901EB9D
:10F52000C00018309DF8981001EBC10100EB0110EC
:10F53000223009902C9800EBC00101EB00117248B9
:10F5400000EB81010D3110220891DDE90801F8F787
:10F550007CFE9DF8AC0040F2231110FB01F06649DF
:10F5600001EBC00118319DF8980000EBC00001EBE1
:10F5700000112C9800EBC00202EB0012624800EB75
:10F58000820051F81A2F40F8012F496841609DF818
:10F59000AC0000EB400101EB0010594901EB0011F8
:10F5A00030319DF8980001EB001001782C9800EBA9
:10F5B000C00202EB0012544800F822102C9800EB15
:10F5C000C00101EB0011504800EB81014D48C269B8
:10F5D00041F8212F008C88809DF8AC0040F2231167
:10F5E00010FB01F0444901EBC00118319DF898006F
:10F5F00000EBC00001EB0010416B2C9800EBC00247
:10F6000002EB0012404800EB8200C0F809109DF8A0
:10F61000AC0000EB400101EB0010394901EB001197
:10F6200030319DF8980001EB001041682C9800EBF8
:10F63000C00202EB0012344800EB8200C0F8271031
:10F640002C9881B208200991FAF784FCA7229DF832
:10F65000AC0040F2231110FB01F0274901EBC0017F
:10F6600018319DF8980000EBC00001EB00104271CA
:10F67000A2229DF8AC0040F2231110FB01F01E49BC
:10F6800001EBC00118319DF8980000EBC00001EBC0
:10F690000010827000212C912D91379122E0DDE93C
:10F6A0002C10000140EA11720901CDE92C129DF8DD
:10F6B000AC0000EB4001C1EBC010144901EBC001EC
:10F6C000BDF8DC000B30085C3038C117DDE92C34A4
:10F6D00040EA03022143CDE92C21BDF8DC00401CA7
:10F6E00081B23791BDF8DC000A28D8DB9DF8AC0068
:10F6F000DDE92C120CE00000D4450020BC120020F3
:10F7000014410020BC320020E4140020A87800201E
:10F7100040F2231310FB03F0FE4B03EBC00318333E
:10F720009DF8980000EBC00003EB001040F8221F8A
:10F73000426000222C922D920021379122E0DDE9D7
:10F740002C10000140EA11720901CDE92C129DF83C
:10F75000AC0000EB4001C1EBC010EF4901EBC00170
:10F76000BDF8DC001530085C3038C117DDE92C2409
:10F77000104341EA0402CDE92C02BDF8DC00401C34
:10F7800080B23790BDF8DC000A28D8DB9DF8AC00C9
:10F79000DDE92C2140F2231310FB03F0DD4B03EBDA
:10F7A000C00018309DF8983003EBC30300EB031042
:10F7B00022308260C16000BF00BF06F035BE9DF8F8
:10F7C000AC0000EB4001C1EBC010D34911F8300090
:10F7D000042801D124900BE09DF8AC0000EB40011F
:10F7E000C1EBC010CC4911F83000152800D124908D
:10F7F0009DF8AC0000EB4001C1EBC010C64901EB25
:10F80000C00041789DF8AC0000EB4002C2EBC01094
:10F81000C14A12F8300041EA002041F2300188422A
:10F8200002D1A62024903DE09DF8AC0000EB400101
:10F83000C1EBC010B84901EBC00041789DF8AC00A5
:10F8400000EB4002C2EBC010B34A12F8300041EAAC
:10F85000002041F23101884202D1A720249021E00A
:10F860009DF8AC0000EB4001C1EBC010AA4911F8B3
:10F870003000022816D19DF8AC0000EB4001C1EB2E
:10F88000C010A54901EBC00001799DF8AC0000EB68
:10F890004002C2EBC010A04A02EBC000C07841EAAF
:10F8A000002124919DF8AC0040F2231110FB01F0DF
:10F8B000984901EBC000817826910021974A9DF874
:10F8C000AC0002EB00129DF898001154944890F897
:10F8D0002000012815D19DF8AC0000EB400101EBA0
:10F8E0000010904901EB001030309DF8981000EBAB
:10F8F0000110801C0990007820F080008030099968
:10F900000870BDF89000A7287DD007DC04287BD0C4
:10F9100015287AD0A62841F000844AE0A0F5585076
:10F92000303820B1112871D01228F4D1FEE39DF8AF
:10F93000AC0040F2231110FB01F0764901EBC0004E
:10F9400018309DF8981001EBC10100EB0110007810
:10F9500070BB00219DF8AC0040F2231210FB02F0B6
:10F960006C4A02EBC000017101229DF8AC0040F22C
:10F97000231110FB01F0674901EBC00118319DF81C
:10F98000980000EBC00001EB00100270A7229DF868
:10F99000AC0040F2231110FB01F05E4901EBC00006
:10F9A00018309DF8981001EBC10100EB0110427175
:10F9B000FDE300219DF8AC0040F2231210FB02F0A1
:10F9C000544A02EBC00001719DF8AC0040F22311D3
:10F9D00010FB01F0114601EBC00018309DF89810A3
:10F9E00001EBC10100EB01100078022829DC0322A1
:10F9F0009DF8AC0040F2231110FB01F0454901EBEA
:10FA0000C001183103E0D0E02EE158E286E29DF813
:10FA1000980000EBC00001EB00100270A9229DF8D5
:10FA2000AC0040F2231110FB01F03A4901EBC00099
:10FA300018309DF8981001EBC10100EB01104271E4
:10FA4000B2E09DF8AC0040F2231110FB01F0314907
:10FA500001EBC00018309DF8981001EBC10100EBDC
:10FA600001100078052824DC06229DF8AC0040F245
:10FA7000231110FB01F0274901EBC00118319DF85B
:10FA8000980000EBC00001EB00100270A2229DF86C
:10FA9000AC0040F2231110FB01F01E4901EBC00045
:10FAA00018309DF8981001EBC10100EB0110427174
:10FAB0007AE09DF8AC0040F2231110FB01F01549EB
:10FAC00001EBC00018309DF8981001EBC10100EB6C
:10FAD00001104079A52815D19DF8AC0000EB40013C
:10FAE00001EB00100F4901EB001030309DF8981029
:10FAF00000EB0110801C0990007820F00400001D2C
:10FB0000099908709DF8AC0040F2231110FB01F038
:10FB1000004909E0D4450020A8780020483F002093
:10FB2000BC1200201441002001EBC00018309DF8E9
:10FB3000981001EBC10100EB01108078A12833D0AF
:10FB40009DF8AC0040F2231110FB01F0FE4901EBDF
:10FB5000C00118319DF8980000EBC00001EB0010C7
:10FB600082789DF8AC0040F2231110FB01F0F649B9
:10FB700001EBC00118319DF8980000EBC00001EBCB
:10FB800000104271A1229DF8AC0040F2231110FB3D
:10FB900001F0ED4901EBC00018309DF8981001EB21
:10FBA000C10100EB0110827002E79DF8AC0040F249
:10FBB000231110FB01F0E44901EBC00018309DF85F
:10FBC000981001EBC10100EB01104079A4282DD160
:10FBD0009DF8AC0000EB400101EB0010DB4901EBAC
:10FBE000001030309DF8981000EB0110801C099037
:10FBF000007820F0200020300999087000229DF83C
:10FC0000AC0040F2231110FB01F0CF4901EBC00022
:10FC100018309DF8981001EBC10100EB011080F83D
:10FC20003D209DF8AC100220FAF794F900219DF8D0
:10FC3000AC0040F2231210FB02F0C34A02EBC000FA
:10FC40000171A1229DF8AC0040F2231110FB01F0DC
:10FC5000BD4901EBC00018309DF8981001EBC101BF
:10FC600000EB01104271A3E69DF8AC0040F22311B5
:10FC700010FB01F0B44901EBC00018309DF898105A
:10FC800001EBC10100EB0110007801282FDC0021FD
:10FC90009DF8AC0040F2231210FB02F0AA4A02EBDE
:10FCA000C000017102229DF8AC0040F2231110FB4C
:10FCB00001F0A54901EBC00118319DF8980000EB57
:10FCC000C00001EB00100270A3229DF8AC0040F2CE
:10FCD000231110FB01F09C4901EBC00018309DF886
:10FCE000981001EBC10100EB01104271E6E09DF8B4
:10FCF000AC0040F2231110FB01F0934901EBC0006E
:10FD000018309DF8981001EBC10100EB011000784C
:10FD100004282FDC00219DF8AC0040F2231210FBD8
:10FD200002F0894A02EBC000017105229DF8AC0087
:10FD300040F2231110FB01F0834901EBC00118319F
:10FD40009DF8980000EBC00001EB00100270A322A8
:10FD50009DF8AC0040F2231110FB01F07A4901EB51
:10FD6000C00018309DF8981001EBC10100EB0110A4
:10FD70004271A3E09DF8AC0040F2231110FB01F0AA
:10FD8000714901EBC00018309DF8981001EBC101DA
:10FD900000EB01100078062812DCA1229DF8AC00CF
:10FDA00040F2231110FB01F0674901EBC00018304D
:10FDB0009DF8981001EBC10100EB011042717DE04C
:10FDC0009DF8AC0040F2231110FB01F05E4901EBFD
:10FDD000C00118319DF8980000EBC00001EB001045
:10FDE00001789DF8AC0040F2231210FB02F0564A55
:10FDF00002EBC0004079814260D19DF8AC0040F236
:10FE0000231110FB01F0114601EBC00018309DF8E2
:10FE1000981001EBC10100EB01108078A12830D0CF
:10FE2000A3229DF8AC0040F2231110FB01F04649DB
:10FE300001EBC00118319DF8980000EBC00001EB08
:10FE4000001042719DF8AC0040F2231110FB01F04C
:10FE50003D4901EBC00018309DF8981001EBC1013D
:10FE600000EB01108078A22828D000209DF8AC106B
:10FE700040F2231211FB02F1334A02EBC101087177
:10FE80001CE0A1229DF8AC0040F2231110FB01F010
:10FE90002D4901EBC00118319DF8980000EBC0001E
:10FEA00001EB0010427101219DF8AC0040F22312D9
:10FEB00010FB02F0244A02EBC000017178E5A12298
:10FEC0009DF8AC0040F2231110FB01F01E4901EB3C
:10FED000C00118319DF8980000EBC00001EB001044
:10FEE00042719DF8AC0040F2231110FB01F016495D
:10FEF00001EBC00118319DF8980000EBC00001EB48
:10FF00000010827000219DF8AC0040F2231210FB1B
:10FF100002F00D4A02EBC000017149E500219DF895
:10FF2000AC0040F2231210FB02F0074A02EBC000C3
:10FF30000171A7229DF8AC0040F2231110FB01F0E3
:10FF4000014901EBC00103E0D44500201441002029
:10FF500018319DF8980000EBC00001EB00104271D1
:10FF60009DF8AC0000EB4001C1EBC010F74901EB7C
:10FF7000C000407930287DD19DF8AC0040F22311BB
:10FF800010FB01F0F24901EBC00118319DF8980017
:10FF900000EBC00001EB001001789DF8AC0040F2CE
:10FFA000231210FB02F0EA4A02EBC00040798142C2
:10FFB00060D19DF8AC0000EB400101EB0010A2F510
:10FFC000986101EB001030309DF8981000EB0110A3
:10FFD000801C0990007820F00102099802709DF8B9
:10FFE000AC0000EB400101EB0010DA4901EB00101E
:10FFF00030309DF8981000EB0110801C09900078BB
:020000040801F1
:1000000020F00202099802709DF8AC0040F2231122
:1000100010FB01F0CE4901EBC00018309DF898109C
:1000200001EBC10100EB0110C07831282ED19DF801
:10003000AC0000EB400101EB0010C64901EB0010E1
:1000400030309DF8981000EB0110801C099000786A
:1000500020F020020998027000229DF8AC0040F2C6
:10006000231110FB01F0BA4901EBC00018309DF8D4
:10007000981000E031E001EBC10100EB011080F8C5
:100080003D209DF8AC100220F9F764FF9DF8AC10FC
:1000900040F2231011FB00F0AD4901EBC000183015
:1000A0009DF8981001EBC10100EB011090F83E00A3
:1000B000012811D1A9229DF8AC0040F2231110FBB8
:1000C00001F0A34901EBC00018309DF8981001EB36
:1000D000C10100EB011082707AE29DF8AC1001EBD7
:1000E0004100C0EBC110994901EBC00040793128B3
:1000F0007ED19DF8AC1040F2231011FB00F0944922
:1001000001EBC00118319DF8980000EBC00001EB35
:10011000001001789DF8AC0040F2231210FB02F0B1
:100120008B4A02EBC0004079814200E0ECE35FD1F2
:100130009DF8AC1040F2231011FB00F0114601EBCA
:10014000C00018309DF8981001EBC10100EB0110C0
:1001500090F83E0040BB01229DF8AC0040F2231114
:1001600010FB01F07A4901EBC00118319DF89800AD
:1001700000EBC00001EB001080F83D209DF8AC10B2
:1001800001EB410000EB0110724901EB001030302F
:100190009DF8981000EB0110801C0990007820F069
:1001A0000100401C099908709DF8AC1000E0FCE3C8
:1001B00001EB410000EB0110664901EB001030300B
:1001C0009DF8981000EB0110801C0990007820F039
:1001D000020209980270604890F8A008F0BB5F48DE
:1001E00090F82100012839D15C48D0F8180200E0CD
:1001F000B6E05A49498C884230D29DF8AC1040F2A2
:10020000231011FB00F0524901EBC00018309DF89B
:10021000981001EBC10100EB011090F83D0001289E
:100220001CD19DF8AC1040F2231011FB00F048499E
:1002300001EBC00018309DF8981001EBC10100EBF4
:10024000011090F87E0048B94FF010429DF8AC00C4
:1002500040F2231110FB01F03D4900E075E001EB95
:10026000C00118319DF8980000EBC00001EB0010B0
:1002700082609DF8AC1001EB410000EB01103549A4
:1002800001EB001130319DF8980001EB001001786E
:100290009DF8AC0040F2231210FB02F02C4A02EB56
:1002A000C00041709DF8AC1040F2231011FB00F02B
:1002B000114601EBC00118319DF8980000EBC00019
:1002C00001EB001001789DF8AC0040F2231210FB06
:1002D00002F01F4A02EBC0004079814235D1002272
:1002E0009DF8AC0040F2231110FB01F0184901EB1E
:1002F000C00118319DF8980000EBC00001EB001020
:10030000C271A4229DF8AC0040F2231110FB01F051
:100310000F4901EBC00118319DF8980000EBC000B7
:1003200001EB00108270A3229DF8AC0040F2231173
:1003300010FB01F0064901EBC00018309DF8981041
:1003400001EBC10100EB0110427141E1A8780020EE
:10035000D445002014410020BC320020BC120020F3
:100360009DF8AC1001EB4100C0EBC110FE4901EB60
:10037000C000407933287CD19DF8AC1001EB4100DE
:1003800000EB0110F94901EB001030309DF8981096
:1003900000EB0110801C0990007820F00100401C47
:1003A000099908709DF8AC1001EB410000EB0110B9
:1003B000EE4901EB001030309DF8981000EB011071
:1003C000801C0990007820F02002099802709DF8A6
:1003D000AC1001EB410000EB0110E44901EB00100F
:1003E00030309DF8981000EB0110801C09900078C7
:1003F00020F00200801C099908709DF8AC1040F2B2
:10040000231011FB00F0DA4901EBC00042799DF89E
:10041000AC0040F2231110FB01F0D54901EBC00004
:1004200018309DF8981001EBC10100EB011002702B
:100430009DF8AC1001EB410000EB0110CB4901EB42
:10044000001030309DF8981000EB0110801C0990CE
:10045000007820F080008030099908709DF8AC1079
:1004600001EB410000EB0110C04901EB00103030FE
:1004700000E01FE09DF8981000EB01108078C0F3B9
:10048000400020B99DF8AC100220F9F763FDA222CC
:100490009DF8AC0040F2231110FB01F0B44901EBD0
:1004A000C00018309DF8981001EBC10100EB01105D
:1004B00082708DE09DF8AC1001EB4100C0EBC110E3
:1004C000A94901EBC000407934287DD19DF8AC10DA
:1004D00001EB410000EB0110A44901EB00103030AA
:1004E0009DF8981000EB0110801C0990007820F016
:1004F0002002099802709DF8AC1001EB410000EB5E
:1005000001109A4901EB001030309DF8981000EB73
:100510000110801C0990007820F0020209980270F6
:1005200001229DF8AC0040F2231110FB01F090492C
:1005300001EBC00018309DF8981001EBC10100EBF1
:10054000011080F83E20A9229DF8AC0040F2231152
:1005500010FB01F0864901EBC00018309DF898109F
:1005600001EBC10100EB011082709DF8AC1040F26C
:10057000231011FB00F07E4901EBC00042799DF889
:10058000AC0040F2231110FB01F0794901EBC000EF
:1005900018309DF8981001EBC10100EB01100270BA
:1005A0009DF8AC1001EB410000EB01106F4901EB2D
:1005B000001030309DF8981000EB0110801C09905D
:1005C000007820F0800000E002E080300999087097
:1005D00000202C902D900021379122E0DDE92C1095
:1005E000000140EA11720901CDE92C129DF8AC100E
:1005F00001EB4100C0EBC1105B4901EBC001BDF84C
:10060000DC00801D085C3038C117DDE92C24104364
:1006100041EA0402CDE92C02BDF8DC00401C80B2A6
:100620003790BDF8DC000828D8DB9DF8AC002C9989
:1006300040F2231210FB02F04D4A02EBC0021832C6
:100640009DF8980000EBC00002EB0010C0F81A10F3
:1006500000222C922D920021379122E0DDE92C100E
:10066000000140EA11720901CDE92C129DF8AC108D
:1006700001EB4100C0EBC1103B4901EBC001BDF8EB
:10068000DC000F30085C3038C117DDE92C3418432A
:1006900041EA0402CDE92C02BDF8DC00401C80B226
:1006A0003790BDF8DC000628D8DB9DF8AC002C990B
:1006B00040F2231210FB02F02D4A02EBC002183266
:1006C0009DF8980000EBC00002EB0010416300228F
:1006D0002C922D920021379122E0DDE92C100001AF
:1006E00040EA11720901CDE92C129DF8AC1001EB22
:1006F0004100C0EBC1101C4901EBC001BDF8DC009A
:100700001530085C3038C117DDE92C34184341EA54
:100710000402CDE92C02BDF8DC00401C80B2379009
:10072000BDF8DC000828D8DB9DF8AC002C9940F21D
:10073000231210FB02F00E4A02EBC00218329DF8A1
:10074000980000EBC00002EB0010C0F81E109DF8EE
:10075000AC1001EB4100C0EBC110034901EBC0003C
:1007600042799DF8AC0005E0A878002014410020F3
:10077000D445002040F2231110FB01F0FE4901EBAB
:10078000C00118319DF8980000EBC00001EB00108B
:10079000C2709DF8AC1001EB410000EB0110F7496D
:1007A00001EB001130319DF8980001EB00108278C8
:1007B0009DF8AC0040F2231110FB01F0EE4901EB73
:1007C000C00118319DF8980000EBC00001EB00104B
:1007D00002769DF8AC1040F2231011FB00F0E649C0
:1007E00001EBC00118319DF8980000EBC00001EB4F
:1007F000001001789DF8AC0040F2231210FB02F0CB
:10080000DD4A02EBC000407981427CDA00219DF88C
:10081000AC0040F2231210FB02F0D74A02EBC000FA
:100820000171A7229DF8AC0040F2231110FB01F0EA
:10083000D14901EBC00118319DF8980000EBC000D0
:1008400001EB0010427101219DF8AC0040F223122F
:1008500010FB02F0C84A02EBC00001719DF8AC1019
:1008600040F2231011FB00F0114601EBC000427969
:100870009DF8AC0040F2231110FB01F0BE4901EBE2
:10088000C00118319DF8980000EBC00001EB00108A
:100890000270A1229DF8AC0040F2231110FB01F080
:1008A000B54901EBC00118319DF8980000EBC0007C
:1008B00001EB001042719DF8AC1001EB410000EB20
:1008C0000110AE4901EB001130319DF8980001EBA9
:1008D0000010801C0990007820F080018031099878
:1008E00001709DF8AC1001EB410000EB0110A34931
:1008F00001EB001130319DF8980001EB0010801CD5
:100900000990007801E051E010E120F00400001DA2
:10091000099908709DF8AC1001EB410000EB011043
:10092000964901EB001030309DF8981000EB011053
:100930008078C0F34010C8B39DF8AC1001EB4100C3
:1009400000EB01108D4901EB001030309DF898103C
:1009500000EB0110801C0990007820F0200209981B
:1009600002709DF8AC1001EB410000EB01108349CF
:1009700001EB001030309DF8981000EB01108078EA
:10098000C0F34000F0BB9DF8AC1001EB410000EB60
:1009900001107A4901EB001030309DF8981000EBFF
:1009A0000110801C0990007801E0B6E3BDE020F062
:1009B00008000830099908709DF8AC009DF898105F
:1009C00001EB0010C217CDE92C0200222C9800EB9D
:1009D000C00101EB00116A4800EB8100C0F81D2046
:1009E0009DF8AC1040F2231011FB00F0624901EBBE
:1009F000C00018309DF8981001EBC10100EB011008
:100A0000223000E08CE009902C9800EBC00101EB53
:100A100000115B4800EB81010D3110220891DDE9E6
:100A20000801F7F712FC9DF8AC1040F2231011FBFF
:100A300000F0514901EBC00118319DF8980000EB1E
:100A4000C00001EB00112C9800EBC00202EB001279
:100A50004B4800EB820051F81A2F40F8012F4968EB
:100A600041609DF8AC1001EB410000EB01104349DF
:100A700001EB001130319DF8980001EB0010017876
:100A80002C9800EBC00202EB00123D4800F8221047
:100A90002C9800EBC00101EB0011394800EB8101FB
:100AA0003848C26941F8212F008C88809DF8AC102D
:100AB00040F2231011FB00F02F4901EBC001183167
:100AC0009DF8980000EBC00001EB0010416B2C98E2
:100AD00000EBC00202EB0012294800EB8200C0F8D4
:100AE00009109DF8AC1001EB410000EB0110234907
:100AF00001EB001130319DF8980001EB00104168C6
:100B00002C9800EBC00202EB00121D4800EB8200A3
:100B1000C0F827102C9881B208200991F9F71AFA29
:100B20009DF8AC100220F9F715FAF6E200219DF8C5
:100B3000AC0040F2231210FB02F00F4A02EBC0009F
:100B400001719DF8AC1040F2231011FB00F011462A
:100B500001EBC00018309DF8981001EBC10100EBCB
:100B60000110007803281BDC04229DF8AC0040F241
:100B7000231110FB01F007E0D445002014410020B0
:100B8000E4140020BC320020FE4901EBC000183004
:100B90009DF8981001EBC10100EB0110027000E21A
:100BA0009DF8AC0040F2231110FB01F0F54901EB78
:100BB000C00118319DF8980000EBC00001EB001057
:100BC00001789DF8AC0040F2231210FB02F0ED4AD0
:100BD00002EBC000407981427DD1EB4890F8A0083B
:100BE000E8BBEA48D0F818020521B0FBF1F201FB9E
:100BF000120000EBC00101EB0011E448243000EBCF
:100C000081000021C0F81D10E048D0F8180205212D
:100C1000B0FBF1F201FB120000EBC00101EB00118F
:100C2000DA48243000EB81000D3009909DF8AC00CB
:100C300040F2231110FB01F2D24800EBC20118313F
:100C40009DF8980000EBC00001EB0010223010224C
:100C5000014608900998F7F7F8FACC4800E0B5E0AB
:100C6000D0F818020521B0FBF1F201FB120000EBF5
:100C7000C00101EB0011C548243000EB81029DF852
:100C8000AC0040F2231110FB01F0BE4901EBC001A2
:100C900018319DF8980000EBC00001EB001050F8EF
:100CA0001A1F42F8011F40685060B848D0F8180277
:100CB0000521B0FBF1F201FB120000EBC00101EBDA
:100CC0000013B24924319DF8AC0000EB400202EB66
:100CD0000010AF4A00E064E102EB001230329DF8F0
:100CE000980002EB0010007801F82300A748D0F824
:100CF00018020521B0FBF1F201FB120000EBC0016C
:100D000001EB0011A148243000EB81029DF8AC00FA
:100D100040F2231110FB01F09A4901EBC001183198
:100D20009DF8980000EBC00001EB0010406BC2F88A
:100D300009009648D0F818020521B0FBF1F201FB3A
:100D4000120000EBC00101EB00119048243000EBD1
:100D500081018D48C26941F8212F008C88808B4821
:100D6000D0F818020521B0FBF1F081B20220099100
:100D7000F8F7AEF900210620F9F7ECF88348D0F82F
:100D800018028249498C884206D28048D0F818025D
:100D9000401C7E49C1F8180200210520F9F7DAF855
:100DA0009DF8AC0000EB400101EB0010784901EB2D
:100DB000001030309DF8981000EB0110801C099055
:100DC000007820F008020998027015E09DF8AC0048
:100DD00000EB400101EB00106D4901EB00103030D9
:100DE0009DF8981000EB0110801C0990007820F00D
:100DF000080008300999087000229DF8AC0040F204
:100E0000231110FB01F05F4901EBC00118319DF87F
:100E1000980000EBC00001EB001080F83E209DF828
:100E2000AC100220F9F796F89DF8AC109DF89800E8
:100E300000EB0110C217CDE92C0200222C9800EB28
:100E4000C00101EB0011534800EB8100C0F81D20E8
:100E50009DF8AC0040F2231110FB01F0494901EB71
:100E6000C00018309DF8981001EBC10100EB011093
:100E7000223009902C9800EBC00101EB001145488D
:100E800000EB81010D3110220891DDE90801F7F72F
:100E9000DCF99DF8AC0040F2231110FB01F0394958
:100EA00001EBC00118319DF8980000EBC00001EB88
:100EB00000112C9800EBC00202EB0012354800EB49
:100EC000820051F81A2F40F8012F496841609DF8BF
:100ED000AC0000EB400101EB00102D4901EB0011CB
:100EE00030319DF8980001EB001001782C9800EB50
:100EF000C00202EB0012274800F822102C9800EBE9
:100F0000C00101EB0011234800EB81011E48C269BA
:100F100041F8212F008C88809DF8AC0040F223110D
:100F200010FB01F0174901EBC00118319DF8980042
:100F300000EBC00001EB0010416B2C9800EBC002ED
:100F400002EB0012134800EB8200C0F809109DF874
:100F5000AC0000EB400101EB00100D4901EB00116A
:100F600030319DF8980001EB001041682C9800EB9F
:100F7000C00202EB0012074800EB8200C0F8271005
:100F80002C9809E0D4450020BC320020BC1200207F
:100F900014410020E414002081B208200991F8F7E0
:100FA000D9FF00229DF8AC0040F2231110FB01F0A4
:100FB000FA4901EBC00118319DF8980000EBC00020
:100FC00001EB001080F83E20A7229DF8AC0040F213
:100FD000231110FB01F0F14901EBC00118319DF81C
:100FE000980000EBC00001EB00104271A2229DF8B6
:100FF000AC0040F2231110FB01F0E84901EBC00105
:1010000018319DF8980000EBC00001EB00108270D1
:1010100000222C922D920021379122E0DDE92C1044
:10102000000140EA11720901CDE92C129DF8AC00D3
:1010300000EB4001C1EBC010D94901EBC001BDF884
:10104000DC000B30085C3038C117DDE92C34184364
:1010500041EA0402CDE92C02BDF8DC00401C80B25C
:101060003790BDF8DC000C28D8DB9DF8AC00DDE93A
:101070002C1240F2231310FB03F0C84B03EBC00308
:1010800018339DF8980000EBC00003EB001040F807
:10109000221F426000222C922D920021379122E0E3
:1010A000DDE92C10000140EA11720901CDE92C1292
:1010B0009DF8AC0000EB4001C1EBC010B84901EB5A
:1010C000C001BDF8DC001730085C3038C117DDE91D
:1010D0002C34184341EA0402CDE92C02BDF8DC00AF
:1010E000401C80B23790BDF8DC000C28D8DB9DF89E
:1010F000AC00DDE92C1240F2231310FB03F0A74BE8
:1011000003EBC00018309DF8983003EBC30300EBED
:10111000031022308160C26000BF00BF05F084B9B7
:101120000021A04A9DF8AC0002EB00129DF8980047
:1011300011549DF8AC0000EB4001C1EBC010984980
:1011400001EBC000407870280ED19DF8AC0000EB98
:101150004001C1EBC010924901EBC0008078FA2831
:1011600002D1B121249142E09DF8AC0000EB400196
:10117000C1EBC0108A4901EBC000407800F0F000DC
:10118000C0280ED19DF8AC0000EB4001C1EBC010AF
:10119000834901EBC0008078FA2802D1B620249060
:1011A00025E09DF8AC0000EB4001C1EBC0107C498C
:1011B00011F8300000F0F000502818D19DF8AC0074
:1011C00000EB4001C1EBC010754901EBC000407855
:1011D00000F0F00030280AD19DF8AC0000EB40018F
:1011E000C1EBC0106E4901EBC000817824919DF8DD
:1011F000AC0040F2231110FB01F0684901EBC00084
:10120000817826910021674A9DF8AC0002EB00121C
:101210009DF898001154644890F82000012815D1D9
:101220009DF8AC0000EB400101EB00105F4901EBC1
:10123000001030309DF8981000EB0110801C0990D0
:10124000007820F08000803009990870BDF8900087
:10125000652874D004DC012809D0032805D175E085
:10126000B12802D0B62800D100E082E181E19DF8EA
:10127000AC0000EB4001C1EBC010494901EBC000DC
:101280000079012806D0022805D0032804D00528BB
:101290005AD102E058E057E056E09DF8AC0040F229
:1012A000231110FB01F03D4901EBC00018309DF8FF
:1012B000981001EBC10100EB01100078F0BB002198
:1012C0009DF8AC0040F2231210FB02F0334A02EB0F
:1012D000C000017101229DF8AC0040F2231110FB07
:1012E00001F02E4901EBC00118319DF8980000EB88
:1012F000C00001EB00100270B6229DF8AC0040F275
:10130000231110FB01F0254901EBC00118319DF8B4
:10131000980000EBC00001EB00104271B2229DF872
:10132000AC0040F2231110FB01F01C4901EBC0009E
:1013300018309DF8981001EBC10101E003E039E09D
:1013400000EB0110827000BF00BF12E19DF8AC00FD
:1013500000EB4001C1EBC010114901EBC000C179A5
:10136000134880F8141E9DF8AC0000EB400101EB1F
:1013700000100E4901EB001130319DF8980001EB8F
:101380000010801C09900A4890F8140EC2080998B1
:10139000007862F3000009990870EAE0D445002063
:1013A000A8780020483F0020BC12002014410020F3
:1013B000BC2200209DF8AC0000EB4001C1EBC01046
:1013C000FE4901EBC000007900F0F00010B9B8212F
:1013D000249101E0B92124919DF8AC0000EB40017B
:1013E000C1EBC010F54901EBC000007900F00F011E
:1013F00025910021379120E09DF8AC0000EB4001E1
:1014000001EB0010EE4901EB00113031BDF8DC00BA
:1014100001EB001041789DF8AC0000EB4002C2EBFC
:10142000C010E64A12F830005038814200D112E074
:10143000BDF8DC00401C81B237919DF8AC0000EB98
:10144000400101EB0010DE4901EB0010C179BDF84D
:10145000DC008142D0DC00BFBDF8DC109DF89400B8
:101460000844C1B226919DF8AC0040F2231110FB54
:1014700001F0D44901EBC00018309DF8981001EB41
:10148000C10100EB0110007801282FD100219DF847
:10149000AC0040F2231210FB02F0CA4A02EBC0007B
:1014A000017102229DF8AC0040F2231110FB01F003
:1014B000C44901EBC00118319DF8980000EBC00051
:1014C00001EB00100270B9229DF8AC0040F223112C
:1014D00010FB01F0BB4901EBC00018309DF89810DB
:1014E00001EBC10100EB0110427141E09DF8AC003D
:1014F00040F2231110FB01F0B24901EBC00018309B
:101500009DF8981001EBC10100EB01100078012853
:101510002ED100219DF8AC0040F2231210FB02F006
:10152000A84A02EBC000017102229DF8AC0040F213
:10153000231110FB01F0A34901EBC00118319DF804
:10154000980000EBC00001EB00100270B9229DF87A
:10155000AC0040F2231110FB01F09A4901EBC000EE
:1015600018309DF8981001EBC10100EB0110427199
:1015700000BF00BFD2E59DF8AC0000EB400101EBDD
:1015800000108F4901EB0010007B20B101287DD0B5
:1015900002287CD1E8E28C499DF8AC0031F81000BB
:1015A000801F81B209919DF8AC0000EB4001C1EBB6
:1015B000C011824800EBC100401C08900999F8F75F
:1015C00089F90022CDE92E029DF8AC0000EB400124
:1015D000C1EBC010794901EBC0027B489DF8AC100B
:1015E00030F81100401F111809910421099815F0D5
:1015F00059FCC217CDE92C022DA819C82C995940C5
:10160000604001437DD1714A9DF8AC0002EB0010AF
:1016100001709DF8AC0000EB4001C1EBC0106749C0
:1016200001EBC00001792491BDF89000312802D06F
:10163000452867D1FAE064489DF8AC1030F81100F5
:101640001838412190FBF1F0C217C1B2CDE92C024C
:101650005F4880F8BC1100203790DDE09DF8AC00B9
:1016600000EB4001C1EBC010544901EBC001BDF8D3
:10167000DC0000EB80101430095C564ABDF8DC0039
:1016800011549DF8AC0000EB400101E0D1E06AE2AA
:10169000C1EBC010494901EBC001BDF8DC0000EB13
:1016A00080101A30014409910821099815F0B8FBFF
:1016B0008DED0E0A474A0C32BDF8DC000E9902EBA4
:1016C000001041609DF8AC0000EB4001C1EBC01080
:1016D0003A4901EBC001BDF8DC0000EB801032306C
:1016E000014409910821099815F09AFB8DED0E0A25
:1016F000384A0C32BDF8DC000E9902EB0010016094
:1017000001E095E093E09DF8AC0000EB4001C1EBF7
:10171000C0102A4901EBC001BDF8DC0000EB8010CD
:101720003A30014409910821099815F079FB8DEDB3
:101730000E0A284A0C32BDF8DC000E9902EB0010AC
:1017400081609DF8AC0000EB4001C1EBC0101B496B
:1017500001EBC001BDF8DC0000EB80104230014419
:1017600009910821099815F05BFB8DED0E0A194AC5
:101770000C32BDF8DC000E9902EB0010C1609DF840
:10178000AC0000EB400101EB00100D4901EB001132
:101790003031BDF8DC0001EB0010801C09900078AE
:1017A00020F080008030099908709DF8AC0000EBB3
:1017B0004001C1EBC01001490EE00000A8780020F4
:1017C00014410020D4450020346A0020483F002006
:1017D000BC3200207934002001EBC002FE489DF8A5
:1017E000AC1030F81100401E125C9DF8AC0040F2C5
:1017F000231110FB01F0F94901EBC00018309DF8EE
:10180000981001EBC10100EB011080F83C20BDF8FD
:10181000DC00401C80B23790BDF8DC000021DDE91F
:101820002C34C01AA141FFF619AF00E000BF00BF81
:10183000AFE29DF8AC0000EB4001C1EBC010E849FD
:1018400001EBC000407D9DF8AC1001EB4102C2EB02
:10185000C111E34A02EBC101897D40EA0120C217B0
:10186000CDE92C029DF8AC0000EB4001C1EBC011AA
:10187000DB4800EBC101099115210998F8F70EF832
:101880000022CDE92E022DA819C82C99594060409C
:1018900001437CD19DF8AC0000EB4001C1EBC010CE
:1018A000CF4911F83000401EC1B226910021CD4A27
:1018B0009DF8AC0002EB00129DF898001154002234
:1018C000C9499DF898000A549FEDC80A10EE101AF5
:1018D000C54A0C329DF8980002EB001041609DF85B
:1018E000AC0000EB4001C1EBC010BD4901EBC000F2
:1018F00081799DF8AC0000EB4002C2EBC010B84A01
:1019000002EBC000407941EA002000EE100AB8EE78
:10191000C00A9FEDB71AC0EE010A9DF8AC0000EBBB
:101920004001C1EBC010114601EBC00001799DF8E8
:10193000AC0000EB4002C2EBC010A94A02EBC000B1
:10194000C07841EA002000EE100AB8EEC00A30EE7E
:10195000800A10EE101AA44A0C329DF8980002EB8F
:10196000001001609DF8AC0000EB4001C1EBC0101D
:101970009B4901EBC000817A9DF8AC0000EB40026E
:10198000C2EBC010964A02EBC000407A00E0EAE0E9
:1019900041EA002000EE100AB8EEC00A9FED941A4A
:1019A000C0EE010A9DF8AC0000EB4001C1EBC01095
:1019B000114601EBC000017A9DF8AC0000EB40023B
:1019C000C2EBC010864A02EBC000C07941EA002099
:1019D00000EE100AB8EEC00A30EE800A10EE101ABF
:1019E000814A0C329DF8980002EB001081609DF84E
:1019F000AC0000EB4001C1EBC010794901EBC00025
:101A0000C07A00F0800038BB9DF8AC0000EB4001CC
:101A1000C1EBC010724901EBC000017B9DF8AC0026
:101A200000EB4002C2EBC0106D4A02EBC000C07A6E
:101A300041EA002000EE100AF8EEC00AB3EE001AE8
:101A400080EE810A10EE100A674A0C329DF8981059
:101A500002EB0111C86047E09DF8AC0000EB4001CB
:101A6000C1EBC0105E4901EBC000017B9DF8AC00EA
:101A700000EB4002C2EBC010594A02EBC000C07A32
:101A800041EA0020404280B200EE100AB8EEC00ADF
:101A90008DED030A0398F6F741FE9FED560B53ECCC
:101AA000102BCDE904019DED040B51EC100BF6F762
:101AB00019FD9FED520B53EC102BCDE906019DED66
:101AC000060B51EC100BF6F798FCCDE908019DEDE3
:101AD000080B51EC100BF6F734FE434A0C329DF81C
:101AE000981002EB0111C8609DF8AC0000EB4001BA
:101AF00001EB0010434901EB001030309DF89810C5
:101B000000EB0110801C0990007820F080008030EC
:101B1000099908709DF8AC1001EB4100C0EBC110B1
:101B20002F4901EBC000C27D9DF8AC0040F22311AB
:101B300010FB01F0294901EBC00018309DF8981006
:101B400001EBC10100EB011080F83C209DF8AC10C6
:101B500001EB410000EB01102A4901EB0010C179B3
:101B6000294880F8BC1114E19DF8AC1001EB41004C
:101B7000C0EBC1101A4901EBC000C0799DF8AC1050
:101B800001EB4102C2EBC111154A02EBC101097A16
:101B900040EA0120C217CDE92C029DF8AC1001EB00
:101BA0004100C0EBC1100E4901EBC00109910721B2
:101BB0000998F7F773FE0022CDE92E02DDE92E42E7
:101BC000DDE92C106140504001437DD19DF8AC10FF
:101BD00001EB41001AE00000346A0020D4450020E7
:101BE000A8780020483F0020793400200000000041
:101BF00000FF7F47000000000000304000000000B0
:101C00000000000014410020BC320020C0EBC110D5
:101C1000FE4911F83000401EC1B226910021FC4A55
:101C20009DF8AC0002EB00100170A2F6CF229DF8E7
:101C3000980011549DF8AC1001EB4100C0EBC110AD
:101C4000F24901EBC000817908460191F6F7E0FC0A
:101C5000CDE902019DED021B9FEDEE0B18F044FE55
:101C60008DED060B9DF8AC1001EB4100C0EBC110EF
:101C7000E64901EBC00001799DF8AC0000EB4002A1
:101C8000C2EBC010E14A02EBC000C07841EA00207C
:101C900000EE100AB8EEC00A8DED030A0398F6F7BD
:101CA0003DFDCDE904019DED060B53EC102B9DEDA0
:101CB000040B51EC100BF6F715FCCDE908019DED76
:101CC000080B51EC100B00E062E0F6F73AFDD34A46
:101CD0009DF8981002EB011148601FED3C0A10EED0
:101CE000101A9DF8980002EB001001601FED410AE8
:101CF00010EE101A9DF8980002EB001081601FEDA5
:101D0000450A10EE101A9DF8980002EB0010C16011
:101D10009DF8AC1001EB410000EB011002F68F4181
:101D200001EB001130319DF8980001EB0010801C90
:101D30000990007820F080018031099801709DF8A9
:101D4000AC1001EB4100C0EBC110B04901EBC00089
:101D5000427A9DF8AC0040F2231110FB01F0B0492B
:101D600001EBC00118319DF8980000EBC00001EBB9
:101D7000001080F83C209DF8AC1001EB410000EB16
:101D80000110A84901EB0010C179A74880F8BC11E7
:101D900000BF00BF04F048BB9DF8AC1001EB410050
:101DA000C0EBC110994901EBC000C1789DF8AC00AF
:101DB00000EB4002C2EBC010944A02EBC0008078F6
:101DC00041EA002127919DF8AC1001EB4100C0EBE6
:101DD000C110114601EBC001BDF89C00401C095C1C
:101DE0009DF8AC0000EB4002C2EBC010874A02EB4A
:101DF000C002BDF89C00105C41EA0020C217CDE98A
:101E00002C029DF8AC1001EB4100C0EBC1107F49E2
:101E100001EBC0000990BDF89C10F7F73FFD0022D0
:101E2000CDE92E022DA819C82C99594060400143D4
:101E30006FD19DF8AC1001EB4100C0EBC1107349AC
:101E400001EBC00041782691002137911CE09DF8FC
:101E5000AC1001EB410000EB0110724901EB0011E5
:101E60003031BDF8DC0001EB001041789DF898009E
:101E7000814204D1BDF8DC00C1B2269112E0BDF868
:101E8000DC00401C81B237919DF8AC1001EB4100A1
:101E900000EB0110634901EB0010C179BDF8DC00D3
:101EA0008142D4DC00BF9DF8AC1001EB410000EB97
:101EB00001105C4901EB001030309DF8981000EBE8
:101EC0000110801C0990007820F080008030099972
:101ED00008709DF8AC1001EB4100C0EBC1104B49FC
:101EE00001EBC000007924900020494A9DF8AC1015
:101EF00002EB01129DF898105054BDF89000F228A2
:101F00007ED007DC05287CD006280AD0F12879D1BC
:101F1000FEE3FEE3F32876D0F42875D0F628F6D158
:101F2000F8E30621109100213491F4E3BDF840005C
:101F3000401C81B210919DF8AC1001EB4100C0EB48
:101F4000C110324901EBC001BDF84000095C249189
:101F5000BDF84000401C81B21091BDF89000F128FE
:101F600004D0F22871D0F32870D1FDE39DF8AC10B5
:101F700001EB4100C0EBC110244901EBC001BDF8E9
:101F80004000095C2791BDF84000401C81B21091CF
:101F90009DF8AC1001EB410000EB0110214901EB71
:101FA000001130319DF89820BDF8D000104401EBAD
:101FB0000010407A00F0010038B39DF8AC1040F2F8
:101FC000231011FB00F0164901EBC00118319DF8F8
:101FD0009820BDF8D000104400EBC00001EB0010C9
:101FE00090F88E0000F0010078B99DF8AC1040F236
:101FF000231011FB00F00A4901EBC001183115E074
:10200000FEE3FEE3FEE3FEE3FEE359E0A8780020F2
:10201000483F0020000000000000244085340020DC
:10202000D445002014410020BC3200209DF89820A7
:10203000BDF8D000104400EBC00001EB001090F898
:102040008100E8B3002137912EE0B2E3B0E39DF8C0
:10205000AC1040F2231011FB00F0FE4901EBC0016F
:1020600018319DF89820BDF8D000104400EBC00056
:1020700001EB001000F18201BDF8DC000A5C9DF864
:10208000AC0000EB400101EB0010F34901EB001044
:102090000E30BDF8DC10405C824200D008E0BDF894
:1020A000DC00401C81B23791BDF8DC000428CEDB97
:1020B00000BFBDF8DC00042854D1042137912DE085
:1020C00050E09DF8AC1040F2231011FB00F0E14904
:1020D00001EBC00118319DF89820BDF8D0001044E4
:1020E00000EBC00001EB001000F18201BDF8DC0044
:1020F0000A5C9DF8AC0000EB400101EB0010D649F2
:1021000001EB00100E30BDF8DC10405C824200D0C4
:1021100008E0BDF8DC00401C81B23791BDF8DC005E
:102120000A28CEDB00BFBDF8DC000A281AD09DF8D3
:10213000AC1040F2231011FB00F0C64901EBC000C7
:1021400018309DF89820BDF8D010114401EBC10162
:1021500000EB01108E300990007820F00100401C47
:1021600009990870BDF89C000F287DD19DF8AC102E
:1021700001EB410000EB0110B74901EB00113031D8
:102180009DF89820BDF8D000104401EB0010801C91
:102190000990007820F00400001D099908700020C3
:1021A00037902AE09DF8AC1001EB4100C0EBC11064
:1021B000AA4901EBC001BDF84020BDF8DC00104485
:1021C0000A5C9DF8AC0040F2231110FB01F0A1491C
:1021D00001EBC00118319DF89830BDF8D0001844CB
:1021E00000EBC00001EB00113F31BDF8DC000A54E8
:1021F000BDF8DC00401C81B23791BDF8DC000A2834
:10220000D0DBBDF840000A3081B210910021379137
:102210002CE09DF8AC1001EB4100C0EBC1108F49E0
:1022200001EBC001BDF84020BDF8DC0010440A5CA1
:102230009DF8AC0040F2231110FB01F0854901EB41
:10224000C00118319DF89830BDF8D000184400EB5B
:10225000C00001EB00115831BDF8DC000A54BDF894
:10226000DC00401C81B200E040E23791BDF8DC00A8
:102270000228CEDBBDF84000801C81B210919DF891
:10228000AC1001EB4100C0EBC110744901EBC0017F
:10229000BDF84000085C01049DF8AC0000EB400272
:1022A000C2EBC0106D4A02EBC002BDF84000401CFA
:1022B000105C41EA00219DF8AC0000EB4002C2EB4B
:1022C000C010664A02EBC002BDF84000801C105CE2
:1022D00001439DF8AC0040F2231210FB02F05D4A6E
:1022E00002EBC00218329DF89830BDF8D0001844B7
:1022F00000EBC00002EB0010C166BDF84000C01C3E
:1023000081B21091564890F8A008E0BB00213791A7
:102310001DE09DF8AC1040F2231011FB00F04D4978
:1023200001EBC00118319DF89820BDF8D000104491
:1023300000EBC00001EB00103F30BDF8DC10405C4A
:1023400000B108E0BDF8DC00401C81B23791BDF857
:10235000DC000A28DDDB00BFBDF8DC000A2818D14C
:1023600040229DF8AC0040F2231110FB01F03949E6
:1023700001EBC00118319DF89830BDF8D000184429
:1023800000EBC00000E059E001EB001080F877207E
:102390004DE19DF8AC1040F2231011FB00F02D49E7
:1023A00001EBC00118319DF89820BDF8D000104411
:1023B00000EBC00001EB001090F87700F0BB0021AB
:1023C00028910EE10021359129E09DF8AC1040F2F2
:1023D000231011FB00F01F4901EBC00118319DF8DB
:1023E0009820BDF8D000104400EBC00001EB0011B4
:1023F0003F31BDF8D400001D095C9DF8A00000EB42
:102400004002184800EB4202BDF8D400105C814243
:1024100000D008E0BDF8D400401C81B23591BDF871
:10242000D4000628D1DB00BFBDF8D40006287DD13A
:1024300003229DF8AC0040F2231100E0F7E010FB0E
:1024400001F0044901EBC00118319DF89830BDF846
:10245000D00009E0D445002014410020A8780020D5
:10246000BC32002048350020184400EBC00001EBCE
:10247000001080F877209DF8AC1001EB410000EBD4
:102480000110FE4901EB001130319DF89820BDF894
:10249000D000104401EB0010801C0990007820F05F
:1024A000040209980270002037901CE020229DF859
:1024B000AC0040F2231110FB01F0F14901EBC00127
:1024C00018319DF89830BDF8D000184400EBC000DA
:1024D00001EB00114931BDF8DC000A54BDF8DC0005
:1024E000401C81B23791BDF8DC000F28DEDB0021F3
:1024F00037911EE020229DF8AC0040F2231110FB22
:1025000001F0DF4901EBC00118319DF89830BDF8AA
:10251000D000184400EBC00001EB00115B31BDF8A6
:10252000DC000A54BDF8DC00401C00E054E081B23D
:102530003791BDF8DC000A28DCDB00229DF8AC00F6
:1025400040F2231110FB01F0CD4901EBC00118311D
:102550009DF89830BDF8D000184400EBC00001EBA6
:10256000001080F87020002137911CE000229DF8B7
:10257000AC0040F2231110FB01F0C14901EBC00196
:1025800018319DF89830BDF8D000184400EBC00019
:1025900001EB00117131BDF8DC000A54BDF8DC001C
:1025A000401C81B23791BDF8DC000528DEDB9DF8C8
:1025B000AC1040F2231011FB00F0B14901EBC00157
:1025C00018319DF89820BDF8D000104400EBC000F1
:1025D00001EB0010C06E0CE09DF8A000401CC1B2E1
:1025E0002891A848B0F88A129DF8A00081423FF7D0
:1025F000E9AE00BFA348B0F88A129DF8A00081425E
:1026000015D140229DF8AC0040F2231110FB01F0DF
:102610009B4901EBC00118319DF89830BDF8D000FE
:10262000184400EBC00001EB001080F877209DF803
:10263000AC1040F2231011FB00F0914901EBC001F6
:1026400018319DF89820BDF8D000104400EBC00070
:1026500001EB001090F87700032804D0112818D05F
:10266000402842D12BE0F2229DF8AC0040F2231129
:1026700010FB01F0824901EBC00118319DF8983040
:10268000BDF8D000184400EBC00001EB001042710F
:102690002BE0F3229DF8AC0040F2231110FB01F077
:1026A000774901EBC00118319DF89830BDF8D00092
:1026B000184400EBC00001EB0010427115E0F2225B
:1026C0009DF8AC0040F2231110FB01F06C4901EBC6
:1026D000C00118319DF89830BDF8D000184400EBC7
:1026E000C00001EB0010427100BF61E09DF8AC102A
:1026F00001EB410000EB0110604901EB00103030AC
:102700009DF89820BDF8D010114400EB011003E0B3
:10271000CDE0EEE3EEE3BAE0801C0990007820F013
:102720000402099802709DF8AC1040F2231011FBCE
:1027300000F0534901EBC00018309DF89820BDF817
:10274000D010114401EBC10100EB011090F88E0094
:1027500000F0010060B300229DF8AC0040F22311AC
:1027600010FB01F0464900E06EE001EBC0011831BA
:102770009DF89830BDF8D000184400EBC00001EB84
:102780000010A0F88C2005229DF8AC0040F2231127
:1027900010FB01F03A4901EBC00118319DF8983067
:1027A000BDF8D000184400EBC00001EB00104271EE
:1027B00060E09DF8AC0040F2231110FB01F03049BD
:1027C00001EBC00118319DF89820BDF8D0001044ED
:1027D00000EBC00001EB001090F8770040281CD1FE
:1027E00000229DF8AC0040F2231110FB01F02449B7
:1027F00001EBC00118319DF89830BDF8D00004E01D
:10280000EFE3EFE3EFE3EFE3EFE3184400EBC000A7
:1028100001EB001080F8772000BF00BFF1229DF887
:10282000AC0040F2231110FB01F0154901EBC0018F
:1028300018319DF89830BDF8D000184400EBC00066
:1028400001EB0010427115E0F1229DF8AC0040F25E
:10285000231110FB01F00A4901EBC00118319DF86A
:102860009830BDF8D000184400EBC00001EB001018
:10287000427100BF00BFBDF8D00005E01441002048
:10288000D4450020BC320020401C81B234919DF818
:10289000AC0000EB4001C1EBC010FC4901EBC000F3
:1028A0004179BDF8D00081423FF740AB9BE39DF8F2
:1028B000AC0040F2231110FB01F0F54901EBC00020
:1028C00018309DF8981001EBC10100EB0110007861
:1028D00020BB01229DF8AC0040F2231110FB01F057
:1028E000EB4901EBC00118319DF8980000EBC000E6
:1028F00001EB00100270F4229DF8AC0040F22311AD
:1029000010FB01F0E24901EBC00118319DF898007D
:1029100000EBC00001EB00104271BEE09DF8AC007E
:1029200000EB400101EB0010DA4901EB0010303000
:102930009DF8981000EB0110407A00F00100E8B318
:102940009DF8AC0040F2231110FB01F0D04901EBDF
:10295000C00018309DF8981001EBC10100EB011088
:1029600090F88E0000F0010040BB9DF8AC0040F2F2
:10297000231110FB01F0C64901EBC00018309DF88F
:10298000981001EBC10100EB011090F88100A8B193
:10299000002037902BE09DF8AC0040F2231110FB93
:1029A00001F0BB4901EBC00118319DF8980000EB24
:1029B000C00001EB001000F1820100E06DE0BDF805
:1029C000DC000A5C9DF8AC0000EB400101EB00105C
:1029D000B04901EB00100E30BDF8DC10405C8242C3
:1029E00000D008E0BDF8DC00401C81B23791BDF892
:1029F000DC000428CFDB00BFBDF8DC0004284CD18C
:102A0000379029E09DF8AC0040F2231110FB01F053
:102A10009F4901EBC00118319DF8980000EBC00000
:102A200001EB001000F18201BDF8DC000A5C9DF8AA
:102A3000AC0000EB400101EB0010964901EB0010E7
:102A40000E30BDF8DC10405C824200D008E0BDF8DA
:102A5000DC00401C81B23791BDF8DC000A28D1DBD4
:102A600000BFBDF8DC000A2817D09DF8AC0040F28A
:102A7000231110FB01F0864901EBC00018309DF8CE
:102A8000981001EBC10100EB01108E300990007825
:102A900020F00100401C09990870BDF89C00112825
:102AA00071D19DF8AC0000EB400101EB00107949B9
:102AB00001EB001030309DF8981000EB0110801CE5
:102AC0000990007820F00400001D0999087000208A
:102AD000379025E09DF8AC0000EB4001C1EBC01041
:102AE0006A4901EBC001BDF8DC00401D0A5C9DF89D
:102AF000AC0040F2231110FB01F0654901EBC0016D
:102B000018319DF8980000EBC00001EB00113F3137
:102B1000BDF8DC000A54BDF8DC00401C81B23791DE
:102B2000BDF8DC000A28D5DB0020379025E09DF8B1
:102B3000AC0000EB4001C1EBC010544901EBC001F7
:102B4000BDF8DC000F300A5C9DF8AC0040F22311A8
:102B500010FB01F04E4901EBC00118319DF89800BF
:102B600000EBC00001EB00115831BDF8DC000A5445
:102B7000BDF8DC00401C81B23791BDF8DC000228B2
:102B8000D5DBC8E2FFE7BDF89C0014287DD19DF895
:102B9000AC0000EB400101EB00103E4901EB0010DE
:102BA00030309DF8981000EB0110801C09900078DF
:102BB00020F00400001D099908700020379025E0DE
:102BC0009DF8AC0000EB4001C1EBC0102F4901EBB8
:102BD000C001BDF8DC00401D0A5C9DF8AC0040F26D
:102BE000231110FB01F02A4901EBC00118319DF8B7
:102BF000980000EBC00001EB00113F31BDF8DC0094
:102C00000A54BDF8DC00401C81B23791BDF8DC00ED
:102C10000A28D5DB0020379025E09DF8AC0000EBBA
:102C20004001C1EBC010194901EBC001BDF8DC0047
:102C30000F300A5C9DF8AC0040F2231110FB01F04C
:102C4000134901EBC00118319DF8980000EBC0005A
:102C500001EB00115831BDF8DC000A54BDF8DC006E
:102C6000401C81B23791BDF8DC000228D5DB9DF80D
:102C7000AC0000EB4001C1EBC010044901EBC00007
:102C8000407C01049DF8AC0006E0E9E1A878002052
:102C9000D44500201441002000EB4002C2EBC010DC
:102CA000FE4A02EBC000807C41EA00219DF8AC00A6
:102CB00000EB4002C2EBC010F84A02EBC000C07C3F
:102CC00001439DF8AC0040F2231210FB02F0F44ADD
:102CD00002EBC00018309DF8982002EBC20200EB16
:102CE0000210C166EF4890F8A008C8BB00203790DA
:102CF0001AE09DF8AC0040F2231110FB01F0E84906
:102D000001EBC00118319DF8980000EBC00001EB09
:102D100000103F30BDF8DC10405C00B108E0BDF8A9
:102D2000DC00401C81B23791BDF8DC000A28E0DBF2
:102D300000BFBDF8DC000A2813D140229DF8AC008A
:102D400040F2231110FB01F0D54901EBC00018300F
:102D50009DF8981001EBC10100EB011080F877207D
:102D600026E19DF8AC0040F2231110FB01F0CC49A4
:102D700001EBC00018309DF8981001EBC10100EB89
:102D8000011090F87700E8BB00202890EDE00020CB
:102D9000359026E09DF8AC0040F2231110FB01F0C5
:102DA000BF4901EBC00118319DF8980000EBC0004D
:102DB00001EB00113F31BDF8D400001D095C9DF806
:102DC000A00000EB4002B84800EB4202BDF8D4007E
:102DD000105C814200D008E0BDF8D400401C81B2F4
:102DE0003591BDF8D4000628D4DB00BFBDF8D4006F
:102DF00006287DD103229DF8AC0040F2231110FB80
:102E000001F000E0D4E0A64901EBC00118319DF8C3
:102E1000980000EBC00001EB001080F877209DF8CF
:102E2000AC0000EB400101EB0010A04901EB0011E8
:102E300030319DF8980001EB0010801C099000785B
:102E400020F00402099802700020379019E0202237
:102E50009DF8AC0040F2231110FB01F0904901EB0A
:102E6000C00118319DF8980000EBC00001EB001183
:102E70004931BDF8DC000A54BDF8DC00401C81B2C9
:102E80003791BDF8DC000F28E1DB0020379019E016
:102E900020229DF8AC0040F2231110FB01F0804984
:102EA00001EBC00118319DF8980000EBC00001EB68
:102EB00000115B31BDF8DC000A54BDF8DC00401C99
:102EC00081B23791BDF8DC000A28E1DB00229DF8D1
:102ED000AC0040F2231110FB01F0714901EBC0017D
:102EE00018319DF8980000EBC00001EB001002E0E3
:102EF00036E0AAE25FE180F870200021379119E006
:102F000000229DF8AC0040F2231110FB01F064494F
:102F100001EBC00118319DF8980000EBC00001EBF7
:102F200000117131BDF8DC000A54BDF8DC00401C12
:102F300081B23791BDF8DC000528E1DB9DF8AC10CB
:102F400040F2231011FB00F0554901EBC00018308E
:102F50009DF8981001EBC10100EB0110C06E0CE070
:102F60009DF8A000401CC1B228914E48B0F88A02DA
:102F70009DF8A01088423FF70AAF00BF4948B0F85B
:102F80008A029DF8A010884212D140229DF8AC0020
:102F900040F2231110FB01F0414901EBC000183051
:102FA0009DF8981001EBC10100EB011080F877202B
:102FB0009DF8AC1040F2231011FB00F0384901EBF2
:102FC000C00018309DF8981001EBC10100EB011012
:102FD00090F87700032809D011281AD040283ED154
:102FE0002AE099E0C0E12FE2D2E009E1F2229DF867
:102FF000AC0040F2231110FB01F0294901EBC000A5
:1030000018309DF8981001EBC10100EB01104271DE
:1030100025E0F3229DF8AC0040F2231110FB01F0F3
:103020001F4901EBC00118319DF8980000EBC0006A
:1030300001EB0010427112E0F2229DF8AC0040F268
:10304000231110FB01F0164901EBC00018309DF868
:10305000981001EBC10100EB0110427100BF5AE072
:103060009DF8AC1001EB410000EB01100F4901EBA2
:10307000001030309DF8981000EB0110801C099072
:10308000007820F00402099802709DF8AC1040F21C
:10309000231011FB00F002490AE00000A87800208C
:1030A000D4450020BC3200204835002014410020C7
:1030B00001EBC00018309DF8981001EBC10100EB46
:1030C000011090F88E0000F0010020B300229DF85E
:1030D000AC0040F2231110FB01F0FE4901EBC001EE
:1030E00018319DF8980000EBC00001EB0010A0F82B
:1030F0008C2005229DF8AC0040F2231110FB01F05A
:10310000F44901EBC00018309DF8981001EBC101A3
:1031100000EB0110427197E19DF8AC1040F22310D2
:1031200011FB00F0EB4901EBC00018309DF898103E
:1031300001EBC10100EB011090F87700402813D19A
:1031400000229DF8AC0040F2231110FB01F0E14990
:1031500001EBC00018309DF8981001EBC10100EBA5
:10316000011080F8772000BF00BFF1229DF8AC006D
:1031700040F2231110FB01F0D64901EBC0001830DA
:103180009DF8981001EBC10100EB011042715BE169
:10319000F1229DF8AC0040F2231110FB01F0CD4963
:1031A00001EBC00018309DF8981001EBC10100EB55
:1031B0000110427148E103229DF8AC0040F2231156
:1031C00010FB01F0C34901EBC00118319DF89800D4
:1031D00000EBC00001EB00100270F1229DF8AC0082
:1031E00040F2231110FB01F0BA4901EBC001183184
:1031F0009DF8980000EBC00001EB0010427123E144
:1032000002229DF8AC0040F2231110FB01F0B149FD
:1032100001EBC00118319DF8980000EBC00001EBF4
:1032200000100270F6229DF8AC0040F2231110FB52
:1032300001F0A84901EBC00118319DF8980000EB9E
:10324000C00001EB0010427101229DF8AC0040F279
:10325000231110FB01F09F4901EBC00118319DF8CB
:10326000980000EBC00001EB001080F881200021E5
:10327000379126E09DF8AC1001EB4100C0EBC11086
:10328000954901EBC001BDF8DC00401D0A5C9DF8CA
:10329000AC0040F2231110FB01F08E4901EBC0019C
:1032A00018319DF8980000EBC00001EB001000F110
:1032B0008201BDF8DC000A54BDF8DC00401C81B27C
:1032C0003791BDF8DC000A28D4DBBDF89C00152836
:1032D00049D19DF8AC1001EB4100C0EBC1107E4913
:1032E00001EBC000C27B9DF8AC0040F2231110FB43
:1032F00001F0784901EBC00118319DF8980000EB0E
:10330000C00001EB001080F878200021379126E002
:103310009DF8AC1001EB4100C0EBC1106E4901EB10
:10332000C001BDF8DC0010300A5C9DF8AC0040F232
:10333000231110FB01F0674901EBC00118319DF822
:10334000980000EBC00001EB001000F17A01BDF81D
:10335000DC000A54BDF8DC00401C81B23791BDF896
:10336000DC000428D4DB6FE09DF8AC1001EB4100D9
:10337000C0EBC110584901EBC00081799DF8AC0049
:1033800000EB4002C2EBC010534A02EBC000407990
:1033900041EA00229DF8AC0040F2231110FB01F03D
:1033A0004C4901EBC00118319DF8980000EBC000BA
:1033B00001EB0010A0F88C209DF8AC1040F2231017
:1033C00011FB00F0434901EBC00118319DF8980052
:1033D00000EBC00001EB0010B0F88C109DF8AC00C1
:1033E00000EB400202EB00103C4A02EB0010408B65
:1033F000814228DBF1229DF8AC0040F2231110FB42
:1034000001F0344901EBC00118319DF8980000EB40
:10341000C00001EB001042719DF8AC1040F2231087
:1034200011FB00F02B4901EBC00118319DF8980009
:1034300000EBC00001EB00108E300990007820F006
:1034400001020998027000BF00BF02F0EDBF9DF8B5
:10345000AC1001EB4100C0EBC1101F4901EBC000F3
:1034600001792691002134911CE09DF8AC1001EB0C
:10347000410000EB0110194901EB00113031BDF89A
:10348000D00001EB001041789DF89800814204D1F2
:10349000BDF8D000C1B2269112E0BDF8D000401CAA
:1034A00081B234919DF8AC1001EB410000EB0110AA
:1034B0000A4901EB0010C179BDF8D0008142D4DC8B
:1034C00000BF9DF8AC1001EB4100C0EBC1100249F8
:1034D00006E00000D4450020A87800201441002018
:1034E00001EBC000C1782491BDF89000172834D2B8
:1034F000DFE800F0330C0F331215181B1E33333383
:1035000033333321242733332A2D300007212791E9
:1035100023E00721279120E0062027901DE00621C7
:1035200027911AE00621279117E01221279114E034
:103530000721279111E0092127910EE0062127910B
:103540000BE00621279108E00B21279105E00B21D4
:10355000279102E02A21279100BF00BFBDF89C00FF
:10356000001FC1B209919DF8AC1001EB4100C0EB06
:10357000C110FE4901EBC000C01C08900999F5F785
:10358000A9FF35909DF8AC1001EB4100C0EBC110D4
:10359000F64901EBC001BDF89C00401E095CBDF876
:1035A000D40081427ED19DF8AC1001EB4100C0EB0C
:1035B000C110EE4901EBC0004078002872DD9DF893
:1035C000AC1001EB4100C0EBC110E84901EBC001B8
:1035D000BDF89C000A5C9DF8AC0040F2231110FB82
:1035E00001F0E34901EBC00118319DF8980000EBB0
:1035F000C00001EB001080F83C200021DD4A9DF85E
:10360000AC0002EB00129DF898001154DA4890F8D3
:103610002000012815D19DF8AC1001EB410000EB12
:103620000110D64901EB001030309DF8981000EBE6
:103630000110801C0990007820F0800080300999EA
:103640000870BDF8900007287ED00ADC07287CD2DD
:10365000DFE810F07B00D9042F057B00C60491043D
:10366000830910380728F2D2DFE810F0E709D409FF
:103670006F006F0007000800570500BFBDF89000FD
:1036800014287DD19DF8AC1001EB4100C0EBC110B6
:10369000B64901EBC000407901069DF8AC0000EB93
:1036A000400200E0FEE3C2EBC010B04A02EBC000F3
:1036B000807941EA00419DF8AC2002EB4200C0EB6A
:1036C000C210AA4A02EBC000C07941EA00219DF86D
:1036D000AC2002EB4200C0EBC210A44A02EBC000D7
:1036E000007A01439DF8AC0040F2231210FB02F077
:1036F0009F4A02EBC00218329DF8980000EBC00010
:1037000002EB0010C0F81A109DF8AC1040F2231024
:1037100011FB00F0964901EBC00118319DF89800AB
:1037200000EBC00001EB0010D0F81A100846099118
:10373000002109F09BFDCDE92C019DF8AC1001EBB7
:10374000410000EB011001E0FDE3FDE38B4901EBDB
:103750000010007F00F003019DF8AC2002EB420056
:1037600000EB0210854A02EB0010007FC0F301104D
:1037700001449DF8AC0000EB400202EB001000E0B9
:1037800062E07E4A02EB0010007FC0F38100091A5C
:1037900008460591F4F72BFFCDE906019DED061BC8
:1037A0009FED770B17F0A0F88DED080B9DED080B42
:1037B00051EC100BF4F78DFFCDE92E019DF8AC1004
:1037C00040F2231011FB00F0694901EBC0011831F0
:1037D0009DF8980000EBC00001EB0010416B08461B
:1037E0000791002109F042FDDDE92C32A0FB0345E1
:1037F00001FB035100FB021502220023DDE92E012B
:10380000F4F7E0FC20186941CDE90801DDE92E2339
:10381000F4F7D8FCCDE92C01DDE92C010AF0DCFA43
:1038200001469DF8AC2040F2231012FB00F0504AF4
:1038300002EBC00018309DF8982002EBC20200EBAA
:103840000210C0F81E1043E0BDF8900015283FD1CB
:103850009DF8AC1001EB4100C0EBC110434901EBF6
:10386000C000407901069DF8AC0000EB4002C2EBBD
:10387000C0103E4A02EBC000807941EA00419DF849
:10388000AC0000EB4002C2EBC010384A02EBC000B3
:10389000C07941EA00219DF8AC2002EB4200C0EB68
:1038A000C210324A02EBC000007A01439DF8AC20FE
:1038B00040F2231012FB00F02D4A02EBC00018303A
:1038C0009DF8982002EBC20200EB0210C0F81E1017
:1038D0009DF8AC1001EB4100C0EBC110234901EB96
:1038E000C000417A284880F8131E9DF8AC1001EB07
:1038F000410000EB0110214901EB001130319DF82E
:10390000980001EB0010801C09901F4890F8130EDE
:10391000C2090998007862F30000099908701A48F2
:1039200090F8130E00F00300012806D0164890F816
:10393000130E00F0030003283CD19DF8AC1001EBFE
:10394000410000EB01100D4901EB001030309DF8F3
:10395000981000EB0110801C0990007820F0020004
:10396000801C099908709DF8AC100FE0A878002021
:10397000D4450020483F0020BC1200201441002004
:103980000000000000002440BC22002001EB4100A8
:1039900000EB0110FE4901EB001030309DF898104B
:1039A00000EB0110801C0990007820F0200209989B
:1039B000027014E09DF8AC1001EB410000EB011027
:1039C000F34901EB001030309DF8981000EB011026
:1039D000801C0990007820F00202099802709DF87E
:1039E000AC1001EB410000EB0110E94901EB0011C3
:1039F00030319DF8980001EB00108078C0F3400250
:103A00009DF8AC0040F2231110FB01F0E14901EBFD
:103A1000C00018309DF8981001EBC10100EB0110B7
:103A2000007EC0F34000824266D09DF8AC1040F2A8
:103A3000231011FB00F0D74901EBC00018309DF8AE
:103A4000981001EBC10100EB0110183009909DF8AE
:103A5000AC1001EB410000EB0110CD4901EB00106F
:103A600030309DF8981000EB0110807842080998DA
:103A7000007862F34100099908709DF8AC1001EBE1
:103A8000410000EB0110C24901EB001030309DF8FD
:103A9000981000EB01108078C0F3400038BB9DF80F
:103AA000AC1001EB410000EB0110B94901EB001033
:103AB00030309DF8981000EB0110801C09900078C0
:103AC00020F020020998027001229DF8AC1040F20B
:103AD000231011FB00F0AF4901EBC00018309DF836
:103AE000981001EBC10100EB011080F83E209DF819
:103AF000AC100220F6F72EFA9DF8AC1001EB410055
:103B000000EB0110A24901EB001130319DF8980043
:103B100001EB0010807800F001029DF8AC0040F24B
:103B2000231110FB01F09B4901EBC00018309DF8F8
:103B3000981001EBC10100EB0110007E00F00100C4
:103B400082425FD09DF8AC1040F2231011FB00F0D0
:103B5000904901EBC00018309DF8981001EBC101AD
:103B600000EB0110183009909DF8AC1001EB4100FA
:103B700000EB0110864901EB001030309DF89810E1
:103B800000EB0110807809990A7860F300020A704E
:103B90009DF8AC1001EB410000EB01107C4901EBFA
:103BA000001030309DF8981000EB0110807800F084
:103BB000010040BB9DF8AC1001EB410000EB01108F
:103BC000734901EB001030309DF8981000EB0110A4
:103BD000801C0990007820F02002099802700022D1
:103BE0009DF8AC1040F2231011FB00F0694901EB85
:103BF000C00018309DF8981001EBC10100EB0110D6
:103C000080F83D2013E19DF8AC1040F2231011FB29
:103C100000F0604901EBC00018309DF8981001EBEE
:103C2000C10100EB011090F83E0098B901229DF807
:103C3000AC1040F2231011FB00F0564901EBC0011B
:103C400018319DF8980000EBC00001EB001080F8DF
:103C50003D2027E000229DF8AC0040F2231110FB2C
:103C600001F04C4901EBC00118319DF8980000EBC0
:103C7000C00001EB001080F83D209DF8AC1001EB76
:103C8000410000EB0110424901EB001130319DF879
:103C9000980001EB0010801C0990007820F00102D0
:103CA000099802703C4890F8A008E8BB3B4890F89F
:103CB0002100012838D13948D0F818023749498CF9
:103CC000884231D29DF8AC1040F2231011FB00F075
:103CD000304901EBC00018309DF8981001EBC1018C
:103CE00000EB011090F83D0001281DD19DF8AC10AB
:103CF00040F2231011FB00F0264901EBC000183000
:103D00009DF8981001EBC10100EB011090F87E00C6
:103D100050B99DF8AC1001EB410000EB01101C49BB
:103D200001EB0011303100E081E09DF8980001EBDB
:103D3000001001789DF8AC0040F2231210FB02F055
:103D4000144A02EBC000417005229DF8AC0040F21D
:103D5000231110FB01F00F4901EBC00118319DF850
:103D6000980000EBC00001EB0010427100229DF8AA
:103D7000AC1001EB410000EB0110054901EB001113
:103D800030319DF8980001EB0010426008E000001F
:103D900014410020D4450020BC320020BC12002079
:103DA0009DF8AC100220F6F7D5F80021379119E004
:103DB00000229DF8AC0040F2231110FB01F0FA49FB
:103DC00001EBC00118319DF8980000EBC00001EB39
:103DD00000113F31BDF8DC000A54BDF8DC00401C86
:103DE00081B23791BDF8DC001428E1DB0021379166
:103DF00019E000229DF8AC1040F2231011FB00F0F6
:103E0000E94901EBC00118319DF8980000EBC000B2
:103E100001EB00115B31BDF8DC000A54BDF8DC0099
:103E2000401C81B23791BDF8DC000A28E1DB9DF827
:103E3000AC1040F2231011FB00F0DB4901EBC00095
:103E400018309DF8981001EBC10100EB01100078CB
:103E5000012812DC02229DF8AC0040F2231110FB75
:103E600001F0D14901EBC00018309DF8981001EB2A
:103E7000C10100EB011002707CE09DF8AC1040F233
:103E8000231011FB00F0C84901EBC00018309DF869
:103E9000981001EBC10100EB01100078022831DC21
:103EA000002100E0F4E39DF8AC2040F2231012FB67
:103EB00000F0BD4A02EBC000017103229DF8AC1076
:103EC00040F2231011FB00F0B74901EBC00118319B
:103ED0009DF8980000EBC00001EB00100270072273
:103EE0009DF8AC0040F2231110FB01F0AE4901EB4C
:103EF000C00018309DF8981001EBC10100EB0110D3
:103F0000427137E09DF8AC1040F2231011FB00F035
:103F1000A54901EBC00118319DF8980000EBC000E5
:103F200001EB001001789DF8AC2040F2231012FB49
:103F300000F09D4A02EBC000407981421AD19B48B3
:103F400090F8130E01E0C0E1FEE3C0F3401088B129
:103F500016229DF8AC0040F2231110FB01F09249AB
:103F600001EBC00018309DF8981001EBC10100EB87
:103F700001104271E8E314229DF8AC1040F22310C6
:103F800011FB00F0884901EBC00118319DF8980041
:103F900000EBC00001EB0010427101219DF8AC2044
:103FA00040F2231012FB00F07F4A02EBC0000171C7
:103FB0009DF8AC1001EB410000EB0110A2F59861F7
:103FC00001EB001130319DF8980001EB0010801CCE
:103FD0000990007820F02000203009990870B3E3A0
:103FE00014229DF8AC1040F2231011FB00F06E4932
:103FF00001EBC00018309DF8981001EBC10100EBF7
:1040000001104271A0E39DF8AC1040F2231011FBA7
:1040100000F0654901EBC0001830BDF8D01001EB8D
:10402000C10100EB01108079012824D100229DF804
:10403000AC0040F2231110FB01F05B4901EBC00121
:104040001831BDF8D00000EBC00001EB0010827108
:1040500014229DF8AC1040F2231011FB00F05249DD
:1040600001EBC00018309DF8981001EBC10100EB86
:10407000011042711CE000219DF8AC2040F2231099
:1040800012FB00F0484A02EBC000017105229DF8C6
:10409000AC1040F2231011FB00F0434901EBC000CB
:1040A00018309DF8981001EBC10100EB011042712E
:1040B0004AE301219DF8AC2040F2231012FB00F0EE
:1040C000394A02EBC000017114229DF8AC0040F2A5
:1040D000231110FB01F0344901EBC00118319DF8A8
:1040E000980000EBC00001EB001042719DF8AC108D
:1040F00001EB410000EB01102D4901EB00113031C3
:104100009DF8980001EB0010801C0990007820F0C9
:104110000400001D0999087016E300202C902D90D2
:10412000002137911FE0DDE92C10000240EA116206
:104130000902CDE92C129DF8AC1001EB4100C0EB57
:10414000C1101C4901EBC001BDF8DC00401D085C3A
:10415000DDE92C3440EA0302CDE92C24BDF8DC0073
:10416000401C81B23791BDF8DC000328DBDBDDE9C0
:104170002C0109F031FE01469DF8AC2040F22310DD
:1041800012FB00F0084A02EBC00218329DF89800BA
:1041900000EBC00002EB0010C0F81E1000222C92B1
:1041A0002D920021379127E0D4450020BC22002029
:1041B00014410020A8780020DDE92C10000240EA1C
:1041C00011620902CDE92C129DF8AC1001EB4100FF
:1041D000C0EBC110FE4901EBC001BDF8DC000830A6
:1041E000085CDDE92C3440EA0302CDE92C24BDF85B
:1041F000DC00401C81B23791BDF8DC000328DBDB1A
:10420000DDE92C0109F0E8FD01469DF8AC0040F223
:10421000231210FB02F0EF4A02EBC00218329DF8A5
:10422000980000EBC00002EB0010C0F81A1000224A
:104230002C922D92002137911EE0DDE92C10000216
:1042400040EA11620902CDE92C129DF8AC1001EB95
:104250004100C0EBC110DE4901EBC001BDF8DC003C
:104260001330085CDDE92C341843CDE92C04BDF88B
:10427000DC00401C80B23790BDF8DC000328DCDB9A
:104280009DF8AC202C9940F2231012FB00F0D14A8B
:1042900002EBC00218329DF8980000EBC00002EB60
:1042A0000010416307229DF8AC1040F2231011FB6F
:1042B00000F0C84901EBC00018309DF8981001EBE0
:1042C000C10100EB01104271CAE300202C902D9037
:1042D000002137911FE0DDE92C10000240EA116255
:1042E0000902CDE92C129DF8AC1001EB4100C0EBA6
:1042F000C110B74901EBC001BDF8DC00401D085CEE
:10430000DDE92C3440EA0302CDE92C24BDF8DC00C1
:10431000401C81B23791BDF8DC000428DBDBDDE90D
:104320002C0109F059FD9DF8AC2040F2231312FB3B
:1043300003F2A84B03EBC20318339DF8982002EB5D
:10434000C20203EB021222329060D16000212C9154
:104350002D91002037901FE0DDE92C10000240EA8B
:1043600011620902CDE92C129DF8AC1001EB41005D
:10437000C0EBC110964901EBC001BDF8DC0009306B
:10438000085CDDE92C3440EA0302CDE92C24BDF8B9
:10439000DC00401C81B23791BDF8DC000428DBDB77
:1043A000DDE92C0109F018FD9DF8AC2040F2231343
:1043B00012FB03F2874B03EBC20318339DF89820DE
:1043C00002EBC20203EB021242F8220F51609DF889
:1043D000AC1040F2231011FB00F07E4901EBC0004D
:1043E00018309DF8981001EBC10100EB0110007826
:1043F0009DF8AC1040F2231211FB02F1754A02EB5A
:10440000C101497988426ED1734890F8130EC0F308
:10441000401090B117229DF8AC1040F2231011FB10
:1044200000F06C4901EBC00018309DF8981001EBCA
:10443000C10100EB0110427111E014229DF8AC1093
:1044400040F2231011FB00F0624901EBC00118316A
:104450009DF8980000EBC00001EB001042715F482E
:1044600090F8A008F0BB00229DF8AC1040F2231099
:1044700011FB00F0574901EBC00018309DF898106F
:1044800001EBC10100EB011080F83E205448D0F848
:1044900018020521B0FBF1F201FB120101EBC10092
:1044A00000EB01114E48243000EB81000021C0F8E0
:1044B0001D104B48D0F818020521B0FBF1F201FBAA
:1044C000120101EBC10000EB01114548243000EB63
:1044D00081000D3009909DF8AC1040F2231011FBC3
:1044E00000F001E0D5E0B6E13A4901EBC000183038
:1044F0009DF8981001EBC10100EB01102230102251
:10450000014608900998F3F7A0FE3548D0F8180244
:104510000521B0FBF1F201FB120101EBC10000EB40
:1045200001112F48243000EB81029DF8AC1040F2BD
:10453000231011FB00F0274901EBC00118319DF851
:10454000980000EBC00001EB001050F81A1F42F871
:10455000011F406850602248D0F818020521B0FBC6
:10456000F1F201FB120101EBC10000EB01131C4948
:1045700024319DF8AC0000EB400202EB0010194A18
:1045800002EB001230329DF8980002EB0010007828
:1045900001F823001248D0F818020521B0FBF1F20F
:1045A00001FB120101EBC10000EB01110C482430AA
:1045B00000EB81029DF8AC0040F2231110FB01F0EA
:1045C000044901EBC00118319DF898000CE000008F
:1045D000A8780020D4450020BC220020BC32002056
:1045E000BC1200201441002000EBC00001EB0010C1
:1045F000406BC2F80900FE48D0F818020521B0FB54
:10460000F1F201FB120101EBC10000EB0111F848CE
:10461000243000EB8101F748C26941F8212F008C5A
:104620008880F348D0F818020521B0FBF1F081B280
:1046300002200991F4F74CFD00210620F5F78AFCD1
:10464000EB48D0F81802EA49498C884206D2E8487B
:10465000D0F81802401CE649C1F8180200210520D4
:10466000F5F778FC9DF8AC1001EB410000EB011070
:10467000E14901EB001030309DF8981000EB01107B
:10468000801C0990007820F008020998027029E047
:10469000E7E19DF8AC1001EB410000EB0110D649B9
:1046A00001EB001030309DF8981000EB0110801CD9
:1046B0000990007820F0080008300999087000225D
:1046C0009DF8AC0040F2231110FB01F0CB4901EB47
:1046D000C00018309DF8981001EBC10100EB0110EB
:1046E00080F83E209DF8AC100220F5F733FC9DF8D1
:1046F000AC109DF8980000EB0110C217CDE92C0218
:1047000000222C9800EBC00101EB0011BC4800EB2B
:104710008100C0F81D209DF8AC1040F2231011FB61
:1047200000F0B64901EBC00018309DF8981001EB7D
:10473000C10100EB0110223009902C9800EBC00160
:1047400001EB0011AE4800E08AE100EB81000D3082
:10475000102208900999F3F778FD9DF8AC1040F20B
:10476000231011FB00F0A54901EBC00118319DF8A1
:10477000980000EBC00001EB00112C9800EBC00288
:1047800002EB00129E4800EB820051F81A2F40F80D
:10479000012F496841609DF8AC1001EB410000EB2E
:1047A0000110954901EB001130319DF8980001EBA3
:1047B000001001782C9800EBC00202EB0012904828
:1047C00000F822102C9800EBC00101EB00118C487E
:1047D00000EB81018748C26941F8212F008C888055
:1047E0009DF8AC1040F2231011FB00F0834901EB5F
:1047F000C00118319DF8980000EBC00001EB0010DB
:10480000416B2C9800EBC00202EB00127C4800EBDD
:104810008200C0F809109DF8AC1001EB410000EBDC
:104820000110754901EB001130319DF8980001EB42
:10483000001041682C9800EBC00202EB0012704897
:1048400000EB8200C0F827102C9881B20820099153
:10485000F5F780FB80E09DF8AC1040F2231011FBCF
:1048600000F0664901EBC00118319DF8980000EB9B
:10487000C00001EB001001789DF8AC0040F223125B
:1048800010FB02F05D4A02EBC0004079814263DA1E
:104890009DF8AC1001EB410000EB0110564901EB13
:1048A000001030309DF8981000EB0110801C09902A
:1048B000007820F00400001D099908709DF8AC10E4
:1048C00001EB410000EB01104B4901EB00103030CF
:1048D0009DF8981000EB0110801C0990007820F0E2
:1048E000800080300999087001209DF8AC1040F2DA
:1048F000231211FB02F1414A02EBC10108719DF83C
:10490000AC1040F2231011FB00F0114601EBC00087
:1049100042799DF8AC1040F2231011FB00F03749AA
:1049200001EBC00018309DF8981001EBC10100EBBD
:104930000110027014229DF8AC0040F2231110FB0C
:1049400001F02E4901EBC00018309DF8981001EBE2
:10495000C10100EB0110427182E00121254880F87D
:10496000C4179DF8AC1040F2231011FB00F023494E
:1049700001EBC00118319DF8980000EBC00001EB7D
:10498000001001789DF8AC2040F2231012FB00F0DB
:104990001A4A02EBC000407981423ADA00219DF8C0
:1049A000AC2040F2231012FB00F0144A02EBC000CE
:1049B000017101229DF8AC0040F2231110FB01F0BF
:1049C0000E4901EBC00118319DF8980000EBC000C2
:1049D00001EB0010027014229DF8AC1040F223107D
:1049E00011FB00F0054901EBC00018300AE000009F
:1049F000BC120020BC32002014410020D44500200D
:104A0000E41400209DF8981001EBC10100EB0110A7
:104A1000427125E014229DF8AC1040F2231011FBE6
:104A200000F0FE4901EBC00018309DF8981001EB32
:104A3000C10100EB0110427112E014229DF8AC009C
:104A400040F2231110FB01F0F44901EBC0001830D3
:104A50009DF8981001EBC10100EB0110427100BFFD
:104A600000BFF7E39DF8AC1040F2231011FB00F0FB
:104A7000EA4901EBC000817826919DF8AC1001EB6A
:104A80004100C0EBC110E64911F8301027919DF8A4
:104A9000AC1040F2231011FB00F0E04901EBC00123
:104AA00018319DF8980000EBC00001EB001041792F
:104AB00024919DF8AC1001EB4100C0EBC110D84926
:104AC00001EBC0010991BDF89C100998F5F7D2FFE0
:104AD00035909DF8AC1001EB4100C0EBC110D049FE
:104AE00001EBC001BDF89C00095CBDF8D400814217
:104AF0007DD19DF8AC1001EB4100C0EBC110C8495D
:104B000001EBC0004078002871DD0021C54A9DF806
:104B1000AC0002EB00129DF898001154BDF8900013
:104B2000892865D00CDC14287ED004DC08287CD0D1
:104B300010287BD1FDE3152879D08028F9D1F9E33D
:104B40008B2875D08C2874D08E2873D08F28F0D104
:104B5000BDF89C000D286ED19DF8AC1001EB410012
:104B6000C0EBC110AE4901EBC0004178AE4880F8FF
:104B7000151E9DF8AC1001EB4100C0EBC110A84917
:104B800001EBC000C17AA84880F8161E9DF8AC1051
:104B900040F2231011FB00F0A04901EBC0001830D7
:104BA0009DF8981001EBC10100EB0110007803287B
:104BB0007EDC9D4890F8160E00287ADD9DF8AC103A
:104BC00040F2231011FB00F0944901EBC0011831B1
:104BD0009DF8980000EBC00001EB001109910878E6
:104BE000401CC1B2099801709DF8AC1001E0FCE3D3
:104BF000FCE340F2231011FB00F0884901EBC000F8
:104C000018309DF8981001EBC10100EB01100078FD
:104C100004284EDB9DF8AC1001EB410000EB0110C5
:104C2000824901EB001007E0FDE3FDE3FDE3FDE356
:104C3000FDE3FDE3FDE3FDE330309DF8981000EB6C
:104C40000110801C0990784890F8160EC0F30010EF
:104C5000C0F101000999097860F300010998017019
:104C6000714890F8150EC0F3C000E8BB9DF8AC1079
:104C700001EB410000EB01106C4901EB00103030FA
:104C80009DF8981000EB01108078C0F3401058B3E5
:104C90009DF8AC1001EB410000EB0110634901EB02
:104CA000001030309DF8981000EB0110801C01E0DE
:104CB00056E0F0E00990007820F00200801C09998D
:104CC00008709DF8AC1040F2231011FB00F053491E
:104CD00001EBC00018309DF8981001EBC10100EB0A
:104CE00001101830099000E00AE0007820F002007E
:104CF000801C099908709DF8AC100220F5F72AF97C
:104D000000219DF8AC2040F2231012FB00F0434A32
:104D100002EBC000017104229DF8AC0040F22311A7
:104D200010FB01F03D4901EBC00118319DF89800DE
:104D300000EBC00001EB001002708C229DF8AC105B
:104D400040F2231011FB00F0344901EBC00118318F
:104D50009DF8980000EBC00001EB00104271B4E335
:104D60009DF8AC1040F2231011FB00F02B4901EB31
:104D7000C00118319DF8980000EBC00001EB001055
:104D800001789DF8AC0040F2231210FB02F0234A98
:104D900002EBC000407981427DD19DF8AC1001EB5F
:104DA000410000EB0110214901EB001030309DF86B
:104DB000981000EB0110801C09901B4890F8160E0B
:104DC000C0F30010C0F1010009990A7860F30002F5
:104DD0000A709DF8AC1001EB410000EB0110134983
:104DE00001EB001030309DF8981000EB0110801C92
:104DF00009900D4890F8150EC2080998017862F3E1
:104E0000410101709DF8AC1001EB410000EB011075
:104E1000064901EB001130310AE00000D4450020C2
:104E2000A8780020483F0020BC2200201441002028
:104E30009DF8980001EB00108078C0F340029DF8C7
:104E4000AC1040F2231011FB00F0FE4901EBC00052
:104E500018309DF8981001EBC10100EB0110007EA5
:104E6000C0F34000824264D09DF8AC1040F22310A1
:104E700011FB00F0F34901EBC00018309DF89810C9
:104E800001EBC10100EB0110183009909DF8AC1046
:104E900001EB410000E0D5E200EB0112EA4800EB33
:104EA000021030309DF8981000EB01108078420815
:104EB0000998007862F34100099908709DF8AC10D8
:104EC00001EB410000EB0110DF4901EB0010303035
:104ED0009DF8981000EB01108078C0F3400018BBDB
:104EE00001229DF8AC0040F2231110FB01F0D549DE
:104EF00001EBC00118319DF8980000EBC00001EBF8
:104F0000001042739DF8AC1040F2231011FB00F02A
:104F1000CC4901EBC00018309DF8981001EBC1019D
:104F200000EB011080F83E209DF8AC100220F5F750
:104F300011F89DF8AC1001EB410000EB0110C249E3
:104F400001EB001130319DF8980001EB00108078E2
:104F500000F001029DF8AC1040F2231011FB00F0AC
:104F6000B84901EBC00018309DF8981001EBC10161
:104F700000EB0110007E00F00100824277D09DF826
:104F8000AC1040F2231011FB00F0AE4901EBC00061
:104F900018309DF8981001EBC10100EB011018309A
:104FA00009909DF8AC1001EB410000EB0110A649FF
:104FB00001EB001130319DF8980001EB0010817871
:104FC0000998027861F3000202709DF8AC1001EBC1
:104FD000410000EB01109C4901EB001030309DF8BE
:104FE000981000EB0110807800F00100F0BB9DF8F4
:104FF000AC1001EB410000EB0110934901EB0010F4
:1050000030309DF8981000EB01108078C0F340100C
:1050100070B39DF8AC1040F2231011FB00F08949E9
:1050200001EBC00018309DF8981001EBC10100EBB6
:10503000011090F83E00D8B99DF8AC1040F2231052
:1050400011FB00F07F4901EBC00018309DF898106B
:1050500001EBC10100EB0110407B48B99DF8AC1099
:1050600001EB410000EB0110774902E044E070E100
:105070002EE001EB001030309DF8981000EB01108D
:105080008078C0F3400018BB01229DF8AC0040F2CC
:10509000231110FB01F06B4901EBC00118319DF8A1
:1050A000980000EBC00001EB001042739DF8AC10BB
:1050B00040F2231011FB00F0624901EBC0001830F0
:1050C0009DF8981001EBC10100EB011080F83E2023
:1050D00000229DF8AC0040F2231110FB01F0594969
:1050E00001EBC00018309DF8981001EBC10100EBF6
:1050F000011080F83D2027E19DF8AC1040F223100C
:1051000011FB00F04F4901EBC00018309DF89810DA
:1051100001EBC10100EB011090F83E0098B90122AB
:105120009DF8AC1040F2231011FB00F0454901EB53
:10513000C00018309DF8981001EBC10100EB011080
:1051400080F83D2027E000229DF8AC1040F22310AB
:1051500011FB00F03B4901EBC00118319DF89800AC
:1051600000EBC00001EB001080F83D209DF8AC1072
:1051700001EB410000EB0110334901EB001130312C
:105180009DF8980001EB0010801C0990007820F039
:105190000102099802702D4890F8A00880B19DF88E
:1051A000AC1001EB410000EB0110274901EB0010AE
:1051B00030309DF8981000EB0110807A022870D1F1
:1051C000234890F8210001286BD12148D0F818021B
:1051D0001F49498C884264D29DF8AC1040F22310DC
:1051E00011FB00F0174901EBC00018309DF8981032
:1051F00001EBC10100EB011090F83D00012850D1F6
:105200009DF8AC1040F2231011FB00F00D4901EBAA
:10521000C00018309DF8981001EBC10100EB01109F
:1052200090F87E00E8BB9DF8AC1001EB410000EB6C
:105230000110054901EB001130319DF8980001EB98
:10524000001008E0D445002014410020BC320020AA
:10525000BC120020FEE301789DF8AC0040F223125E
:1052600010FB02F0FE4A02EBC000417008229DF8DC
:10527000AC0040F2231110FB01F0F94901EBC00131
:1052800018319DF8980000EBC00001EB001042714E
:1052900000229DF8AC1001EB410000EB0110F14938
:1052A00000E051E001EB001130319DF8980001EB76
:1052B000001042609DF8AC100220F4F74BFE002174
:1052C000379119E000229DF8AC0040F2231110FB49
:1052D00001F0E34901EBC00118319DF8980000EBA3
:1052E000C00001EB00113F31BDF8DC000A54BDF8ED
:1052F000DC00401C81B23791BDF8DC001428E1DBF2
:10530000002037901CE000229DF8AC1040F22310E2
:1053100011FB00F0D24901EBC00118319DF8980053
:1053200000EBC00001EB00115B31BDF8DC000A545A
:1053300001E0FFE1C8E3BDF8DC00401C81B2379119
:10534000BDF8DC000A28DEDB9DF8AC100220F4F783
:1053500001FE9DF8AC1040F2231011FB00F0C04993
:1053600001EBC00018309DF8981001EBC10100EB73
:1053700001108078802835D19DF8AC1001EB4100F8
:1053800000EB0110B74901EB001030309DF8981088
:1053900000EB01108078C0F3400018BB9DF8AC1002
:1053A00001EB410000EB0110AE4901EB0010303081
:1053B0009DF8981000EB01108078C0F3401088B978
:1053C00015229DF8AC0040F2231110FB01F0A44916
:1053D00001EBC00018309DF8981001EBC10100EB03
:1053E000011042719DF8AC1001E0F0E3B9E101EB6E
:1053F000410000EB01109B4901EB001030309DF89B
:10540000981000EB01108078C0F34000D8B18F22D3
:105410009DF8AC1040F2231011FB00F0904901EB15
:10542000C000183007E0FCE362E14DE2FAE3F2E18C
:105430004BE27DE35BE19DF8981001EBC10100EBCD
:105440000110427141E09DF8AC1040F2231011FBB5
:1054500000F0834901EBC00018309DF8981001EB73
:10546000C10100EB0110807B01282ED100229DF8A4
:10547000AC0040F2231110FB01F0794901EBC001AF
:1054800018319DF8980000EBC00001EB001082730A
:105490008C229DF8AC1040F2231011FB00F07049F3
:1054A00001EBC00118319DF8980000EBC00001EB42
:1054B0000010427100219DF8AC2040F2231012FB35
:1054C00000F0674A02EBC00001719DF8AC1001EBDF
:1054D000410000EB0110634901EB0010007BE8BBC9
:1054E0009DF8AC1001EB4100C0EBC1105E4901EB2F
:1054F000C000807800049DF8AC1001EB4102C2EBC3
:10550000C111594A02EBC101C97840EA01209DF856
:10551000AC2002EB4201C1EBC211534A02EBC101C4
:1055200009790843C117CDE9080108F055FC9DF839
:10553000AC1040F2231211FB02F1494A02EBC10206
:1055400018329DF8981001EBC10102EB0111C1F86E
:105550001E009DF8AC1001EB410000E035E0C0EB0F
:10556000C110414901EBC000407900049DF8AC2016
:1055700002EB4201C1EBC2113B4A02EBC101897946
:1055800040EA01209DF8AC2002EB4201C1EBC211C0
:10559000354A02EBC101C9790843C117CDE90801B9
:1055A00008F01AFC9DF8AC1040F2231211FB02F136
:1055B0002B4A02EBC10118319DF8982002EBC20280
:1055C00001EB0211C1F81A0091E09DF8AC1001EB5B
:1055D0004100C0EBC110244901EBC00080780106F6
:1055E0009DF8AC2002EB4200C0EBC2101E4A02EB59
:1055F000C000C07841EA00419DF8AC0000EB4002D9
:10560000C2EBC010184A02EBC000007941EA00204A
:105610009DF8AC2002EB4201C1EBC211124A02EB31
:10562000C10149790843C117CDE9080108F0D4FB4D
:1056300001469DF8AC0040F2231210FB02F0084A2C
:1056400002EBC00218329DF8980000EBC00002EB9C
:105650000010C0F81E109DF8AC1001EB410005E0F1
:10566000D445002014410020A8780020C0EBC110D0
:10567000FE4901EBC000807901069DF8AC0000EB0B
:105680004002C2EBC010F94A02EBC000C07941EA07
:1056900000419DF8AC2002EB4200C0EBC210F34A7F
:1056A00002EBC000007A41EA00219DF8AC0000EB5B
:1056B0004002C2EBC010ED4A02EBC000407A084342
:1056C000C117CDE9080108F087FB9DF8AC2040F236
:1056D000231112FB01F1E64A02EBC10118319DF8DA
:1056E000982002EBC20201EB0211C1F81A00EBE0B4
:1056F000BDF89C0003281CD18F229DF8AC0040F21D
:10570000231110FB01F0DA4901EBC00118319DF8BB
:10571000980000EBC00001EB0010427101219DF8E0
:10572000AC2040F2231012FB00F0D14A02EBC00083
:105730000171C9E0BDF89C00032811D18F229DF8AA
:10574000AC0040F2231110FB01F0C94901EBC0008D
:1057500018309DF8981001EBC10100EB0110427167
:10576000B2E0BDF89C00032854D19DF8AC1040F283
:10577000231011FB00F0BE4901EBC0001830BDF84A
:10578000D01001EBC10100EB01108079012824D178
:1057900000229DF8AC0040F2231110FB01F0B44947
:1057A00001EBC0011831BDF8D00000EBC00001EBE7
:1057B000001082718F229DF8AC1040F2231011FB73
:1057C00000F0AB4901EBC00018309DF8981001EBD8
:1057D000C10100EB011042711CE008229DF8AC00F1
:1057E00040F2231110FB01F0A14901EBC001183177
:1057F0009DF8980000EBC00001EB00104271002101
:105800009DF8AC0040F2231210FB02F0984A02EB24
:10581000C000017158E0BDF89C00032854D19DF8E8
:10582000AC1040F2231011FB00F0914901EBC000D5
:105830001830BDF8D01001EBC10100EB01108079E8
:10584000012824D100229DF8AC1040F2231011FB56
:1058500000F0874901EBC0011831BDF8D00000EB22
:10586000C00001EB001082718F229DF8AC0040F265
:10587000231110FB01F07E4901EBC00018309DF8A8
:10588000981001EBC10100EB011042711CE00822ED
:105890009DF8AC1040F2231011FB00F0744901EBAD
:1058A000C00118319DF8980000EBC00001EB00101A
:1058B000427100219DF8AC2040F2231012FB00F051
:1058C0006B4A02EBC0000171FEE3BDF89C000828A2
:1058D0007ED19DF8AC1001EB4100C0EBC1106349D3
:1058E00001EBC000807801069DF8AC0000EB40029F
:1058F000C2EBC0105D4A02EBC000C07841EA004133
:105900009DF8AC2002EB4200C0EBC210574A02EBFC
:10591000C000007941EA00209DF8AC1001EB410283
:10592000C2EBC111514A02EBC10149790843C117C9
:10593000CDE9080108F050FA9DF8AC2040F223119F
:1059400012FB01F14A4A02EBC10218329DF898108D
:1059500001EBC10102EB011148639DF8AC1040F26C
:10596000231011FB00F0424901EBC00018309DF8F4
:10597000981001EBC10100EB011000789DF8AC100C
:1059800040F2231211FB02F1394A02EBC1014979BD
:10599000884231DA00219DF8AC2040F2231012FB3E
:1059A00000F0334A02EBC000017105229DF8AC0003
:1059B00040F2231110FB01F02D4901EBC001183119
:1059C0009DF8980000EBC00001EB0010027000E0B1
:1059D00079E08E229DF8AC1040F2231011FB00F00C
:1059E000234901EBC00018309DF8981001EBC1016C
:1059F00000EB0110427166E09DF8AC1040F22310FC
:105A000011FB00F01A4901EBC0001830BDF8D010AE
:105A100001EBC10100EB01108079012836D1002291
:105A20009DF8AC0040F2231110FB01F0104901EB8E
:105A3000C0011831BDF8D00000EBC00001EB001030
:105A400082718F229DF8AC1040F2231011FB00F000
:105A5000074900E0FDE301EBC00118319DF8980013
:105A600000EBC00001EB0010427103E0A8780020B9
:105A7000D445002001219DF8AC2040F2231012FBF8
:105A800000F0FE4A02EBC00001711CE08E229DF87E
:105A9000AC1040F2231011FB00F0F84901EBC001FB
:105AA00018319DF8980000EBC00001EB0010427126
:105AB00000219DF8AC0040F2231210FB02F0EF4AE7
:105AC00002EBC0000171FFE2BDF89C0003282ED15B
:105AD00000219DF8AC2040F2231012FB00F0E74AB1
:105AE00002EBC000017101229DF8AC1040F22310BE
:105AF00011FB00F0E14901EBC0011831BDF8D00005
:105B000000EBC00001EB001082718C229DF8AC10FC
:105B100040F2231011FB00F0D84901EBC00018300F
:105B20009DF8981001EBC10100EB01104271CBE22E
:105B3000BDF89C000F2876D19DF8AC1001EB410018
:105B400000EB0110CE4901EB0010007BF0BB002000
:105B50002C902D90002137911FE0DDE92C100002E0
:105B600040EA11620902CDE92C129DF8AC1001EB5C
:105B70004100C0EBC110C34901EBC001BDF8DC001E
:105B8000C0F10600085CDDE92C341843CDE92C0493
:105B9000BDF8DC00401C80B23790BDF8DC00052861
:105BA000DBDB9DF8AC00DDE92C1240F2231310FB87
:105BB00003F0B24B03EBC00318339DF8980000EBE1
:105BC000C00003EB001040F8221F01E046E0FDE3B7
:105BD000426000222C922D920021379120E0DDE9D5
:105BE0002C10000240EA11620902CDE92C129DF846
:105BF000AC1001EB4100C0EBC110A24901EBC001A8
:105C0000BDF8DC00C0F10B00085CDDE92C3440EA93
:105C10000302CDE92C24BDF8DC00401C81B2379191
:105C200002E0E4E349E347E3BDF8DC000528D6DB06
:105C30009DF8AC00DDE92C1240F2231310FB03F0B9
:105C40008E4B03EBC00018309DF8983003EBC30374
:105C500000EB031022308160C2607EE000202C90B7
:105C60002D900021379120E0DDE92C10000240EA60
:105C700011620902CDE92C129DF8AC1001EB410034
:105C8000C0EBC1107F4901EBC001BDF8DC00C0F1E1
:105C90000700085CDDE92C3440EA0302CDE92C243E
:105CA000BDF8DC00401C81B23791BDF8DC0006284D
:105CB000DADB9DF8AC00DDE92C1240F2231310FB77
:105CC00003F06E4B03EBC00318339DF8980000EB14
:105CD000C00003EB001040F8221F426000222C920B
:105CE0002D92002137911FE0DDE92C10000240EADF
:105CF00011620902CDE92C129DF8AC1001EB4100B4
:105D0000C0EBC1105F4901EBC001BDF8DC00C0F180
:105D10000D00085CDDE92C341843CDE92C04BDF8F6
:105D2000DC00401C80B23790BDF8DC000628DBDBCD
:105D30009DF8AC00DDE92C2140F2231310FB03F0A9
:105D40004E4B03EBC00018309DF8983003EBC303B3
:105D500000EB031022308260C1609DF8AC1040F26D
:105D6000231011FB00F0454901EBC00118319DF8EB
:105D7000980000EBC00001EB001001789DF8AC002A
:105D800040F2231210FB02F03C4A02EBC0004079C3
:105D9000814272D13C4890F8A008E8BB3B48D0F85B
:105DA00018020521B0FBF1F201FB120101EBC10069
:105DB00000EB01113548243000EB81000021C0F8D0
:105DC0001D103248D0F818020521B0FBF1F201FB9A
:105DD000120101EBC10000EB01112C48243000EB53
:105DE00081000D3009909DF8AC1040F2231011FB9A
:105DF00000F0224901EBC00118319DF8980000EB3A
:105E0000C00001EB001022301022014608900998D2
:105E1000F2F71BFA1D4800E0E4E0D0F81802052173
:105E2000B0FBF1F201FB120101EBC10000EB01112B
:105E30001648243000EB81029DF8AC0040F223119B
:105E400010FB01F00D4901EBC00118319DF89800DD
:105E500000EBC00001EB001050F81A1F42F8011FC0
:105E6000406850600948D0F818020521B0FBF1F2F3
:105E700001FB120101EBC1000AE0ABE1D4450020B7
:105E800014410020A8780020BC320020BC12002061
:105E900000EB0113FE499DF8AC0000EB400202EB61
:105EA0000010FC4A02EB001230329DF8980002EB21
:105EB0000010007801F82300A1F12400D0F81802A6
:105EC0000521B0FBF1F201FB120101EBC10000EB77
:105ED0000111EF4800EB8101EF48C26941F8212F21
:105EE000008C8880EA482438D0F818020521B0FBDD
:105EF000F1F201FB120101EBC10000EB0111E448DA
:105F000000EB81029DF8AC1040F2231011FB00F071
:105F1000E24901EBC00118319DF8980000EBC00088
:105F200001EB0010406BC2F80900D9482438D0F8C2
:105F300018020521B0FBF1F201FB120101EBC100D7
:105F400000EB0111D24800EB81029DF8AC0000EBA0
:105F5000400101EB0010CF4901EB001130319DF8F9
:105F6000980001EB00104068C2F82700C8482438A8
:105F7000D0F818020521B0FBF1F081B2022009919E
:105F8000F3F7A6F800210620F3F7E4FFC048243811
:105F9000D0F81802BE492439498C884208D2BC483E
:105FA0002438D0F81802401CB9492439C1F8180225
:105FB00000210520F3F7CEFF9DF8AC1001EB410066
:105FC00000EB0110B34901EB001030309DF8981040
:105FD00000EB0110801C0990007820F0080209985D
:105FE000027015E09DF8AC1001EB410000EB0110D0
:105FF000A84901EB001030309DF8981000EB01101B
:10600000801C0990007820F0080008300999087079
:106010009DF8AC1001EB410000EB01109D4901EB34
:10602000001030309DF8981000EB0110801C099092
:10603000007820F02002099802709DF8AC10022030
:10604000F3F788FF9DF8AC009DF8981001EB001065
:10605000C217CDE92C0200222C9800EBC00101EB05
:1060600000118F4800EB8100C0F81D209DF8AC1096
:1060700040F2231011FB00F0884901EBC0001830FA
:106080009DF8981001EBC10100EB0110223009903E
:106090002C9800EBC00101EB0011814800EB81015D
:1060A0000D3110220891DDE90801F2F7CEF89DF8D4
:1060B000AC1040F2231011FB00F0784901EBC00155
:1060C00018319DF8980000E0ACE100EBC00001EB56
:1060D00000112C9800EBC00202EB0012704800EB9C
:1060E000820051F81A2F40F8012F496841609DF84D
:1060F000AC1001EB410000EB0110664901EB00110F
:1061000030319DF8980001EB001001782C9800EBDD
:10611000C00202EB0012624800F822102C9800EB3B
:10612000C00101EB00115E4800EB81015A48C269D1
:1061300041F8212F008C88809DF8AC1040F223108C
:1061400011FB00F0554901EBC00118319DF8980092
:1061500000EBC00001EB0010416B2C9800EBC0027B
:1061600002EB00124E4800EB8200C0F809109DF8C7
:10617000AC1001EB410000EB0110464901EB0011AE
:1061800030319DF8980001EB001041682C9800EB2D
:10619000C00202EB0012424800EB8200C0F8271058
:1061A0002C9881B208200991F3F7D4FE00229DF8C3
:1061B000AC0040F2231110FB01F0384901EBC000A4
:1061C00018309DF8981001EBC10100EB011080F828
:1061D0003E2053E09DF8AC1001EB410000EB0110B4
:1061E0002C4901EB001030309DF8981000EB0110A5
:1061F000801C0990007820F00401091D09980170A5
:106200009DF8AC1001EB410000EB0110214901EBBE
:10621000001130319DF8980001EB0010801C0990AE
:10622000007820F0800080300999087001209DF8E6
:10623000AC1040F2231211FB02F1184A02EBC1012B
:1062400008719DF8AC1040F2231011FB00F01146CC
:1062500000E0E9E001EBC00042799DF8AC0040F2BB
:10626000231110FB01F00D4901EBC00018309DF81F
:10627000981001EBC10100EB011002708F229DF814
:10628000AC0040F2231110FB01F004490AE00000C9
:10629000E012002014410020BC320020D445002030
:1062A000E414002001EBC00018309DF8981001EBB9
:1062B000C10100EB01104271B4E0BDF89C0003285D
:1062C0004FD10121FE4880F8C4179DF8AC1040F270
:1062D000231011FB00F0FB4901EBC00118319DF8C0
:1062E000980000EBC00001EB001001789DF8AC00B5
:1062F00040F2231210FB02F0F24A02EBC000407998
:1063000081422FDA00219DF8AC2040F2231012FBCD
:1063100000F0EC4A02EBC000017101229DF8AC10C4
:1063200040F2231011FB00F0E64901EBC0011831E7
:106330009DF8980000EBC00001EB001002708F2266
:106340009DF8AC0040F2231110FB01F0DD4901EB98
:10635000C00018309DF8981001EBC10100EB01104E
:10636000427143E09DF8AC1040F2231011FB00F0A5
:10637000D44901EBC00018309DF8981001EBC10121
:1063800000EB01108078802830D100219DF8AC20EE
:1063900040F2231012FB00F0CA4A02EBC000017168
:1063A00080229DF8AC1040F2231011FB00F0C5498B
:1063B00001EBC00118319DF8980000EBC00001EB23
:1063C0000010427100229DF8AC0000E02BE040F28A
:1063D000231110FB01F0BB4901EBC00018309DF800
:1063E000981001EBC10100EB011082701AE0BDF8BA
:1063F0009C00032815D10021B14880F8C4178F22D2
:106400009DF8AC1040F2231011FB00F0AD4901EBF8
:10641000C00018309DF8981001EBC10100EB01108D
:10642000427100BF00BF00BF00BFA548C07EB0B131
:10643000A5499DF8AC0031F8101009919DF8AC10F9
:1064400001EB4100C0EBC111A04800EBC1010123E9
:1064500008919DF8AC20DDE90801F4F723FB002149
:10646000379111E000219DF8AC0000EB4002C2EB37
:10647000C010964A02EBC002BDF8DC001154BDF812
:10648000DC00401C81B23791BDF8DC00142843DAEF
:10649000E8E78F499DF8AC0011F81000C009D8BB9F
:1064A0009DF8AC0011F81000C0F3C300062832D2EA
:1064B000DFE800F0036291FDFC339DF8AC1001EBC6
:1064C0004100C0EBC110814901EBC001099181A1DC
:1064D000099815F047FD11901198E0B100219DF841
:1064E000AC0000EB40007A4A3C3202EB8000416095
:1064F00001219DF8AC0000EB400002EB80008170B0
:1065000073499DF8AC0001EB40010991087820F037
:1065100078002830087060E160E19DF8AC1001EB74
:106520004100C0EBC110694901EBC001099169A1AB
:10653000099815F017FD11901198E0B100219DF810
:10654000AC0000EB4000624A3C3202EB800041604C
:1065500001219DF8AC0000EB400002EB800081704F
:106560005B499DF8AC0001EB40010991087820F0EF
:1065700078002030087030E19DF8AC1001EB41004C
:10658000C0EBC110514901EBC001099151A109981B
:1065900015F0E8FC11901198E0B100219DF8AC00D5
:1065A00000EB40004A4A3C3202EB8000416001218E
:1065B0009DF8AC0000EB400002EB80008170444984
:1065C0009DF8AC0001EB40010991087820F07800BB
:1065D0001830087001E100219DF8AC0000EB40008C
:1065E0003B4A3C3202EB8000416001219DF8AC0047
:1065F00000EB400002EB800081709DF8AC1001EBD5
:106600004100C0EBC110314901EBC0011198801D60
:10661000095C30399DF8AC2002EB4200C0EBC2109F
:106620002A4A02EBC0031198401D185C303841EA39
:106630000010C117CDE9080106F018FE264988713F
:106640009DF8AC1001EB4100C0EBC1101F4901EBFC
:10665000C001099121A1099815F084FC11901198AD
:1066600030B39DF8AC1001EB4100C0EBC1101749ED
:1066700001EBC0011198401C085C302837DB9DF805
:10668000AC1001EB4100C0EBC110104901EBC0019F
:106690001198401C095C30399DF8AC2002EB420097
:1066A000C0EBC210094A02EBC00302E06BE03DE020
:1066B00030E01198185C303841EA0010C1170FE043
:1066C000BC320020D4450020346A0020A878002085
:1066D000DC3E00204F4B00005C3B00202C00000003
:1066E000CDE9080106F0C2FD4449C87112E09DF8E9
:1066F000AC1001EB4100C0EBC110414901EBC001FE
:106700001198085C3038C117CDE9080106F0AEFDDC
:106710003A49C8713B499DF8AC0001EB4001099131
:10672000087820F078001830087056E09DF8AC101A
:1067300001EB4100C0EBC110314901EBC0010991EF
:10674000AFF27001099815F00DFC11901198C8B1C5
:1067500000202D4908602B499DF8AC0001EB400159
:106760000991087820F080018031099801704FF478
:106770007A719DF8AC0000EB4000224A3C3202EBFB
:106780008000816029E09DF8AC1001EB4100C0EB76
:10679000C1101B4901EBC0010991AFF2C801099872
:1067A00015F0E0FB11901198B0B1184890F8C607A9
:1067B00020F08001154880F8C61712499DF8AC00FA
:1067C00001EB40010991087820F07800083008704A
:1067D00000200F498870486000BF00BF0D48007856
:1067E0000D49097808440D49097808440C4909788D
:1067F0000844002874F46AAB38B070BD5C3B0020DC
:10680000A8780020DC3E002088024242BC320020F2
:10681000746A0020120000201300002014000020E1
:106820001500002007B5D4B000211A9119911891D4
:1068300017911691159114910022129213921092B1
:1068400011920F910E910D910C910B910A91F7A05D
:1068500006C8CDE90812F7A006C8CDE90612002146
:1068600005910020F5490870549800EB400101EBB8
:106870000010F34901EB001081791691F149549809
:1068800001EB00115598085C05287DDD0621ED4AD5
:10689000549802EB001255981154002240F2231133
:1068A00054984843E84901EBC0011831559800EB72
:1068B000C00001EB00100270549800EB400101EBA6
:1068C0000010DF4901EB00113031559801EB001049
:1068D000807820F08002549800EB400101EB00101A
:1068E000D74901EB00113031559801EB001082704F
:1068F00040F2231154984843D34901EBC0011831A9
:10690000559800EBC00001EB001090F88E0020F0CD
:10691000080240F2231154984843CB4901EBC001CF
:106920001831559800EBC00001EB001080F88E2064
:1069300040F2231154984843C34901EBC001183178
:10694000559800EBC00001EB001090F88E0020F08D
:10695000010240F2231154984843BB4901EBC001A6
:106960001831559800EBC00001EB001080F88E2024
:10697000549800EB400101EB0010B14901EB00100D
:106980008079092817D200E087E0DFE800F085056C
:106990001525354555657500E52240F223115498BB
:1069A0004843A94901EBC0001830559901EBC101DA
:1069B00000EB011042716FE0A12240F223115498C4
:1069C0004843A14901EBC0001830559901EBC101C2
:1069D00000EB011042715FE0A12240F223115498B4
:1069E0004843994901EBC0001830559901EBC101AA
:1069F00000EB011042714FE0B12240F22311549894
:106A00004843914901EBC0001830559901EBC10191
:106A100000EB011042713FE0312240F22311549803
:106A20004843894901EBC0001830559901EBC10179
:106A300000EB011042712FE0F42240F22311549830
:106A40004843814901EBC0001830559901EBC10161
:106A500000EB011042711FE0062240F2231154980E
:106A60004843794901EBC0001830559901EBC10149
:106A700000EB011042710FE0152240F223115498EF
:106A80004843714901EBC0001830559901EBC10131
:106A900000EB0110427100BF00BF6A496C39549885
:106AA00011F810000121B1EBD01F46F0F4816748C6
:106AB00090F82000012806F0DF819DF8580000289A
:106AC000F9D09DF858000A2886F06E81DFE810F0B2
:106AD0001F2B0A004A094F0EC4123A167C17712068
:106AE00021279F2D549800EB400101EB00105449E1
:106AF00001EB00113031559801EB00104178084648
:106B00000491002107F068F9C1B2159140F22311F8
:106B1000549848434C4901EBC0011831559800EB9B
:106B2000C00001EB0010017840F22312549850434A
:106B3000454A02EBC0004079814208D1012140F270
:106B4000231254985043404A02EBC00001713D4962
:106B5000549801EB00115598085C401CC1B2394AA9
:106B6000549802EB00125598115440F22311549896
:106B70004843354901EBC0001830559901EBC1017C
:106B800000EB011090F88E00C0F3C00090B1549853
:106B900000EB400101EB0010294901EB00104179A5
:106BA0000B464FF4805204914FF4E131549807F0B2
:106BB00001F819E0549800EB400101EB0010204966
:106BC00001EB001041790491549800EB400101EB76
:106BD00000101B4901EB0010016803914FF4805233
:106BE000049B549806F0E6FF5698C52876D012DC30
:106BF000B52874D008DC112872D0122871D013285F
:106C000070D0B22869D1A0E3B6286CD0B9286BD077
:106C1000C328F7D1DCE2D92868D019DCCA287DD096
:106C2000CE287CD0D528EDD119E0000001693230A2
:106C3000313030000169323045303000160000201C
:106C400014410020483F0020D4450020BC12002001
:106C5000E12865D0E5287DD0E728D3D1FAE3F521F6
:106C60005498C0EB001000EB8000F54A02F8301099
:106C70009DF854105498C0EB001000EB800002EB1C
:106C8000C0004170A2215498C0EB001000EB8000BE
:106C900002EBC0008170D5215498C0EB001000EBCE
:106CA000800002EBC000C1705498C0EB001000EBF4
:106CB0008000114601EBC00104910321049806F005
:106CC00067FF01465498C0EB001000EB8000DC4ADF
:106CD00002EBC000017105210F91FDE3FDE34AE0E5
:106CE000FCE3FCE3FCE3F1E258E1FFE7F521549813
:106CF000C0EB001000EB8000D14A02F830109DF884
:106D000054105498C0EB001000EB800002EBC00060
:106D10004170A2215498C0EB001002E097E2F4E326
:106D2000F4E300EB800002EBC0008170D92154989D
:106D3000C0EB001000EB800002EBC000C170549863
:106D4000C0EB001000EB8000114601EBC001049184
:106D5000032100E0FAE3049806F01AFF0146549874
:106D6000C0EB001000EB8000B54A02EBC0000171DF
:106D700005210F91B1E7F5215498C0EB001000EB0D
:106D80008000AF4A02F830109DF854105498C0EBC0
:106D9000001000EB800002EBC0004170549800EB43
:106DA000400101EB0010A74901EB0010007B002817
:106DB0007AD140F2231154984843A34901EBC00013
:106DC0001830559901EBC10100EB01108068B0F556
:106DD000100F05D34FF410000021CDE9100110E091
:106DE00040F2231154984843974901EBC0001830F2
:106DF000559901EBC10100EB011080680022CDE93B
:106E00001002A5215498C0EB001000EB80008C4AC2
:106E100002EBC000817000211A911CE0BDF86800EF
:106E2000C0F10200C200DDE91001CDE91B10F1F74D
:106E3000FAF9C2B25498C0EB001000EB8000804910
:106E400001EBC003BDF86800C01C1A54BDF868000F
:106E5000401C80B21A90BDF868000328DEDBB52123
:106E60005498C0EB001000EB8000754A02EBC000A4
:106E700081715498C0EB001000EB8000114601EBCB
:106E8000C00104910621049806F082FE0146549840
:106E9000C0EB001000EB8000694A02EBC000C1713A
:106EA00008210F9179E0FFE740F2231154984843FD
:106EB000654901EBC0001830559901EBC10100EBA9
:106EC00001108068B0F1104F05D34FF01041002041
:106ED000CDE9101010E040F22311549848435A496C
:106EE00001EBC0001830559901EBC10100EB011016
:106EF00080680022CDE91002A6215498C0EB001052
:106F000000EB80004E4A02EBC000817000211A9114
:106F10001CE0BDF86800C0F10300C200DDE910010B
:106F2000CDE91D10F1F77FF9C2B25498C0EB001003
:106F300000EB8000424901EBC003BDF86800C01CB3
:106F40001A54BDF86800401C80B21A90BDF8680061
:106F50000428DEDBB5215498C0EB001000EB800064
:106F6000374A02EBC000C1715498C0EB001000EB2F
:106F70008000114601EBC00104910721049806F03E
:106F800007FE01465498C0EB001000EB80002C4A2D
:106F900002EBC000017209210F919EE6F521549881
:106FA000C0EB001000EB8000254A02F830109DF87D
:106FB00054105498C0EB001000EB800002EBC000AE
:106FC0004170549800EB400101EB00101D4901EBAA
:106FD0000010007BD0BB40F22311549848431A495B
:106FE00001EBC0001830559901EBC10100EB011015
:106FF0008068B0F5100F05D14FF410010020CDE9E5
:10700000101010E040F22311549848430E4901EB50
:10701000C0001830559901EBC10100EB01108068E8
:107020000022CDE91002A5215498C0EB001000EB1E
:107030008000034A02EBC000817000211A9123E016
:10704000486F002014410020D445002044E0BDF8E2
:107050006800C0F10200C200DDE91001CDE91F1097
:10706000F1F7E1F8C2B25498C0EB001000EB8000D9
:10707000F94901EBC003BDF86800C01C1A54BDF803
:107080006800401C80B21A90BDF868000328DEDB5F
:10709000B9215498C0EB001000EB8000EE4A02EBDF
:1070A000C00081715498C0EB001000EB80001146C5
:1070B00001EBC00104910621049806F069FD014628
:1070C0005498C0EB001000EB8000E34A02EBC000D4
:1070D000C17108210F917AE040F22311549848437E
:1070E000DE4901EBC0001830559901EBC10100EBFE
:1070F00001108068B0F1104F05D14FF01040002111
:10710000CDE9100110E040F2231154984843D349CF
:1071100001EBC0001830559901EBC10100EB0110E3
:1071200080680022CDE91002A6215498C0EB00101F
:1071300000EB8000C84A02EBC000817000211A9168
:107140001EE0BDF86800C0F10300C200DDE91010C8
:10715000CDE9210108462199F1F765F8C2B25498AA
:10716000C0EB001000EB8000BB4901EBC003BDF891
:107170006800C01C1A54BDF86800401C80B21A9008
:10718000BDF868000428DCDBB9215498C0EB00107E
:1071900000EB8000B04A02EBC000C1715498C0EB14
:1071A000001000EB8000114601EBC00104910721A3
:1071B000049806F0EDFC01465498C0EB001000EB7B
:1071C0008000A54A02EBC000017209210F9184E5FD
:1071D000F5215498C0EB001000EB80009E4A02F8A5
:1071E00030109DF854105498C0EB001000EB800054
:1071F00002EBC0004170A2215498C0EB001000EBDC
:10720000800002EBC0008170C3215498C0EB0010D5
:1072100000EB800002EBC000C1705498C0EB00107E
:1072200000EB8000114601EBC0010491032104989A
:1072300006F0AEFC01465498C0EB001000EB800055
:10724000854A02EBC000017105210F9145E5F5214A
:107250005498C0EB001000EB80007F4A02F8301019
:107260009DF854105498C0EB001000EB800002EB26
:10727000C0004170A2215498C0EB001000EB8000C8
:1072800002EBC0008170CA215498C0EB001000EBE3
:10729000800002EBC000C1705498C0EB001000EBFE
:1072A0008000114601EBC00104910321049806F00F
:1072B0006FFC01465498C0EB001000EB8000664A5A
:1072C00002EBC000017105210F9106E5F5215498EC
:1072D000C0EB001000EB80005F4A02F830109DF810
:1072E00054105498C0EB001000EB800002EBC0007B
:1072F0004170A2215498C0EB001000EB800002EB1B
:10730000C0008170B6215498C0EB001000EB8000E3
:1073100002EBC000C1705498C0EB001000EB80007D
:10732000114601EBC00104910321049806F030FCE2
:1073300001465498C0EB001000EB8000464A02EB77
:10734000C000017105210F91C7E4F5215498C0EBED
:10735000001000EB8000404A02F830109DF85410F5
:107360005498C0EB001000EB800002EBC0004170AD
:10737000549800EB400101EB0010394901EB00107B
:10738000007BE0BBA4215498C0EB001000EB800010
:1073900002EBC000817000211A9124E040F2231119
:1073A000549848432D4901EBC0011831559800EB22
:1073B000C00001EB0010416BBDF86800C0F1010096
:1073C000C000C1405498C0EB001000EB8000224A7E
:1073D00002EBC002BDF86800C01C1154BDF8680083
:1073E000401C81B21A91BDF868000228D6DBB22198
:1073F0005498C0EB001000EB8000174A00E01CE03E
:1074000002EBC00041715498C0EB001000EB80000B
:10741000114601EBC00104910521049806F0B8FB68
:1074200001465498C0EB001000EB80000A4A02EBC2
:10743000C000817107210F9166E0A5215498C0EB2F
:10744000001000EB8000044A02EBC00081700021B4
:107450001A912CE094E20000486F0020D4450020EF
:107460001441002040F2231154984843F74901EB9E
:10747000C0011831559800EBC00001EB0010416BC2
:10748000BDF86800C0F10200C000C1405498C0EBD4
:10749000001000EB8000EE4A02EBC002BDF868006D
:1074A000C01C1154BDF86800401C81B21A91BDF88F
:1074B00068000328D6DBB2215498C0EB001000EB23
:1074C0008000E34A02EBC00081715498C0EB0010C9
:1074D00000EB8000114604E012E285E08FE2EBE26F
:1074E00044E301EBC00104910621049806F050FB2F
:1074F00001465498C0EB001000EB8000D44A02EB28
:10750000C000C17108210F91FAE1ACE0FFE7F5215D
:107510005498C0EB001000EB8000CD4A02F8301008
:107520009DF854105498C0EB001000EB800002EB63
:10753000C0004170A6215498C0EB001000EB800001
:1075400002EBC000817000211A9125E0D9E140F2E0
:10755000231154984843BD4901EBC0011831559897
:1075600000EBC00001EB0010816BBDF86800C0F1BA
:107570000300C000C1405498C0EB001000EB800035
:10758000B34A02EBC002BDF86800C01C1154BDF83C
:107590006800401C81B21A91BDF868000428D6DB4F
:1075A000E1215498C0EB001000EB8000A84A02EBE8
:1075B000C000C1715498C0EB001000EB8000114670
:1075C00001EBC00104910721049806F0E1FA01469D
:1075D0005498C0EB001000EB80009D4A02EBC00005
:1075E000017209210F91BAE3F5215498C0EB001004
:1075F00000EB8000964A02F830109DF85410549821
:10760000C0EB001000EB800002EBC0004170A22133
:107610005498C0EB001000EB800002EBC0008170BA
:10762000C5215498C0EB001000EB800002EBC000B5
:10763000C1705498C0EB001000EB8000114601EBC4
:10764000C00104910321049806F0A2FA014654985F
:10765000C0EB001000EB80007D4A02EBC00001711E
:1076600005210F917BE3F5215498C0EB001000EB4E
:107670008000774A02F830109DF854105498C0EBFF
:10768000001000EB800002EBC0004170549800EB4A
:10769000400101EB00106F4901EB0010007BE8BBDB
:1076A000AC215498C0EB001000EB800002EBC0004E
:1076B000817000211A912CE040F223115498484324
:1076C000624901EBC0001830559901EBC10100EB94
:1076D000011050F8221F4068BDF86820C2F1040272
:1076E000D200CDE9230108462399F0F79CFDC2B2F0
:1076F0005498C0EB001000EB8000554901EBC0032B
:10770000BDF86800C01C1A54BDF86800401C80B267
:107710001A90BDF868000528CEDB00E055E0002196
:107720001A912AE040F2231154984843474901EB4B
:10773000C0001830559901EBC10100EB0111223155
:107740008868C968BDF86820C2F10402D200CDE99A
:107750002510F0F768FDC2B25498C0EB001000EBA2
:1077600080003B4901EBC003BDF8680008301A54A3
:10777000BDF86800401C80B21A90BDF8680005286A
:10778000D0DBCE215498C0EB001000EB8000304AD3
:1077900002EBC00041735498C0EB001000EB800076
:1077A000114601EBC00104910D21049806F0F0F997
:1077B00001465498C0EB001000EB8000244A02EB15
:1077C000C00081730F210F919AE0AE215498C0EB55
:1077D000001000EB80001E4A02EBC0008170002107
:1077E0001A912CE040F2231154984843174901EBB9
:1077F000C0001830559901EBC10100EB011050F8A1
:10780000221F4068BDF86820C2F10502D200CDE910
:10781000270108462799F0F706FDC2B25498C0EB3D
:10782000001000EB80000A4901EBC003BDF86800BE
:10783000C01C1A54BDF86800401C80B21A90BDF8F4
:1078400068000628CEDB00211A9132E0D4450020E2
:10785000486F00201441002040F2231154984843FF
:10786000FE4901EBC0001830559901EBC10100EB56
:10787000011022308168C068BDF86820C2F105029D
:10788000D200CDE9290108462999F0F7CCFCC2B213
:107890005498C0EB001000EB8000F14901EBC003ED
:1078A000BDF8680009301A54BDF86800401C80B269
:1078B0001A90BDF868000628CEDBCE215498C0EBA4
:1078C000001000EB8000E64A02EBC000C173549840
:1078D000C0EB001000EB8000114601EBC0010491E9
:1078E0000F21049806F054F901465498C0EB00109B
:1078F00000EB8000DA4A02EBC000017411210F9105
:107900002DE2F5215498C0EB001000EB8000D44A22
:1079100002F830109DF854105498C0EB001000EBA2
:10792000800002EBC0004170A2215498C0EB00100F
:1079300000EB800002EBC0008170E5215498C0EBA1
:10794000001000EB800002EBC000C1705498C0EB47
:10795000001000EB8000114601EBC00104910321EF
:10796000049806F015F901465498C0EB001000EB9E
:107970008000BB4A02EBC000017105210F91EEE1CE
:10798000F5215498C0EB001000EB8000B44A02F8D7
:1079900030109DF854105498C0EB001000EB80009C
:1079A00002EBC0004170A2215498C0EB001000EB24
:1079B000800002EBC0008170E7215498C0EB0010FA
:1079C00000EB800002EBC000C1705498C0EB0010C7
:1079D00000EB8000114601EBC001049103210498E3
:1079E00006F0D6F801465498C0EB001000EB80007A
:1079F0009B4A02EBC000017105210F91AFE1F52117
:107A00005498C0EB001000EB8000954A02F830104B
:107A10009DF854105498C0EB001000EB800002EB6E
:107A2000C0004170A2215498C0EB001000EB800010
:107A300002EBC000817011215498C0EB001000EBE4
:107A4000800002EBC000C1705498C0EB001000EB46
:107A50008000114601EBC00104910321049806F057
:107A600097F801465498C0EB001000EB80007C4A68
:107A700002EBC000017105210F91012240F2231198
:107A800054984843754901EBC0011831559800EBF3
:107A9000C00001EB00100270D52240F2231154986F
:107AA00048436E4901EBC0001830559901EBC10104
:107AB00000EB0110427152E1F5215498C0EB001027
:107AC00000EB8000664A02F830109DF8541054987C
:107AD000C0EB001000EB800002EBC0004170A5215C
:107AE0005498C0EB001000EB800002EBC0008170E6
:107AF00001215498C0EB001000EB800002EBC000A5
:107B0000C170C2215498C0EB001000EB800002EB62
:107B1000C000017100215498C0EB001000EB800000
:107B200002EBC000417112215498C0EB001000EB31
:107B3000800002EBC00081715498C0EB001000EB94
:107B40008000114601EBC00104910621049806F063
:107B50001FF801465498C0EB001000EB8000404A2B
:107B600002EBC000C17108210F91F8E0F521549893
:107B7000C0EB001000EB8000394A02F830109DF88D
:107B800054105498C0EB001000EB800002EBC000D2
:107B90004170FF215498C0EB001000EB800002EB15
:107BA000C000817000211A911CE0549800EB400144
:107BB00001EB00102B4901EB00110E31BDF86800FC
:107BC000095C5498C0EB001000EB8000244A02EBE3
:107BD000C002BDF86800C01C1154BDF86800401C0C
:107BE00081B21A91BDF868000A28DEDB549800EBD8
:107BF000400101EB00101B4901EB0010408B01120A
:107C00005498C0EB001000EB8000154A02EBC00056
:107C10004173549800EB400101EB0010114901EB56
:107C20000010408BC1B25498C0EB001000EB8000F4
:107C300002EBC000817340F2231154984843074976
:107C400001EBC0011831559800EBC00001EB0010AA
:107C5000B0F88C000112549806E00000D4450020D2
:107C6000486F002014410020C0EB001000EB8000A2
:107C700002EBC000C17340F2231154984843FE49FF
:107C800001EBC0011831559800EBC00001EB00106A
:107C9000B0F88C00C1B25498C0EB001000EB80002B
:107CA00002EBC000017440F2231154984843F2499A
:107CB00001EBC0011831559800EBC00001EB00103A
:107CC000B0F88C10549801EB802081B2032004910D
:107CD000F1F762F900211A9114E0E849BDF8680053
:107CE000095C5498C0EB001000EB8000E44A02EB02
:107CF000C002BDF8680011301154BDF86800401C86
:107D000081B21A91BDF86800B0F5007FE5DB132160
:107D10005498C0EB001000EB8000D94A02EBC00081
:107D200080F811125498C0EB001000EB800011464F
:107D300001EBC001049140F21121049805F028FFE5
:107D400001465498C0EB001000EB8000CC4A02EBD7
:107D5000C00080F8121240F213210F9100BF00BF43
:107D600005F022B8549800EB400101EB0010C54922
:107D700001EB00113031559801EB0010417815915D
:107D800040F2231154984843BB4901EBC00118311C
:107D9000559800EBC00001EB0010017840F223126F
:107DA00054985043B44A02EBC0004079814208D154
:107DB000012140F2231254985043AF4A02EBC00015
:107DC0000171B149549801EB00115598085C401CB1
:107DD000C1B2AD4A549802EB0012559811549DF867
:107DE0005400002804DD9DF85400401EC1B21591D6
:107DF0005698A1380A287CD2DFE800F0FEFDFCFB93
:107E0000FAF9F805F7F602215498C0EB001000EBE0
:107E100080009B4A02F830109DF854004030C1B2F7
:107E20005498C0EB001000EB800002EBC0004170E2
:107E300041215498C0EB001000EB800002EBC00021
:107E4000817030215498C0EB001000EB800002EBF1
:107E5000C000C1705498C0EB001000EB800002EB32
:107E6000C000017140F2231154984843824901EB4C
:107E7000C0011831559800EBC00001EB00100079EB
:107E800001095498C0EB001000EB800002EBC00029
:107E900041715498C0EB001000EB8000114601EBDB
:107EA000C00040790A2812DA5498C0EB001000EBA9
:107EB000800001EBC00040793030C1B25498C0EB73
:107EC000001000EB800002EBC000417115E05498F7
:107ED000C0EB001000EB8000694901EBC000407965
:107EE0003730C1B25498C0EB001000EB8000644AF8
:107EF00000E044E202EBC000417140F223115498CB
:107F000048435D4901EBC0011831559800EBC000B2
:107F100001EB0010007900F00F015498C0EB001045
:107F200000EB8000564A02EBC00081715498C0EB10
:107F3000001000EB8000114601EBC00080790A2898
:107F400012DA5498C0EB001000EB800001EBC00087
:107F500080793030C1B25498C0EB001000EB800043
:107F600002EBC000817113E05498C0EB001000EBED
:107F70008000434901EBC00080793730C1B254988A
:107F8000C0EB001000EB80003D4A02EBC0008171A5
:107F900003225498C0EB001000EB8000384901EB3D
:107FA000C000C2715498C0EB001000EB800001EBE0
:107FB000C000401C07210490F1F78CFA0146549848
:107FC000C0EB001000EB80002D4A02EBC0000172F4
:107FD00009210F9140F2231154984843264901EB9F
:107FE000C0001830559908E05BE1BEE0A7E391E3DB
:107FF000E2E2C5E10CE165E02EE001EBC10100EB3E
:108000000110007804280ED1052240F22311549863
:108010004843194901EBC0001830559901EBC101E3
:1080200000EB01100270002140F2231254985043DB
:10803000114A02EBC0000171062240F2231154984C
:1080400048430D4901EBC0001830559901EBC101BF
:1080500000EB0110027087E304215498C0EB00107C
:1080600000EB8000064A02F830109DF854004030C2
:10807000C1B254980AE00000D4450020D630002058
:10808000486F002014410020483F0020C0EB001042
:1080900000EB800002EBC000417051215498C0EB0E
:1080A000001000EB800002EBC000817005215498A5
:1080B000C0EB001000EB800002EBC000C170042197
:1080C0000F9151E302215498C0EB001000EB8000A7
:1080D000FE4A02F830109DF854004030C1B2549866
:1080E000C0EB001000EB800002EBC00041704121AA
:1080F0005498C0EB001000EB800002EBC0008170D0
:1081000031215498C0EB001000EB800002EBC0005E
:10811000C17035215498C0EB001000EB800002EBD9
:10812000C000017103215498C0EB001000EB8000E7
:1081300002EBC00041715498C0EB001000EB8000CE
:10814000114601EBC000401C05210490F1F7C2F973
:1081500001465498C0EB001000EB8000DB4A02EBB4
:10816000C000817107210F91FEE202215498C0EBFB
:10817000001000EB8000D54A02F830109DF8540042
:108180004030C1B25498C0EB001000EB800002EB0D
:10819000C000417041215498C0EB001000EB8000FA
:1081A00002EBC000817032215498C0EB001000EB4C
:1081B000800002EBC000C17030215498C0EB001069
:1081C00000EB800002EBC000017103215498C0EB6A
:1081D000001000EB800002EBC00041715498C0EB2E
:1081E000001000EB8000114601EBC000401C05218F
:1081F0000490F1F76FF901465498C0EB001000EBC2
:108200008000B24A02EBC000817107210F91ABE2FE
:1082100004215498C0EB001000EB8000AB4A02F838
:1082200030109DF854004030C1B25498C0EB00109B
:1082300000EB800002EBC000417041215498C0EB7C
:10824000001000EB800002EBC00081700521549803
:10825000C0EB001000EB800002EBC000C1700421F5
:108260000F9140F2231154984843994901EBC00003
:108270001830559901EBC10100EB0110007802287C
:108280000ED1032240F2231154984843904901EB48
:10829000C0001830559901EBC10100EB01100270CC
:1082A00062E202215498C0EB001000EB8000874A84
:1082B00002F830109DF854004030C1B25498C0EB21
:1082C000001000EB800002EBC00041704121549887
:1082D000C0EB001000EB800002EBC0008170312188
:1082E0005498C0EB001000EB800002EBC000C1709E
:1082F00032215498C0EB001000EB800002EBC0006C
:10830000017103215498C0EB001000EB800002EBD8
:10831000C00041715498C0EB001000EB8000114682
:1083200001EBC000401C05210490F1F7D3F8014691
:108330005498C0EB001000EB8000644A02EBC000D0
:10834000817107210F91549800EB400101EB00105F
:10835000604901EB00113031559801EB0010807835
:1083600020F02002549800EB400101EB0010594925
:1083700001EB00103030559900EB01108270F3E1F1
:1083800002215498C0EB001000EB80004F4A02F825
:1083900030109DF854004030C1B25498C0EB00102A
:1083A00000EB800002EBC000417041215498C0EB0B
:1083B000001000EB800002EBC00081703121549866
:1083C000C0EB001000EB800002EBC000C170302158
:1083D0005498C0EB001000EB800002EBC00001716C
:1083E00040F2231154984843394901EBC00018303A
:1083F000559901EBC10100EB01108068B0F5100F39
:1084000009D330215498C0EB001000EB800002EB40
:10841000C000417109E032215498C0EB001000EB1C
:1084200080002A4A02EBC000417140F223115498A7
:108430004843274901EBC0001830559901EBC101B1
:1084400000EB0110C07901280AD131215498C0EB0A
:10845000001000EB80001D4A02EBC000817118E0A3
:1084600040F2231154984843194901EBC0001830D9
:10847000559901EBC10100EB0110C07948B93221D7
:108480005498C0EB001000EB8000104A02EBC000D3
:10849000817100201A902FE040F223115498484334
:1084A0000B4901EBC0011831559800EBC00001EBFE
:1084B00000108168BDF86800C0F105008000C1406F
:1084C00001F00F013031549806E00000486F0020A1
:1084D000D445002014410020C0EB001000EB8000C8
:1084E000FE4A02EBC002BDF86800C01D1154BDF881
:1084F0006800401C81B21A91BDF868000628CBDBE9
:1085000032215498C0EB001000EB8000F34A02EBDC
:10851000C000417300211A9127E040F223115498C2
:108520004843EF4901EBC0011831559800EBC000FA
:1085300001EB0010416BBDF86800C0F10300800042
:10854000C14001F00F0130315498C0EB001000EB36
:108550008000E24A02EBC002BDF868000E30115400
:10856000BDF86800401C81B21A91BDF8680004286B
:10857000D3DB03225498C0EB001000EB8000D749F6
:1085800001EBC00082745498C0EB001000EB800037
:1085900001EBC000401C12210490F0F79BFF014644
:1085A0005498C0EB001000EB8000CC4A02EBC000F6
:1085B000C17414210F91D7E002215498C0EB001030
:1085C00000EB8000C54A02F830109DF8540040309E
:1085D000C1B25498C0EB001000EB800002EBC00069
:1085E000417041215498C0EB001000EB800002EB79
:1085F000C000817032215498C0EB001000EB800065
:1086000002EBC000C17031215498C0EB001000EBA8
:10861000800002EBC000017132215498C0EB0010C1
:1086200000EB800002EBC00041715498C0EB0010D9
:1086300000EB800002EBC000817100211A9127E05D
:1086400040F2231154984843A54901EBC001183169
:10865000559800EBC00001EB0010416BBDF86800BD
:10866000C0F103008000C14001F00F013031549887
:10867000C0EB001000EB8000984A02EBC002BDF88E
:108680006800C01D1154BDF86800401C81B21A91E9
:10869000BDF868000428D3DB00201A9011E03021D7
:1086A0005498C0EB001000EB80008C4A02EBC00233
:1086B000BDF868000B301154BDF86800401C81B251
:1086C0001A91BDF868001928E9DB03225498C0EB21
:1086D000001000EB8000814901EBC00080F82420ED
:1086E0005498C0EB001000EB800001EBC000401C70
:1086F00024210490F0F7EEFE01465498C0EB0010E0
:1087000000EB8000754A02EBC00080F8251026219E
:108710000F9129E010215498C0EB001000EB80006D
:108720006E4A02F8301030215498C0EB001000EB74
:10873000800002EBC000417002210F9114E0102173
:108740005498C0EB001000EB8000644A02F830102F
:1087500031215498C0EB001000EB800002EBC00008
:10876000417002210F9100BF00BF04F01DBB54985F
:1087700000EB400101EB00105A4901EB00113031D0
:10878000559801EB00104178159140F2231154984F
:108790004843534901EBC0011831559800EBC00024
:1087A00001EB0010017840F22312549850434C4AD8
:1087B00002EBC0004079814208D1012140F223122E
:1087C00054985043464A02EBC00001714649549800
:1087D00001EB00115598085C401CC1B2424A549804
:1087E00002EB0012559811549DF85400002804DD46
:1087F0009DF85400401EC1B215915698A1380A2820
:108800002FD2DFE800F0052FDFFDFCFBFA2E8CF9FC
:1088100004215498C0EB001000EB80002F4A02F8AE
:1088200030109DF854004030C1B25498C0EB001095
:1088300000EB800002EBC000417051215498C0EB66
:10884000001000EB800002EBC000817005215498FD
:10885000C0EB001000EB800002EBC000C1700421EF
:108860000F91F6E302215498C0EB001000EB80005A
:108870001A4A02F830109DF854004030C1B25498A2
:10888000C0EB001000EB800002EBC0004170412102
:108890005498C0EB001000EB800002EBC000817028
:1088A00031215498C0EB001000EB800002EBC000B7
:1088B000C17035215498C0EB001000EB800002EB32
:1088C000C000017103215498C0EB001000EB800040
:1088D00002EBC0004171549808E00000486F00208E
:1088E000D445002014410020483F0020C0EB001078
:1088F00000EB8000114601EBC000401C05210490F4
:10890000F0F7E8FD01465498C0EB001000EB800042
:10891000FB4A02EBC000817107210F9199E302210C
:108920005498C0EB001000EB8000F54A02F83010BC
:108930009DF854004030C1B25498C0EB001000EBD9
:10894000800002EBC000417041215498C0EB001040
:1089500000EB800002EBC000817032215498C0EB24
:10896000001000EB800002EBC000C1703021549871
:10897000C0EB001000EB800002EBC000017103218E
:108980005498C0EB001000EB800002EBC000417176
:108990005498C0EB001000EB8000114601EBC000C2
:1089A000401C05210490F0F795FD01465498C0EB5A
:1089B000001000EB8000D24A02EBC0008171072159
:1089C0000F9146E304215498C0EB001000EB8000A7
:1089D000CB4A02F830109DF854004030C1B2549890
:1089E000C0EB001000EB800002EBC00041704121A1
:1089F0005498C0EB001004E014E015E3FFE24FE2EE
:108A00007FE000EB800002EBC000817005215498EC
:108A1000C0EB001000EB800002EBC000C17004212D
:108A20000F9116E302215498C0EB001000EB800078
:108A3000B34A02F830109DF854004030C1B2549847
:108A4000C0EB001000EB800002EBC0004170412140
:108A50005498C0EB001000EB800002EBC000817066
:108A600031215498C0EB001000EB800002EBC000F5
:108A7000C17032215498C0EB001000EB800002EB73
:108A8000C000017103215498C0EB001000EB80007E
:108A900002EBC00041715498C0EB001000EB800065
:108AA000114601EBC000401C05210490F0F712FDB7
:108AB00001465498C0EB001000EB8000904A02EB96
:108AC000C0008171549800EB400101EB00108D490A
:108AD00001EB00113031559801EB0010807820F047
:108AE0002002549800EB400101EB0010854901EB96
:108AF00000113031559801EB0010827007210F9161
:108B0000A7E202215498C0EB001000EB80007C4AE1
:108B100002F830109DF854004030C1B25498C0EBB8
:108B2000001000EB800002EBC0004170412154981E
:108B3000C0EB001000EB800002EBC000817031211F
:108B40005498C0EB001000EB800002EBC000C17035
:108B500041215498C0EB001000EB800002EBC000F4
:108B6000017140F2231154984843674901EBC0005A
:108B70001830559901EBC10100EB01108068B0F18C
:108B8000104F09D130215498C0EB001000EB800049
:108B900002EBC000417109E032215498C0EB001093
:108BA00000EB8000564A02EBC000417140F22311F5
:108BB00054984843544901EBC0001830559901EBD3
:108BC000C10100EB0110C07901280AD1312154986C
:108BD000C0EB001000EB8000494A02EBC00081713D
:108BE00018E040F2231154984843474901EBC00074
:108BF0001830559901EBC10100EB0110C07948B95B
:108C000032215498C0EB001000EB80003C4A02EB8C
:108C1000C000817100201A9027E040F2231154987F
:108C20004843394901EBC0011831559800EBC000A9
:108C300001EB00108168BDF86800C0F107008000FA
:108C4000C14001F00F0130315498C0EB001000EB2F
:108C500080002B4A02EBC002BDF86800C01D115411
:108C6000BDF86800401C81B21A91BDF86800082860
:108C7000D3DB32215498C0EB001000EB8000204A77
:108C800002EBC000C17300211A9127E040F22311CA
:108C9000549848431C4901EBC0011831559800EB2A
:108CA000C00001EB0010416BBDF86800C0F1050089
:108CB0008000C14001F00F0130315498C0EB00102A
:108CC00000EB80000E4A02EBC002BDF868001030D5
:108CD0001154BDF86800401C81B21A91BDF86800BB
:108CE0000628D3DB30215498C0EB001000EB800045
:108CF000034A02EBC000817500211A9118E00000C0
:108D0000486F002014410020D445002030215498A1
:108D1000C0EB001000EB8000F94A02EBC002BDF886
:108D2000680017301154BDF86800401C81B21A91D8
:108D3000BDF868000628E9DB30215498C0EB00102C
:108D400000EB8000EE4A02EBC000417700211A914F
:108D500011E030215498C0EB001000EB8000E84A8D
:108D600002EBC002BDF868001E301154BDF8680067
:108D7000401C81B21A91BDF868000628E9DB302159
:108D80005498C0EB001000EB8000DD4A02EBC000FD
:108D900080F8241000211A9111E030215498C0EB82
:108DA000001000EB8000D64A02EBC002BDF868005C
:108DB00025301154BDF86800401C81B21A91BDF8ED
:108DC00068000628E9DB30215498C0EB001000EB66
:108DD0008000CB4A02EBC00080F82B1000211A91D2
:108DE00011E030215498C0EB001000EB8000C44A21
:108DF00002EBC002BDF868002C301154BDF86800C9
:108E0000401C81B21A91BDF868000628E9DB3021C8
:108E10005498C0EB001000EB8000B94A02EBC00090
:108E200080F8321000211A9111E030215498C0EBE3
:108E3000001000EB8000B24A02EBC002BDF86800EF
:108E400033301154BDF86800401C81B21A91BDF84E
:108E500068000628E9DB03225498C0EB001000EB01
:108E60008000A74901EBC00080F839205498C0EB7E
:108E7000001000EB800001EBC000401C3921049081
:108E8000F0F728FB01465498C0EB001000EB80007F
:108E90009B4A02EBC00080F83A103B210F91D8E0CA
:108EA00002215498C0EB001000EB8000944A02F8B5
:108EB00030109DF854004030C1B25498C0EB0010FF
:108EC00000EB800002EBC000417041215498C0EBE0
:108ED000001000EB800002EBC0008170322154983A
:108EE000C0EB001000EB800002EBC000C17031212C
:108EF0005498C0EB001000EB800002EBC000017141
:108F000033215498C0EB001000EB800002EBC0004E
:108F1000417132215498C0EB001000EB800002EB4D
:108F2000C000817100211A9127E040F2231154986A
:108F30004843744901EBC0011831559800EBC0005B
:108F400001EB0010416BBDF86800C0F10500800026
:108F5000C14001F00F0130315498C0EB001000EB1C
:108F60008000674A02EBC002BDF86800C01D1154C2
:108F7000BDF86800401C81B21A91BDF8680006284F
:108F8000D3DB00201A9011E030215498C0EB001080
:108F900000EB80005A4A02EBC002BDF868000D30B9
:108FA0001154BDF86800401C81B21A91BDF86800E8
:108FB0001928E9DB03225498C0EB001000EB800075
:108FC0004F4901EBC00080F826205498C0EB0010F8
:108FD00000EB800001EBC000401C26210490F0F75C
:108FE00079FA01465498C0EB001000EB8000444A27
:108FF00002EBC00080F8271028210F9129E01021F2
:109000005498C0EB001000EB80003D4A02F830108D
:1090100030215498C0EB001000EB800002EBC00040
:10902000417002210F9114E010215498C0EB001000
:1090300000EB8000324A02F8301031215498C0EB26
:10904000001000EB800002EBC000417002210F9184
:1090500000BF00BF03F0A8BE549800EB400101EB35
:109060000010294901EB00113031559801EB001037
:109070004178159140F2231154984843214901EB5E
:10908000C0011831BDF8680000EBC00001EB001012
:10909000017840F22312549850431A4A02EBC00060
:1090A0004079814208D1012140F223125498504363
:1090B000144A02EBC00001711449549801EB0011ED
:1090C0005598085C401CC1B2104A549802EB00123B
:1090D0005598115400211A911FE0549800EB40015B
:1090E00001EB0010084901EB00113031BDF86800B8
:1090F00001EB001041789DF85400814208D119E03D
:10910000486F0020D445002014410020483F002033
:10911000BDF86800401C81B21A91549800EB4001E0
:1091200001EB0010FE4901EB0010C179BDF86800A9
:109130008142D2DC00BF549800EB400101EB0010EB
:10914000F74901EB00113031BDF8680001EB001068
:1091500001785598401A401CC1B214919DF85400F2
:10916000002804DD9DF85400401EC1B2159140F264
:10917000231154984843EB4901EBC000183055992E
:1091800001EBC10100EB011040780F281EDA40F21C
:10919000231154984843E34901EBC0011831559815
:1091A00000EBC00001EB00104078401CC2B240F25E
:1091B000231154984843DB4901EBC00018305599FE
:1091C00001EBC10100EB011042700EE0002240F201
:1091D000231154984843D34901EBC00018305599E6
:1091E00001EBC10100EB011042705698B13809281B
:1091F00026D2DFE800F00526FD2525FC25B2FB0080
:109200009DF854005030C1B25498C0EB001000EBF0
:109210008000C54A02F8301020215498C0EB00109D
:1092200000EB800002EBC0004170FA215498C0EBC3
:10923000001000EB800002EBC000817003210F9151
:109240007EE29DF854005030C1B25498C0EB00103B
:1092500000EB8000B44A02F8301040F22311549819
:109260004843B04901EBC0011831559800EBC000EC
:1092700001EB0010407840F030015498C0EB001032
:1092800000EB800002EBC000417001215498C0EB5C
:10929000001000EB800002EBC00081705498C0EB1E
:1092A000001000EB800002EBC000C1700021549858
:1092B000C0EB001000EB800002EBC000017154987D
:1092C000C0EB001000EB8000114601EBC0010491DF
:1092D00005210498F0F72EFD0022CDE91002109828
:1092E000C2B25498C0EB001000EB80008E4901EB35
:1092F000C0004271DDE91001000A40EA0160C2B21B
:109300005498C0EB001000EB8000874901EBC000CF
:10931000827103225498C0EB001000EB800001EB37
:10932000C000C271FA225498C0EB001000EB80001C
:1093300001EBC000027209200F90B12240F223110C
:1093400054984843774901EBC0011831559800EB18
:10935000C00001EB00104271F2E19DF85400503062
:10936000C1B25498C0EB001000EB80006E4A02F8C6
:10937000301040F22311549848436A4901EBC00170
:109380001831559800EBC00001EB0010407840F018
:1093900030015498C0EB001000EB800002EBC000DD
:1093A000417065215498C0EB001000EB800002EB87
:1093B000C000817001215498C0EB001000EB8000C8
:1093C00002EBC000C1709DF850105498C0EB001023
:1093D00000EB800002EBC00001715498C0EB00105C
:1093E00000EB8000114601EBC00102E038E03CE1F7
:1093F000BEE0049105210498F0F79CFC0022CDE921
:1094000010021098C2B25498C0EB001000EB80001C
:10941000454901EBC0004271DDE91001000A40EA54
:109420000160C2B25498C0EB001000EB80003E49CE
:1094300001EBC000827103225498C0EB001000EBD6
:10944000800001EBC000C271FA225498C0EB0010FA
:1094500000EB800001EBC000027209200F906FE169
:109460009DF854005030C1B25498C0EB001000EB8E
:1094700080002D4A02F8301040F2231154984843DE
:10948000284901EBC0011831559800EBC00001EBF1
:109490000010407840F030015498C0EB001000EB11
:1094A000800002EBC000417065215498C0EB0010B1
:1094B00000EB800002EBC000817001215498C0EBEA
:1094C000001000EB800002EBC000C1709DF850005E
:1094D00040F010015498C0EB001000EB800002EB4C
:1094E000C00001715498C0EB001000EB80001146E1
:1094F00001EBC001049105210498F0F71BFC002248
:10950000CDE910021098C2B25498C0EB001000EBE5
:109510008000054901EBC0004271DDE9100105E062
:1095200014410020D4450020486F0020000A40EA82
:109530000160C2B25498C0EB001000EB8000FE49FD
:1095400001EBC000827103225498C0EB001000EBC5
:10955000800001EBC000C271FA225498C0EB0010E9
:1095600000EB800001EBC000027209200F90E7E0E1
:109570009DF854005030C1B25498C0EB001000EB7D
:109580008000ED4A02F8301040F22311549848430D
:10959000EA4901EBC0011831559800EBC00001EB1E
:1095A0000010407840F030015498C0EB001000EB00
:1095B000800002EBC000417001215498C0EB001004
:1095C00000EB800002EBC00081705498C0EB0010EB
:1095D00000EB800002EBC000C17005215498C0EB85
:1095E000001000EB800002EBC00001715498C0EB4A
:1095F000001000EB8000114601EBC0010491052131
:109600000498F0F797FB0022CDE910021098C2B23F
:109610005498C0EB001000EB8000C74901EBC0007C
:109620004271DDE91001000A40EA0160C2B25498BB
:10963000C0EB001000EB8000BF4901EBC00082715D
:1096400003225498C0EB001000EB800001EBC00037
:10965000C271FA225498C0EB001000EB800001EBBD
:10966000C000027209200F906AE040F22311549862
:109670004843B24901EBC0001830559901EBC101D4
:1096800000EB01108078B1282AD040F223115498C1
:109690004843AA4901EBC0011831559800EBC000BE
:1096A00001EB0010827840F2231154984843A349FB
:1096B00001EBC0011831559800EBC00001EB001020
:1096C0004271B12240F22311549848439B4901EB67
:1096D000C0001830559901EBC10100EB01108270F8
:1096E0009DF854005030C1B25498C0EB001000EB0C
:1096F0008000914A02F8301040F2231154984843F8
:109700008E4901EBC0011831559800EBC00001EB08
:109710000010407840F0C0015498C0EB001000EBFE
:10972000800002EBC0004170FA215498C0EB001099
:1097300000EB800002EBC000817003210F9100BF9D
:1097400000BF87E4012140F22312549850437B4A22
:1097500002EBC0000171A2F28C61549801EB001180
:109760005598085C401CC1B2A2F28C62549802EB7E
:10977000001255981154549800EB400101EB001071
:109780006F4901EB0010007B20B1012846D0022870
:1097900043D1AAE05698312802D045283CD11DE09B
:1097A00000201A9013E008A9BDF86800095C5498DD
:1097B000C0EB001000EB80005F4A02EBC002BDF876
:1097C00068001154BDF86800401C81B21A91BDF8C0
:1097D00068000728E7DB07200F901DE000201A90A3
:1097E00013E006A9BDF86800095C5498C0EB0010AE
:1097F00000EB8000504A02EBC002BDF86800115433
:10980000BDF86800401C81B21A91BDF868000728B5
:10981000E7DB07200F9000BF00BFD3E05598401C46
:10982000C1B215919DF854105498C0EB001000EB94
:109830008000414A02F8301003215498C0EB001018
:1098400000EB800002EBC000417000215498C0EB97
:10985000001000EB800002EBC000817002215498E0
:10986000C0EB001000EB800002EBC000C1700021D3
:109870005498C0EB001000EB800002EBC0000171B7
:1098800009215498C0EB001000EB800002EBC000EF
:1098900041715498C0EB001000EB8000114601EBC1
:1098A000C001049106210498EFF7F8FF0022CDE9EA
:1098B0001002DDE91020010641EA1220C2B25498DC
:1098C000C0EB001000EB80001B4901EBC000C2712F
:1098D0001098C2B25498C0EB001000EB800001EB6E
:1098E000C000827108200F906CE05598401CC1B2F6
:1098F00015919DF854105498C0EB001000EB8000B7
:109900000D4A02F8301003215498C0EB001000EB10
:10991000800002EBC000417000215498C0EB0010A1
:1099200000EB800002EBC00081705498C0EB001087
:1099300000EB800006E00000486F0020D4450020C6
:109940001441002002EBC000C1705498C0EB00101D
:1099500000EB800002EBC000017102215498C0EBC3
:10996000001000EB800002EBC00041715498C0EB86
:10997000001000EB8000114601EBC00104910621AC
:109980000498EFF78BFF0022CDE91002DDE91020EB
:10999000010641EA1220C2B25498C0EB001000EB5D
:1099A0008000FE4901EBC000C2711098C2B2549809
:1099B000C0EB001000EB800001EBC00082710820BA
:1099C0000F9000BF00BFBCE6549800EB400101EBD4
:1099D0000010F34901EB00113031559801EB0010F4
:1099E0004178159140F2231154984843ED4901EB19
:1099F000C0011831559800EBC00001EB0010017850
:109A000040F2231254985043E64A02EBC0004079DA
:109A1000814208D1012140F2231254985043E14A77
:109A200002EBC0000171E049549801EB0011559818
:109A3000085C401CC1B2DC4A549802EB00125598F5
:109A4000115440F2231154984843D64901EBC00009
:109A50001830559901EBC10100EB011090F8780026
:109A600000284FDD00201A9020E040F22311549886
:109A70004843CC4901EBC0011831BDF86800559A44
:109A8000104400EBC00001EB0010017840F22312FB
:109A900054985043C34A02EBC0004079814200D041
:109AA00017E0BDF86800401C81B21A9140F2231102
:109AB00054984843BB4901EBC0011831559800EB5D
:109AC000C00001EB001090F87810BDF868008142EA
:109AD000CBDC00BF40F2231154984843B14901EB5D
:109AE000C0011831559800EBC00001EB001090F850
:109AF0007810BDF86800814204D15698052801D03D
:109B0000062056905698F2287ED006DC05287CD098
:109B1000062809D0F12879D1C8E3F32877D0F428B2
:109B200076D0F628F7D1FDE340F22311549848434C
:109B30009C4901EBC0001830559901EBC10100EBC5
:109B4000011090F87800002873DD40F2231154983A
:109B50004843944901EBC0011831559800EBC0000F
:109B600001EB001090F87A109DF85400814238D033
:109B700040F22311549848438A4901EBC00118313F
:109B8000559800EBC00001EB001090F87B109DF899
:109B90005400814225D040F2231154984843814912
:109BA00001EBC0011831559800EBC00001EB00102B
:109BB00090F87C109DF85400814212D040F223119D
:109BC00054984843774901EBC0011831559800EB90
:109BD000C00001EB001090F87D109DF85400814208
:109BE00027D140F22311549848436E4901EBC0013C
:109BF0001831559800EBC00001EB001090F8781078
